:100000000C9428310C9459310C9459310C94593179
:100010000C9459310C94E59A0C9459310C94593143
:100020000C94769E0C9459310C9459310C94FDAC7F
:100030000C9459310D9455290C9459310C94593123
:100040000C9459310C94F5D30C9459310C945931CA
:100050000C9459310C9459310D948A200D94168BBF
:100060000C9459310D94B80F0C9459310C945931AA
:100070000C9459310C9459310C9459310C945931D8
:100080000C9459310C9459310C9459310C945931C8
:100090000D94740F0C9459310C9459310C945931BE
:1000A0000C9459310C9459310C9459310C945931A8
:1000B0000C9459310C9459310C9459310C94593198
:1000C0000C9459310C9459310C9459310C94E0B77B
:1000D0000C9459310C9459310C9459310C94593178
:1000E0000C9459315D89648925890E89EF885D8C6E
:1000F0008889B18A2F8B5D8C5D8C5D8C5D8C5D8C6D
:100100005D8CA08B5D8C5D8C5D8C5D8C5D8C5D8C65
:100110005D8C5D8C5D8C558C7CA880A886A88FA892
:10012000A7A8C4A801A938A979C48FC4A2C4AFC420
:10013000B9C4D1C4F2C4F8C406C51EC53AC544C585
:1001400055C566C56A0144018C016C0190014801E6
:100150004601DA019A01D801A8017E014C01A201F1
:100160003A0186013E0142016801CC019201800101
:100170005E01D00172013E018A01BC01BA01C201D7
:10018000B801C00150018201A4015A01BE01DE0183
:10019000640176015C019E01AA01A4019801CA01D3
:1001A0009601084AD73B3BCE016E84BCBFFDC12FF0
:1001B0003D6C74319ABD56833DDA3D00C77F11BE58
:1001C000D9E4BB4C3E916BAAAABE000000803F055B
:1001D000A84CCDB2D44EB93836A9020C50B991868C
:1001E00088083CA6AAAA2ABE000000803F076342F6
:1001F00036B79BD8A71A39685618AEBAAB558C1DBE
:100200003CB7CC5763BD6DEDFD753EF6177231BF3F
:10021000000000803F08000000BE922449123EAB5F
:10022000AAAA2ABECDCCCC4C3E00000080BEABAA10
:10023000AAAA3E00000000BF000000803F000000AE
:100240000000084178D3BB4387D1133D190E3CC34E
:10025000BD4282AD2B3E68EC8276BED98FE1A93ECD
:100260004C80EFFFBE01C4FF7F3F00000000000094
:100270000D94335D0D943E860D9490280D948286E6
:100280000D94018C0D944F860D94D5300D9415313D
:100290000D940F310D94139D0D944B860D942B5D91
:1002A0000D94B4880D943B640D948D8B0D9439643A
:1002B0000D940F5D0D94C8880D94F6880D94678693
:1002C0000D949E280D942F5D0D94E2880D94375D5A
:1002D0000D9453860D94C7300D94ED300D94366413
:1002E0000D940C280D946F860D9438640D94EC8851
:1002F0000D9462630D949CA20D94155D0D94488637
:100300000D9461860D94BE880D94175D0D944486FE
:100310000D9468630D9475860D94DB300D94C78B36
:100320000D9409310D945D860D94708B0D942D897B
:100330000D9419890D9431310D9417280D94058968
:100340000D9412280D943A860D9437890D94115D01
:100350000D9456310D940F890D94135D0D94218CDD
:100360000D9465630D9437640D9408280D943A64D8
:100370000D94A5880D947D860D9479860D94D08872
:100380000D94AA880D94A0880D94E48B0D94101000
:100390000D94BC2D0D9423890D9459860D945F63A3
:1003A0000D946B860D94108C0D94AA8B0D945C6348
:1003B0000D943F310D9423310D943B5D0D94D888FD
:1003C0006E616E00696E66004E414E494E49545949
:1003D000494E46CDCCCC3D0AD7233C17B7D1387710
:1003E000CC2B329595E6241FB14F0A000020410026
:1003F00000C84200401C4620BCBE4CCA1B0E5AAE70
:10040000C59D7400407A10F35A00A0724E1809007E
:1004100010A5D4E80000E87648170000E40B540269
:100420000000CA9A3B000000E1F5050000809698A4
:1004300000000040420F000000A0860100000010F4
:100440002700000000E80300000000640000000036
:10045000000A00000000000100000000002C76D817
:1004600088DC674F0823DFC1DFAE59E1B1B796E5FD
:10047000E3E453C63AE651997696E8E6C28426EB61
:10048000898C9B62ED407C6FFCEFBC9C9F40F2BA74
:10049000A56FA5F490055A2AF75C936B6CF9676D0C
:1004A000C11BFCE0E40D47FEF520E6B500D0ED9061
:1004B0002E0300943577050080841E080000204E2E
:1004C0000A000000C80C333333330F986E128311C7
:1004D00041EF8D2114893BE65516CFFEE6DB18D19E
:1004E000844B381BF77C1D901DA4BBE42420328470
:1004F000725E228100C9F124ECA1E53D27636469A5
:100500006E6F70737578585B00256420627974652E
:1005100073207772697474656E20746F204545503E
:10052000524F4D2061742061646472657373203092
:100530007825303478004433202D20526561642FB3
:10054000577269746520454550524F4D0A0020434B
:100550006F756E7420583A20005344207072696E93
:1005600074696E67206279746520004E6F7420692B
:100570006E206661726D206D6F64652E004163743C
:100580006976652045787472756465723A20004911
:100590006E76616C6964206578747275646572004A
:1005A000746D63323133305F73675F7468725B25DB
:1005B000635D3D25640A005A204F666673657400CA
:1005C000556E6B6E6F776E20636F6D6D616E643A02
:1005D0002022007A5F6D61783A20007A5F6D696E43
:1005E0003A2000795F6D61783A2000795F6D696E1D
:1005F0003A2000785F6D61783A2000785F6D696E0F
:100600003A20005265706F7274696E6720656E647F
:1006100073746F7020737461747573000053494C68
:10062000454E54004E4F524D414C002553204D4FE6
:1006300044453A2050657263656E7420646F6E6540
:100640003A2025643B207072696E742074696D6570
:100650002072656D61696E696E6720696E206D69D3
:100660006E733A2025640A00456E642066696C65E5
:10067000206C69737400426567696E2066696C65F9
:10068000206C6973740025643A2025640A000A50BE
:10069000494E44412074656D706572617475726570
:1006A0003A20252E3166205A207368696674202806
:1006B0006D6D293A20252E3366000A537465703A11
:1006C0002025642F360A000A537465703A20256489
:1006D0002F362028736B6970706564290A50494E63
:1006E00044412074656D70657261747572653A205D
:1006F0002564205A20736869667420286D6D293A34
:10070000300A000A5A45524F3A20252E33660A0015
:1007100073746172742074656D7065726174757242
:10072000653A20252E31660A0025642020252E32C8
:100730006600255320583A20252E356620593A2048
:10074000252E3566205A3A20252E35660A004E6F32
:100750007420696E206661726D206D6F64652E0075
:1007600025640045303A25642052504D0A50524EBF
:10077000303A25642052504D0A00256400417574BA
:100780006F0020452F443D00416476616E63652013
:100790004B3D004D323230205325690025534669C8
:1007A0006C616D656E742073657474696E67733AFD
:1007B0002044697361626C65640A00255346696C64
:1007C000616D656E742073657474696E67733A0A3F
:1007D00025532020204D3230302044252E32660A09
:1007E000002553526574726163743A20533D4C6521
:1007F0006E67746820286D6D2920463A53706565D0
:100800006420286D6D2F6D29205A3A205A4C696654
:100810007420286D6D290A25532020204D32303751
:100820002053252E32662046252E3266205A252E4C
:1008300032660A25535265636F7665723A20533DDE
:100840004578747261206C656E67746820286D6DE0
:100850002920463A537065656420286D6D2F6D29F7
:100860000A25532020204D3230382053252E326661
:100870002046252E32660A25534175746F2D526528
:1008800074726163743A20533D3020746F20646940
:100890007361626C652C203120746F20696E746501
:1008A000727072657420657874727564652D6F6EF0
:1008B0006C79206D6F766573206173207265747238
:1008C00061637473206F72207265636F76657269FD
:1008D00065730A25532020204D323039205325647A
:1008E0000A0025535049442068656174626564209C
:1008F00073657474696E67733A0A25532020204D1E
:100900003330342050252E32662049252E32662081
:1009100044252E32660A00255350494420736574DD
:1009200074696E67733A0A25532020204D333031A5
:100930002050252E32662049252E32662044252E51
:1009400032660A00255353746570732070657220F7
:10095000756E69743A0A255320204D393220582586
:100960002E32662059252E3266205A252E326620D8
:1009700045252E32660A25534D6178696D756D20C7
:10098000666565647261746573202D206E6F726D8B
:10099000616C20286D6D2F73293A0A255320204D54
:1009A0003230332058252E32662059252E326620CB
:1009B0005A252E32662045252E32660A25534D6172
:1009C00078696D756D206665656472617465732004
:1009D0002D20737465616C746820286D6D2F7329E8
:1009E0003A0A255320204D3230332058252E3266C6
:1009F0002059252E3266205A252E32662045252E76
:100A000032660A25534D6178696D756D20616363A7
:100A1000656C65726174696F6E202D206E6F726DEA
:100A2000616C20286D6D2F7332293A0A25532020DE
:100A30004D3230312058256C752059256C75205A5F
:100A4000256C752045256C750A25534D6178696DB7
:100A5000756D20616363656C65726174696F6E208A
:100A60002D20737465616C746820286D6D2F73324E
:100A7000293A0A255320204D3230312058256C75F3
:100A80002059256C75205A256C752045256C750AF2
:100A90002553416363656C65726174696F6E3A20BA
:100AA000533D616363656C65726174696F6E2C2080
:100AB000543D7265747261637420616363656C6533
:100AC000726174696F6E0A255320204D32303420D4
:100AD00053252E32662054252E32660A2553416452
:100AE00076616E636564207661726961626C6573BC
:100AF0003A20533D4D696E20666565647261746588
:100B000020286D6D2F73292C20543D4D696E207463
:100B1000726176656C206665656472617465202813
:100B20006D6D2F73292C20423D6D696E696D756D59
:100B3000207365676D656E742074696D6520286D1E
:100B400073292C20583D6D6178696D756D20585959
:100B5000206A65726B20286D6D2F73292C20205A16
:100B60003D6D6178696D756D205A206A65726B20E4
:100B7000286D6D2F73292C2020453D6D6178696D9E
:100B8000756D2045206A65726B20286D6D2F732965
:100B90000A255320204D3230352053252E32662031
:100BA00054252E32662042252E32662058252E32BC
:100BB000662059252E3266205A252E32662045257C
:100BC0002E32660A2553486F6D65206F6666736521
:100BD0007420286D6D293A0A255320204D32303675
:100BE0002058252E32662059252E3266205A252E71
:100BF00032660A004D4D55203C3D20274625642095
:100C00002564270A00504944204175746F74756E3D
:100C1000652066696E69736865642120507574206B
:100C2000746865206C617374204B702C204B6920B4
:100C3000616E64204B6420636F6E7374616E7473B5
:100C40002066726F6D2061626F766520696E746FC9
:100C500020436F6E66696775726174696F6E2E6886
:100C600000504944204175746F74756E652066614B
:100C7000696C6564212074696D656F75740020402E
:100C80003A00543A00423A00504944204175746F8A
:100C900074756E65206661696C6564212054656DAC
:100CA000706572617475726520746F6F2068696712
:100CB0006800204B643A2000204B693A2000204B0A
:100CC000703A200020436C6173736963205049447B
:100CD00020002054753A2000204B753A2000206DEA
:100CE00061783A2000206D696E3A200020643A2035
:100CF0000020626961733A200020453A00205A3A88
:100D00000020593A0020453A00205A3A0020593A2A
:100D100000583A00005A30005A3100593000593119
:100D200000583000583100456E642073746F707342
:100D30002064696167002E0044656C6574696F6E9C
:100D4000206661696C65642C2046696C653A2000F8
:100D500046696C652064656C657465643A004E6F25
:100D600074205344207072696E74696E670050720B
:100D7000696E7420736176656400534420707269F3
:100D80006E7420706175736564000A002F000A009C
:100D90002F2F20616374696F6E3A63616E63656CB7
:100DA0000043524153485F43414E43454C00435238
:100DB0004153485F5245434F5645520043524153B9
:100DC000485F5245434F564552002228322900546D
:100DD00000496E76616C6964205420636F64652EEF
:100DE00000556E6B6E6F776E204D20636F64653AB1
:100DF000202573200A006E6F2076616C6964206381
:100E00006F6D6D616E64002C20002C20002C200082
:100E10006E2F61002C20002C20002C20006E2F61F2
:100E2000002F00503A005761697420666F7220509D
:100E3000494E4441207461726765742074656D7019
:100E4000657261747572653A004C414E4720534596
:100E50004C20464F5243454400222831290030306F
:100E60003030303030302D303030302D3030303088
:100E70002D303030302D3030303030303030303078
:100E800030300020555549443A003100204558542F
:100E900052554445525F434F554E543A0050727577
:100EA0007361206933204D4B3300204D4143484945
:100EB0004E455F545950453A00312E300020626152
:100EC000736564206F6E204D61726C696E204649B7
:100ED000524D574152455F55524C3A687474707385
:100EE0003A2F2F6769746875622E636F6D2F707269
:100EF00075736133642F50727573612D4669726D1D
:100F0000776172652050524F544F434F4C5F5645A6
:100F10005253494F4E3A004649524D574152455F50
:100F20004E414D453A50727573612D4669726D7729
:100F300061726520004D31313320530020423A0068
:100F400020453A00543A0020413A0020503A00200F
:100F500042403A0020403A00202F003A002054003E
:100F6000202F0020423A00202F006F6B20543A00BF
:100F70002569206D696E2C20256920736563004901
:100F80006E76616C6964204D20636F64653A20253C
:100F900073200A00556E6B6E6F776E204720636F6B
:100FA00064653A202573200A004D657368206265E8
:100FB00064206C6576656C696E67206E6F74206165
:100FC00063746976652E000A002020000A4D656171
:100FD000737572656420706F696E74733A000A5A93
:100FE00020736561726368206865696768743A2078
:100FF000002C004E756D20582C593A2000206D6948
:1010000063726F6E730045786365737369766520EC
:10101000626564206C6576656C696E6720636F72CB
:1010200072656374696F6E3A20004732382057301A
:101030000050494E44412070726F62652063616CBC
:101040006962726174696F6E2073746172740047B3
:101050003238205730004D3234005345545F4348F6
:101060004F505F005345545F535445505F00534504
:10107000545F574156455F00544D435F0043524112
:1010800053485F005072657373206B6E6F622074FB
:101090006F2070726568656174206E6F7A7A6C6516
:1010A00020616E6420636F6E74696E75652E0050EA
:1010B0006C65617365207072657373207468652058
:1010C0006B6E6F6220746F20756E6C6F616420664A
:1010D000696C616D656E740052656D6F7665206F29
:1010E0006C642066696C616D656E7420616E64204D
:1010F000707265737320746865206B6E6F62207404
:101100006F207374617274206C6F6164696E672004
:101110006E65772066696C616D656E742E00616E18
:101120006420707265737320746865206B6E6F62E3
:1011300000496E736572742066696C616D656E74CA
:101140000046696C2E2073656E736F722072657332
:10115000706F6E736520697320706F6F722C2064DE
:10116000697361626C652069743F00436F6C6F72D4
:10117000206E6F7420636F72726563740046696CD1
:10118000616D656E74206E6F74206C6F6164656450
:10119000004368616E67656420636F727265637493
:1011A0006C793F004C6F6164696E6720636F6C6F90
:1011B00072004368616E676520737563636573735E
:1011C0002100506C65617365206F70656E206964E5
:1011D0006C657220616E642072656D6F7665206645
:1011E000696C616D656E74206D616E75616C6C7992
:1011F0002E005761732066696C616D656E74207591
:101200006E6C6F6164207375636365737366756C70
:101210003F00506C6561736520757067726164652D
:101220002E004E6577206669726D77617265207653
:10123000657273696F6E20617661696C61626C655D
:101240003A0057616974696E6720666F7220504971
:101250004E44412070726F626520636F6F6C696EDF
:1012600067004372617368206465746563746564C4
:101270002E20526573756D65207072696E743F0023
:1012800043726173682064657465637465642E00DD
:1012900045787472756465720043686F6F7365207A
:1012A00065787472756465723A0043686F6F736530
:1012B0002066696C616D656E743A004D3230302085
:1012C000496E76616C6964206578747275646572C4
:1012D00020006F70656E005452494747455245449F
:1012E000004E6F206D6F76652E0057616974206621
:1012F0006F7220757365722E2E2E00426564206C0D
:101300006576656C696E67206661696C65642E2020
:1013100053656E736F722074726967676572656476
:1013200020746F6F20686967682E2057616974693F
:101330006E6720666F722072657365742E00426559
:1013400064206C6576656C696E67206661696C65A2
:10135000642E2053656E736F7220646973636F6EC1
:101360006E6563746564206F72206361626C6520D2
:1013700062726F6B656E2E2057616974696E6720AB
:10138000666F722072657365742E00537461626CAF
:101390006520616D6269656E742074656D7065723B
:1013A00061747572652032312D32364320697320A5
:1013B0006E65656465642061207269676964207385
:1013C00074616E64206973207265717569726564F9
:1013D0002E00506C656173652072756E2058595AE5
:1013E0002063616C6962726174696F6E20666972F4
:1013F00073742E00536C6565702E2E2E007374610D
:1014000072740A006164635F696E69740A001B5B31
:10141000324A1B5B313B31484F726967696E616CC0
:101420002050727573612069331B5B323B33485027
:1014300072757361205265736561726368004661FD
:1014400063746F7279205245534554004E6F762075
:101450003131203230313800436F6D70696C656412
:101460003A2000286E6F6E652C2064656661756C8D
:101470007420636F6E66696729004E6F7620313184
:1014800020323031382030393A31373A3136002085
:10149000352E302E312D323133320A002055706C0A
:1014A0006F616420696E2070726F6772657373007C
:1014B000205A3A0020593A0020583A0043524153EA
:1014C000485F4445544543544544585900435241AC
:1014D00053485F44455445435445445900435241A1
:1014E00053485F444554454354454458004D3239B0
:1014F000005072757361206933204D4B3320726543
:101500006164792E00426C61636B6F7574206F6348
:101510006375727265642E205265636F7665722002
:101520007072696E743F0053656C667465737420E5
:1015300077696C6C2062652072756E20746F206311
:10154000616C696272617465206163637572617454
:10155000652073656E736F726C6573732072656856
:101560006F6D696E672E005468657265206973201F
:101570007374696C6C2061206E65656420746F20E3
:101580006D616B65205A2063616C69627261746978
:101590006F6E2E20506C6561736520666F6C6C6F8A
:1015A0007720746865206D616E75616C2C206368AE
:1015B000617074657220466972737420737465700B
:1015C000732C2073656374696F6E2043616C69626C
:1015D000726174696F6E20666C6F772E005072694D
:1015E0006E74657220686173206E6F742062656529
:1015F0006E2063616C6962726174656420796574E0
:101600002E20506C6561736520666F6C6C6F77205F
:10161000746865206D616E75616C2C206368617003
:101620007465722046697273742073746570732CCC
:101630002073656374696F6E2043616C69627261C7
:1016400074696F6E20666C6F772E004F6C64207328
:10165000657474696E677320666F756E642E2044BE
:10166000656661756C74205049442C20457374651F
:101670007073206574632E2077696C6C206265201E
:101680007365742E005761726E696E673A20626FDF
:101690007468207072696E74657220747970652048
:1016A000616E64206D6F74686572626F6172642030
:1016B00074797065206368616E6765642E00576198
:1016C000726E696E673A207072696E74657220740A
:1016D000797065206368616E6765642E005761727A
:1016E0006E696E673A206D6F74686572626F6172C1
:1016F000642074797065206368616E6765642E008C
:101700002020506C616E6E6572427566666572422D
:10171000797465733A20002046726565204D656DC9
:101720006F72793A2000204C6173742055706461A7
:101730007465643A2000506F776572557000457883
:101740007465726E616C2053504920666C617368D9
:1017500020573235583230434C206E6F74207265FA
:1017600073706F6E64696E672E006572726F72209F
:1017700077726974696E6720746F2066696C6500A2
:10178000656E6473746F7073206869743A20006FBB
:101790006B004372617368446574656374204449E7
:1017A0005341424C4544004372617368446574651B
:1017B000637420454E41424C45442100207C204129
:1017C0007574686F723A200020536F667477617287
:1017D0006520526573657400205761746368646F97
:1017E00067205265736574002042726F776E206FB8
:1017F0007574205265736574002045787465726E47
:10180000616C20526573657400446F6E652073616E
:1018100076696E672066696C652E0058595A206398
:10182000616C6962726174696F6E20616C6C2072A8
:10183000696768742E20536B65772077696C6C201C
:10184000626520636F72726563746564206175748C
:101850006F6D61746963616C6C792E0058595A2000
:1018600063616C6962726174696F6E20616C6C2077
:1018700072696768742E20582F592061786573202B
:1018800061726520736C696768746C7920736B652D
:101890007765642E20476F6F64206A6F622100585D
:1018A000595A2063616C6962726174696F6E206F4E
:1018B0006B2E20582F592061786573206172652046
:1018C00070657270656E646963756C61722E204319
:1018D0006F6E67726174756C6174696F6E732100ED
:1018E00058595A2063616C6962726174696F6E2025
:1018F0006661696C65642E2052696768742066723F
:101900006F6E742063616C6962726174696F6E20BE
:10191000706F696E74206E6F7420726561636861A8
:10192000626C652E0058595A2063616C696272615D
:1019300074696F6E206661696C65642E2046726FF3
:101940006E742063616C6962726174696F6E20707D
:101950006F696E7473206E6F742072656163686165
:10196000626C652E0058595A2063616C696272611D
:1019700074696F6E206661696C65642E20506C65B9
:1019800061736520636F6E73756C74207468652075
:101990006D616E75616C2E0058595A2063616C69D7
:1019A00062726174696F6E20636F6D70726F6D69C2
:1019B0007365642E2052696768742066726F6E7456
:1019C0002063616C6962726174696F6E20706F6907
:1019D0006E74206E6F7420726561636861626C65FD
:1019E0002E0058595A2063616C6962726174696F84
:1019F0006E20636F6D70726F6D697365642E204623
:101A0000726F6E742063616C6962726174696F6E6B
:101A100020706F696E7473206E6F742072656163DD
:101A20006861626C652E0058595A2063616C696266
:101A3000726174696F6E206661696C65642E204204
:101A400065642063616C6962726174696F6E207095
:101A50006F696E7420776173206E6F7420666F7586
:101A60006E642E00506C6561736520706C616365F7
:101A700020737465656C207368656574206F6E20D3
:101A8000686561746265642E0043616C69627261AD
:101A900074696E67205A0044697374616E636520CF
:101AA0006265747765656E20746970206F66207456
:101AB0006865206E6F7A7A6C6520616E6420746848
:101AC0006520626564207375726661636520686174
:101AD00073206E6F74206265656E20736574207963
:101AE00065742E20506C6561736520666F6C6C6F39
:101AF0007720746865206D616E75616C2C20636859
:101B000061707465722046697273742073746570B5
:101B1000732C2073656374696F6E204669727374E9
:101B2000206C617965722063616C696272617469AD
:101B30006F6E2E00206F66203400536561726368FB
:101B4000696E67206265642063616C6962726174AA
:101B5000696F6E20706F696E7400506C61636520F0
:101B600061207368656574206F66207061706572AE
:101B700020756E64657220746865206E6F7A7A6C69
:101B80006520647572696E67207468652063616C96
:101B90006962726174696F6E206F66206669727324
:101BA00074203420706F696E74732E20496620741F
:101BB0006865206E6F7A7A6C65206361746368650E
:101BC00073207468652070617065722C20706F7767
:101BD0006572206F666620746865207072696E7425
:101BE000657220696D6D6564696174656C792E003C
:101BF000506C6561736520636C65616E2074686507
:101C0000206E6F7A7A6C6520666F722063616C69F2
:101C100062726174696F6E2E20436C69636B20770A
:101C200068656E20646F6E652E00506C656173652B
:101C30002072656D6F766520737465656C207368BE
:101C40006565742066726F6D206865617462656495
:101C50002E00497320737465656C20736865657424
:101C6000206F6E20686561746265643F0041757421
:101C70006F20686F6D650078797A63616C5F6D6560
:101C80006173737572655F656E7465720A00787949
:101C90007A63616C5F73706972616C382063783D40
:101CA00025642063793D2564207A303D25642064D5
:101CB0007A3D2564207261646975733D25642061F5
:101CC000643D25640A0078797A63616C5F736561AD
:101CD0007263685A206E6F207369676E616C0A20A8
:101CE000783D256C6420793D256C64207A3D256C17
:101CF000640A00204F4E2D5349474E414C206174D9
:101D000020783D256420793D2564207A3D25642096
:101D100061643D25640A0078797A63616C5F73655C
:101D2000617263685A20783D256C6420793D256C8A
:101D300064207A3D256C640A000A00253032780060
:101D400078797A63616C5F7363616E5F70697865DF
:101D50006C735F33327833322063783D25642063BF
:101D6000793D2564206D696E5F7A3D2564206D6143
:101D7000785F7A3D25640A00202532642025640AB4
:101D8000000A002530327800206D696E3D25642000
:101D90006D61783D2564206469663D25640A006DA7
:101DA00061785F633D253264206D61785F6C3D250D
:101DB000640A006D61785F633D2564206D61785F22
:101DC000723D2564206D61785F6D617463683D25A7
:101DD000640A0020783D256420793D2564207A3D01
:101DE00025640A00207061747465726E20666F75D8
:101DF0006E642061742025642025640A000000F0D0
:101E000000F801FC03FE07FE07FE07FE07FC03F8CF
:101E100001F000000073697A656F6628746F746161
:101E20006C293D25640A0073697A656F6628626CC7
:101E30006F636B5F627566666572293D25640A0093
:101E400078797A63616C5F6D656173737572655FD4
:101E50006C656176650A00706F696E743D2564205B
:101E6000783D256420793D2564207A3D25640A006B
:101E700058025802584D584DB004F055F055B00472
:101E800078797A63616C5F66696E645F6265645FCE
:101E9000696E64756374696F6E5F73656E736F727C
:101EA0005F706F696E745F787920783D256C64206F
:101EB000793D256C64207A3D256C640A00203C2025
:101EC000005741524E494E473A2046726F6E742079
:101ED000706F696E74206E6F7420726561636861E3
:101EE000626C652E205920636F6F7264696E617435
:101EF000653A0000000040410000C04000005C4323
:101F00000000C04000005C43000046430000404128
:101F100000004643497465726174696F6E3A20002F
:101F200000007F43008058439AD95143FFFFFF438D
:101F3000616C6962726174696F6E206661696C655B
:101F4000642120436865636B20746865206178654F
:101F50007320616E642072756E20616761696E2EF8
:101F6000002563252D3138532563002563252E3147
:101F700035533A2573253364002563252E313253BA
:101F80003A25732500457872656D65207370616E22
:101F9000206F6620746865205A2076616C756573C1
:101FA000210000004041000000400000E442000029
:101FB000004000005743000000400000574300006D
:101FC000C4420000E4420000C4420000404100005E
:101FD000C44200004041000042430000E4420000CF
:101FE000424300005743000042436F6B0A00737482
:101FF0006172740A004D4D5532206669726D7761C9
:1020000072652076657273696F6E20696E76616C99
:1020100069642E20526571756972656420766572F7
:1020200073696F6E3A206275696C64206E756D62BB
:102030006572202564206F72206869676865722E5A
:1020400000666C0A006E6B0A0046530A0052300AA2
:102050000045340A0045330A0045320A0045310A7A
:102060000045300A0055300A0043300A004C340A5B
:10207000004C330A004C320A004C310A004C300A42
:102080000054340A0054330A0054320A0054310A0E
:102090000054300A004D4D55203D3E2027434D440D
:1020A000205245545259203078253258270A004D85
:1020B0004D55203D3E2027434D442041434B203089
:1020C00078253258270A004D4D55203D3E202745A2
:1020D00072726F20356D2054696D656F7574270AB3
:1020E000004D4D55203D3E20276669785468655067
:1020F000726F626C656D2121270A004D4D55203DA0
:102100003E20276F6B270A004D4D55203D3E20276E
:102110006F6B203A29270A004D4D55203D3E202760
:1021200077616974696E6720666F722066696C6199
:102130006D656E742040204D4B332053656E736F78
:1021400072270A004D363030004D36303020415570
:10215000544F004653454E534F525F5245434F56DE
:10216000455200256868750050300A0045450A0050
:102170004D4D55203C3D202746696C616D656E7460
:10218000207365656E20617420657874727564656E
:1021900072270A0045450A004D4D55203C3D202739
:1021A0005230270A0045450A004D4D55203C3D2040
:1021B00027452564270A0045450A004D4D55203C1A
:1021C0003D20275530270A0045450A004D4D552032
:1021D0003C3D20274330270A0045450A004D4D5518
:1021E000203C3D20274C2564270A0045450A004530
:1021F000450A004D4D55203C3D2027542564270AB3
:102200000046530A0052300A0045340A0045330A9A
:102210000045320A0045310A0045300A0055300AAF
:102220000043300A004C340A004C330A004C320A96
:10223000004C310A004C300A0054340A0054330A6E
:102240000054320A0054310A0054300A004D4D55F2
:10225000202D20454E41424C4544002568687500BC
:1022600050300A0050300A004D4D5520766572738B
:10227000696F6E2076616C69640025750053320ABF
:10228000002575004D4D55206E6F7420726573707A
:102290006F6E64696E67202D2044495341424C455E
:1022A000440053310A00205B6F66665D004265643E
:1022B000206C6576656C696E67206661696C656423
:1022C0002E2053656E736F72206469646E7420747F
:1022D0007269676765722E20446562726973206F48
:1022E0006E206E6F7A7A6C653F2057616974696EF3
:1022F0006720666F722072657365742E00206F66AA
:102300002039004D6561737572696E67207265666C
:102310006572656E636520686569676874206F66BD
:102320002063616C6962726174696F6E20706F699D
:102330006E7400506C6561736520757064617465BE
:10234000206669726D7761726520696E20796F759C
:1023500072204D4D55322E2057616974696E672089
:10236000666F722072657365742E004B494C4C4544
:10237000442E20005072696E7465722068616C741E
:1023800065642E206B696C6C28292063616C6C6518
:102390006421004D31303420496E76616C696420CF
:1023A000657874727564657220004D31303520494E
:1023B0006E76616C696420657874727564657220EC
:1023C000004D31303920496E76616C696420657842
:1023D00074727564657220004D32313820496E7612
:1023E000616C696420657874727564657220004D53
:1023F00032323120496E76616C696420657874727E
:102400007564657220005265636F766572696E67E8
:10241000207072696E7420202020004B494C4C3A89
:102420002025640A0055564C4F202D20656E6420EF
:1024300025640A007374707325640A00776F726CE8
:102440006420636F6F7264696E617465733A2028EB
:10245000252E33662C20252E33662C20252E336620
:10246000290A00706879736963616C20636F6F7209
:1024700064696E617465733A2028252E33662C20BA
:10248000252E33662C20252E3366290A00437572CB
:1024900072656E7420706F73205A5F415849533AC9
:1024A000252E33660A43757272656E7420706F73E1
:1024B00020455F415849533A252E33660A0041664C
:1024C0007465722077616974696E6720666F722027
:1024D00074656D703A0A43757272656E7420706F20
:1024E0007320585F415849533A252E33660A437585
:1024F0007272656E7420706F7320595F4158495332
:102500003A252E33660A0020573A0020453A0054F7
:102510003A005A206C6976652061646A757374208C
:102520006F7574206F662072616E67652E2053652B
:102530007474696E6720746F20302E20436C696359
:102540006B20746F20636F6E74696E75652E005A10
:10255000206C6976652061646A757374206F757488
:10256000206F662072616E67652E205365747469F2
:102570006E6720746F20300020423A0020453A00F8
:10258000543A00494E5434007265636F7665725F49
:102590006D616368696E655F73746174655F6166C0
:1025A0007465725F706F7765725F70616E69632CBE
:1025B00020696E697469616C20007265636F76656D
:1025C000725F6D616368696E655F73746174655F86
:1025D00061667465725F706F7765725F70616E6956
:1025E000632C20696E697469616C20004739322060
:1025F000450050525553412075766C6F004734208A
:102600005330004D32362053256C75004D31303635
:102610002053004D383200473120462564004731B1
:102620002045322A64656661756C745F72657472E8
:10263000616374696F6E2046343830004731205A28
:1026400000204632303030002059004731205800F9
:102650004D383300506F736974696F6E2072656115
:10266000642066726F6D20656570726F6D3A004D03
:102670003233202573002E67636F004665656472F0
:102680006174653A00473120452D64656661756C5B
:10269000745F72657472616374696F6E204634385A
:1026A000300047312045352046313230004D383337
:1026B000004D31393020532564004D3130392053DD
:1026C00025640047323820582059004731205A32BB
:1026D000352046383030006673656E736F725F73F5
:1026E000746F705F616E645F736176655F7072694D
:1026F0006E740A006673656E736F725F72657374D1
:102700006F72655F7072696E745F616E645F636F34
:102710006E74696E75650A0044495341424C4544E4
:102720000A00454E41424C4544004653656E736F66
:10273000722025530A00504154393132355F696E99
:1027400069743A256868750A005041543931323548
:102750005F696E69743A256868750A00504154399A
:102760003132355F696E69743A256868750A0066AA
:1027700073656E736F725F6F715F6D656173737593
:1027800072655F73746172740A006673656E736F4D
:10279000725F6F715F6D656173737572655F73747E
:1027A0006F702C20256868752073616D706C65737F
:1027B0000A004E4721004F4B005041543931323509
:1027C000206E6F7420726573706F6E64696E67201F
:1027D00028256429210A00000E1315110E0000009F
:1027E00004120912040000001C1F11111F00000038
:1027F00006191803130C00040E1F041C000000042B
:102800000A0A0A0A11110E001F1511151F000000F7
:102810000103161C0800000000110A04110A040C30
:1028200012120C000000006673656E736F725F61B8
:1028300075746F6C6F61645F636865636B5F7374FD
:10284000617274202D206175746F6C6F6164204516
:102850004E41424C45440A006673656E736F725F69
:102860006175746F6C6F61645F636865636B5F73E0
:10287000746F70202D206175746F6C6F61642044DB
:10288000495341424C45440A002079645F6D696EAA
:102890003D25752079645F6D61783D2575207964EB
:1028A0005F6176673D25752073685F6176673D25BA
:1028B000750A002073745F73756D3D25752079640A
:1028C0005F73756D3D25752065725F73756D3D2570
:1028D000752065725F6D61783D256868750A0066D0
:1028E00073656E736F725F6F715F726573756C7411
:1028F0002025530A002073685F617667203D2025FC
:102900006868752025530A002079645F717561201D
:102910003D2025752025530A002079645F64657683
:10292000203D2025750A002079645F6D696E203D89
:102930002025752025530A002079645F6D61782079
:102940003D2025752025530A002079645F61766754
:10295000203D20256868752025530A002065725F98
:102960006D6178203D20256868752025530A002078
:1029700065725F73756D203D2025752025530A0013
:102980006673656E736F725F6F715F726573756C7E
:10299000740A00544D4320445249564552204F5624
:1029A000455254454D50005A25362E326620005A65
:1029B0002020202D2D2D200025632533642F256414
:1029C00025630025632533642525002D2D2D002545
:1029D000336868640025335325337325250020535D
:1029E000440020202000555342002025753E2575C7
:1029F00000204625750020463020200025632D2D1F
:102A00003A2D2D2020002563253032753A253032AD
:102A1000752563256300726573756C742076616C2F
:102A200075653A2025640A0020693D2532642063DB
:102A30006E743D2532642076616C3D2532640A0057
:102A4000636C7573746572733A0A0020693D2532B0
:102A50006420737465703D2532640A00736F72746C
:102A600065642073616D706C65733A0A005553415B
:102A70005254322072782046756C6C2121210A0054
:102A80003A2000202020202020202020202020204C
:102A900020202020202000203A200020202020205C
:102AA0002020202020202020202020202020200046
:102AB00020202020202020202020202020002573DE
:102AC0000050494E44412048656174696E67005466
:102AD000656D702E2063616C2E2020202020202028
:102AE0002020200043616C6962726174696F6E20FE
:102AF000646F6E650042656420646F6E65004265B8
:102B0000642048656174696E670048656174696E28
:102B10006720646F6E652E0048656174696E67009A
:102B2000473830004D3435004D3435205A00473792
:102B3000360057697A6172642073746174653A2053
:102B400025640044697361626C65206661726D2062
:102B50006D6F6465004661726D206E756D626572A1
:102B6000004D3834004D3434004732382057004788
:102B700039390044697361626C65206661726D2049
:102B80006D6F64653F0043616C69627261746500DA
:102B9000506C65617365206C6F616420504C4120FE
:102BA00066696C616D656E742066697273742E005F
:102BB000497320504C412066696C616D656E7420CC
:102BC0006C6F616465643F0043616E63656C0046D1
:102BD000696C616D656E740053656C65637420503B
:102BE0004C412066696C616D656E743A0052756E79
:102BF0006E696E672057697A6172642077696C6CC0
:102C00002064656C6574652063757272656E7420EE
:102C100063616C6962726174696F6E20726573754D
:102C20006C747320616E64207374617274206672B8
:102C30006F6D2074686520626567696E6E696E6786
:102C40002E20436F6E74696E75653F005072656823
:102C5000656174696E67206E6F7A7A6C652E20509C
:102C60006C6561736520776169742E00596F7520FA
:102C700063616E20616C7761797320726573756D25
:102C800065207468652057697A6172642066726F86
:102C90006D2043616C6962726174696F6E202D3EB4
:102CA0002057697A6172642E00506C6561736520EB
:102CB000636865636B206F75722068616E64626F14
:102CC0006F6B20616E64206669782074686520707F
:102CD000726F626C656D2E205468656E207265732C
:102CE000756D65207468652057697A617264206229
:102CF00079207265626F6F74696E672074686520F1
:102D00007072696E7465722E00416C6C206973205C
:102D1000646F6E652E204861707079207072696EE4
:102D200074696E672100506C6561736520636C6522
:102D3000616E206865617462656420616E642074F0
:102D400068656E20707265737320746865206B6EA1
:102D50006F622E00446F20796F752077616E74204A
:102D6000746F20726570656174206C617374207378
:102D700074657020746F20726561646A7573742065
:102D800064697374616E6365206265747765656EEE
:102D9000206E6F7A7A6C6520616E6420686561745C
:102DA0006265643F00492077696C6C2073746172BE
:102DB0007420746F207072696E74206C696E652067
:102DC000616E6420796F752077696C6C2067726121
:102DD0006475616C6C79206C6F77657220746865BE
:102DE000206E6F7A7A6C6520627920726F746174DC
:102DF000696E6720746865206B6E6F622C20756E3B
:102E000074696C20796F75207265616368206F70DA
:102E100074696D616C206865696768742E20436809
:102E200065636B207468652070696374757265737F
:102E300020696E206F75722068616E64626F6F6BBF
:102E400020696E20636861707465722043616C69EB
:102E500062726174696F6E2E004E6F772049207721
:102E6000696C6C2063616C6962726174652064696D
:102E70007374616E6365206265747765656E207436
:102E80006970206F6620746865206E6F7A7A6C6551
:102E900020616E6420686561746265642073757278
:102EA000666163652E00497320697420504C41208F
:102EB00066696C616D656E743F004C6F6164696E2C
:102EC000672066696C616D656E7400506C65617336
:102ED0006520696E7365727420504C412066696C80
:102EE000616D656E7420746F2074686520657874F8
:102EF00072756465722C207468656E2070726573DB
:102F000073206B6E6F6220746F206C6F6164206938
:102F1000742E00506C6561736520696E7365727400
:102F200020504C412066696C616D656E7420746F31
:102F300020746865206669727374207475626520F8
:102F40006F66204D4D552C207468656E207072653B
:102F5000737320746865206B6E6F6220746F206CD1
:102F60006F61642069742E00456A65637400556E54
:102F70006C6F61640055736520756E6C6F616420C1
:102F8000746F2072656D6F76652066696C616D6522
:102F90006E7420312069662069742070726F7472BB
:102FA00075646573206F757473696465206F66203E
:102FB0007468652072656172204D4D55207475628C
:102FC000652E2055736520656A65637420696620E7
:102FD00069742069732068696464656E20696E2075
:102FE000747562652E0053656C656374206E6F7A2C
:102FF0007A6C6520707265686561742074656D70A7
:1030000065726174757265207768696368206D61A7
:10301000746368657320796F7572206D6174657271
:1030200069616C2E004E6F7720492077696C6C20A7
:1030300070726568656174206E6F7A7A6C6520665F
:103040006F7220504C412E0049732066696C616D8F
:10305000656E74206C6F616465643F00497320661F
:10306000696C616D656E742031206C6F616465649C
:103070003F00492077696C6C2072756E207A20635E
:10308000616C6962726174696F6E206E6F772E0079
:10309000492077696C6C2072756E2078797A20638C
:1030A000616C6962726174696F6E206E6F772E2039
:1030B00049742077696C6C2074616B652061707055
:1030C000726F782E203132206D696E732E00466942
:1030D0007273742C20492077696C6C2072756E2095
:1030E0007468652073656C667465737420746F20F2
:1030F000636865636B206D6F737420636F6D6D6FB4
:103100006E20617373656D626C792070726F626C92
:10311000656D732E0048692C204920616D20796F00
:103120007572204F726967696E616C205072757399
:1031300061206933207072696E7465722E20576F3A
:10314000756C6420796F75206C696B65206D6520E6
:10315000746F20677569646520796F752074687273
:103160006F7567682074686520736574757020706A
:10317000726F636573733F00452D636F7272656391
:1031800074005A2D636F727265637400592D636FFA
:10319000727265637400582D636F72726563740098
:1031A000536F756E642020202020205B6C6F756447
:1031B0005D00536F756E642020202020205B6D75AC
:1031C00074655D00536F756E64202020205B736909
:1031D0006C656E745D00536F756E64202020202036
:1031E000205B6F6E63655D00536F756E64202020F9
:1031F0002020205B6C6F75645D00536F72743A2001
:1032000020202020205B6E6F6E655D00536F72740E
:103210003A20205B616C7068616265745D00536F79
:1032200072743A2020202020205B74696D655D0057
:103230005344206361726420205B6E6F726D616C19
:103240005D0053442063617264205B666C73684167
:1032500069725D0052506920706F727420202020C6
:10326000205B6F6E5D0052506920706F7274202079
:1032700020205B6F66665D0054656D702E20636173
:103280006C2E2020205B6F6E5D0054656D702E20CB
:1032900063616C2E20205B6F66665D004C696E2E4C
:1032A00020636F7272656374696F6E0046616E733E
:1032B00020636865636B20205B6F66665D00466116
:1032C0006E7320636865636B2020205B6F6E5D000A
:1032D0004175746F206465706C6574655B6F6666BC
:1032E0005D004175746F206465706C657465205B6A
:1032F0006F6E5D00462E204F51206D656173732EF9
:103300005B6F66665D00462E204F51206D656173D0
:10331000732E205B6F6E5D00462E206175746F6C9E
:103320006F6164205B6F66665D00462E2061757478
:103330006F6C6F616420205B6F6E5D00462E2061B4
:1033400075746F6C6F6164205B4E2F415D00466940
:103350006C2E2073656E736F72205B4E2F415D0083
:1033600044697361626C6520737465707065727313
:10337000004D6F766520617869730054656D7065E6
:103380007261747572650054656D702E2063616C96
:103390006962726174696F6E00526573657420585A
:1033A000595A2063616C6962722E0053686F7720EE
:1033B00070696E64612073746174650050494420C3
:1033C00063616C6962726174696F6E00426564204A
:1033D0006C6576656C20636F7272656374004D6511
:1033E000736820426564204C6576656C696E670081
:1033F00043616C696272617465205A0043616C6953
:1034000062726174652058595A0053656C66746520
:103410007374202020202020202020004669727311
:1034200074206C617965722063616C2E0057697A33
:10343000617264004C6F61642066696C616D656ED9
:10344000742035004C6F61642066696C616D656E37
:10345000742034004C6F61642066696C616D656E28
:10346000742033004C6F61642066696C616D656E19
:10347000742032004C6F61642066696C616D656E0A
:10348000742031004C6F616420616C6C00456A658A
:1034900063742066696C616D656E74203500456AE1
:1034A0006563742066696C616D656E7420340045D7
:1034B0006A6563742066696C616D656E74203300A3
:1034C000456A6563742066696C616D656E7420324F
:1034D00000456A6563742066696C616D656E742071
:1034E0003100556E6C6F61642066696C616D656E4C
:1034F00074203500556E6C6F61642066696C616D77
:10350000656E74203400556E6C6F61642066696C62
:10351000616D656E74203300556E6C6F616420665A
:10352000696C616D656E74203200556E6C6F6164FC
:103530002066696C616D656E74203100556E6C6F2C
:10354000616420616C6C00457874727564657220EA
:103550003400457874727564657220330045787460
:103560007275646572203200457874727564657294
:10357000203100506C656173652070756C6C206F34
:1035800075742066696C616D656E7420696D6D651A
:1035900064696174656C7900556E6C6F6164696E05
:1035A000672066696C616D656E740057697A617237
:1035B0006420656E642073746174653A2025640A22
:1035C0000046696C2E2058643A2533642059643AC9
:1035D0002533640A496E743A2025336420205368E9
:1035E00075743A202533640046696C616D656E74AC
:1035F0002073656E736F720A697320646973616208
:103600006C65642E001B5B303B30484E6F7A7A6CE1
:10361000652046414E3A202534642052504D0A50D0
:1036200072696E742046414E3A202025346420523F
:10363000504D0A001B5B324A2553203A1B5B313B3D
:10364000394825382E3266206D0A2553203A0A253E
:10365000376C6464203A253268686468203A253003
:1036600032686864206D001B5B324A25533A1B5B4D
:10367000313B364825382E32666D200A2553203AD4
:103680001B5B333B38482532646820253032646D3B
:103690002025303264730025362E32666D6D004E63
:1036A0002F41001B5B303B304825533A0A25530A13
:1036B00025533A0A25533A001B5B303B3135484EBF
:1036C0002F41001B5B303B31354825342E326601DB
:1036D000001B5B303B304825533A0A25530A2553DB
:1036E0003A202025352E3266010A25533A2020251E
:1036F000352E326601001B5B303B3048546F7461DD
:103700006C206661696C757265731B5B313B314877
:10371000506F776572206661696C757265732020E1
:10372000252D33641B5B323B314846696C616D2E3D
:103730002072756E6F7574732020252D33641B5BAA
:10374000333B3148437261736820205820252D3364
:103750006420205920252D3364001B5B303B30480A
:103760004C617374207072696E74206661696C7547
:103770007265731B5B313B3148506F776572206611
:1037800061696C757265732020252D33641B5B3273
:103790003B314846696C616D2E2072756E6F757491
:1037A000732020252D33641B5B333B31484372610A
:1037B000736820205820252D336420205920252D82
:1037C000336400546F74616C004C617374207072C8
:1037D000696E74001B5B323B3148416D6269656EF6
:1037E000743A2020256425631B5B333B31485049E4
:1037F0004E44413A2020202025642563001B5B3085
:103800003B31484E6F7A7A6C653A2020202564253A
:10381000631B5B313B31484265643A202020202005
:103820002025642563001B5B313B31485057523AD9
:1038300020202020202025642E2530316456001BB6
:103840005B303B314842656C7420737461747573EE
:103850001B5B313B3248582025641B5B323B3248AE
:103860005920256400464C4558202D202032343004
:103870002F35300050502020202D20203235342F7D
:103880003130300048495053202D20203232302F23
:103890003130300041425320202D20203235352F49
:1038A0003130300050455420202D20203233302F2D
:1038B000383500504C4120202D20203231352F3614
:1038C0003000414253202020202D20203235352F3A
:1038D000313030006E6F7A7A6C65202D20203235C1
:1038E000302F30006661726D2020202D202032356F
:1038F000302F363000466C61736841697220495040
:1039000020416464723A004D4D5532202020202021
:1039100020204E2F4100756E6B6E6F776E00256410
:103920002E25642E25642D2564002046573A004D2F
:103930004D553220636F6E6E6563746564004E6F23
:1039400076203131203230313800453344763666C6
:10395000756C6C0045494E53795F31306100315FC1
:1039600037356D6D5F4D4B33002D2D2D2D2D2D2DAC
:103970002D2D2D2D2D00207265706F20556E6B6ED4
:103980006F776E0020352E302E312D3231333200DC
:103990004669726D776172653A0025642E25642E42
:1039A00025642E2564004D373032004D373031000C
:1039B0004578747275646572006D6D000059005829
:1039C00000580059005A002563252E3132533A25FC
:1039D00073252B30362E336600436F6F6C646F7720
:1039E0006E00566F6C74616765730054656D706529
:1039F000726174757265730042656C7420737461D2
:103A000074757300457874727564657220696E66AA
:103A10006F0058595A2063616C2E20646574616987
:103A20006C7300446174653A00686F77746F2E7030
:103A30007275736133642E636F6D00666F72756D9E
:103A40002E707275736133642E636F6D00707275C2
:103A5000736133642E636F6D004175746F6C6F61B9
:103A600064696E672066696C616D656E7420697348
:103A7000206163746976652C206A75737420707296
:103A800065737320746865206B6E6F6220616E646D
:103A900020696E736572742066696C616D656E7401
:103AA0002E2E2E00546F74616C207072696E74201B
:103AB00074696D6500546F74616C2066696C616D2A
:103AC000656E74005072696E742074696D6500468D
:103AD000696C616D656E7420757365640050726504
:103AE0006865617420746865206E6F7A7A6C6521F0
:103AF000004552524F523A005269676874004C6553
:103B0000667400592064697374616E63652066721F
:103B10006F6D206D696E0053657665726520736BFD
:103B2000657700536C6967687420736B6577004D27
:103B30006561737572656420736B6577005B303BFC
:103B4000305D20706F696E74206F666673657400F7
:103B500041646A757374696E67205A0052657365B3
:103B60007400526561722073696465205B756D5DD8
:103B70000046726F6E7420736964655B756D5D00DD
:103B8000526967687420736964655B756D5D004C8C
:103B90006566742073696465205B756D5D005365AF
:103BA000742074656D70657261747572653A002475
:103BB000F4D43050C38E20C2A24017828B701112F1
:103BC0007A910D816CD90AA861E108C7586607612E
:103BD0005143061E4B5D05C145A7041A4111040956
:103BE0003D9803713931034036DB0265339102D4CD
:103BF000305402802E1D02632CEE01752AC501B0DF
:103C000028A001102781018F2564012B244B01E09E
:103C1000223401AC211F018D200D01801FFC008486
:103C20001EED00971DDF00B81CD200E61BC6002069
:103C30001BBC00641AB200B219A8000A19A0006ADD
:103C4000189900D117910040178B00B516840031E8
:103C5000167E00B31579003A157300C7146F00582B
:103C6000146A00EE1366008813630025135E00C714
:103C7000125B006C12570015125400C111510070F4
:103C8000114F0021114B00D61049008D10470046FE
:103C900010440002104200C00F4000800F3E00425E
:103CA0000F3C00060F3B00CB0E3800930E37005C34
:103CB0000E3500270E3400F30D3200C10D31009097
:103CC0000D3000600D2E00320D2D00050D2C00D999
:103CD0000C2B00AE0C2900850C29005C0C2700354C
:103CE0000C27000E0C2600E80B2400C40B2400A0B7
:103CF0000B23007D0B23005A0B2100390B210018E8
:103D00000B2000F80A1F00D90A1E00BB0A1E009DE6
:103D10000A1D00800A1D00630A1C00470A1B002CB4
:103D20000A1B00110A1A00F7091A00DD091900C45C
:103D3000091900AB091900920917007B09180063E3
:103D40000917004C09160036091600200916000A4A
:103D5000091500F5081500E0081400CC081400B897
:103D6000081400A4081400900813007D0812006BCA
:103D700008130058081200460812003408110023E6
:103D80000811001208110001081100F0071000E0EE
:103D9000071000D0071000C0071000B0070F00A1E7
:103DA00007100091070E0083070F0074070F0065CE
:103DB000070E0057070E0049070E003B070D002EA7
:103DC000070E0020070D0013070D0006070D00F970
:103DD000060C00ED060D00E0060C00D4060C00C831
:103DE000060C00BC060C00B0060C00A4060B0099E3
:103DF000060C008D060B0082060B0077060B006C8C
:103E0000060B0061060A0057060B004C060A00422A
:103E1000060A0038060A002E060A0024060A001ABE
:103E2000060A001006090007060A00FD050900F44D
:103E3000050900EB050900E2050900D9050900D0D4
:103E4000050900C7050900BE050900B5050800AD54
:103E5000050800A50509009C050800940508008CCC
:103E6000050800840508007C050800740508006C3E
:103E7000050700650508005D050700560508004EAA
:103E80000507004705070040050800380507003111
:103E90000507002A050700230507001C0506001674
:103EA0000507000F0507000805060002050700FBCF
:103EB000040600F5040700EE040600E8040600E22C
:103EC000040700DB040600D5040600CF040600C981
:103ED000040600C3040600BD040600B7040600B1D2
:103EE000040500AC040600A6040600A00405009B1F
:103EF00004060095040500900406008A0405008568
:103F0000040500800406007A0405007504050070AD
:103F10000405006B04050066040500610405005CEF
:103F200004050057040500520405004D040500482F
:103F3000040500430405003E0404003A040500356E
:103F4000040500300404002C0405002704040023A9
:103F50000405001E0404001A0404001604050011E0
:103F60000404000D04040009040500040404000016
:103F7000040400FC030400F8030400F4030400F04C
:103F8000030400EC030400E8030400E4030400E07D
:103F9000030400DC030400D8030400D4030400D0AD
:103FA000030400CC030400C8030300C5030300247A
:103FB000F404D9201BC40C5C0E9804C4095F02658C
:103FC000077101F405F900FB04B30048048700C140
:103FD0000369005803550003034500BE023A0084FC
:103FE00002310053022A002902250004022000E4C5
:103FF000011C00C8011900AF0117009801140084CA
:10400000011300710110006101100051010E004305
:10401000010D0036010B002B010B0020010B0015D8
:104020000109000C01090003010800FB000800F36E
:10403000000800EB000700E4000600DE000600D8E0
:10404000000600D2000600CC000500C7000500C233
:10405000000500BD000400B9000400B5000400B173
:10406000000400AD000400A9000400A5000300A2A4
:104070000003009F0004009B0003009800030095CC
:1040800000020093000300900003008D0002008BEB
:104090000003008800020086000200840003008103
:1040A0000002007F0002007D0002007B0002007918
:1040B0000002007700010076000200740002007226
:1040C000000100710002006F0002006D0001006C31
:1040D0000002006A0001006900020067000100663A
:1040E000000100650001006400020062000100613F
:1040F000000100600001005F0002005D0001005C43
:104100000001005B0001005A000100590001005845
:104110000001005700010056000100550001005445
:104120000001005300000053000100520001005143
:10413000000100500001004F0001004E0000004E41
:104140000001004D0001004C0001004B0000004B3D
:104150000001004A00010049000100480000004839
:104160000001004700010046000000460001004534
:10417000000000450001004400010043000000432E
:104180000001004200000042000100410000004127
:10419000000100400001003F0000003F0001003E20
:1041A0000000003E0001003D0000003D0001003C19
:1041B0000000003C0000003C0001003B0000003B10
:1041C0000001003A0000003A000100390000003907
:1041D00000010038000000380000003800010037FE
:1041E00000000037000100360000003600000036F5
:1041F00000010035000000350000003500010034EA
:1042000000000034000000340001003300000033DF
:1042100000000033000100320000003200000032D4
:1042200000010031000000310000003100010030C9
:1042300000000030000000300001002F0000002FBF
:104240000000002F0000002F0001002E0000002EB3
:104250000000002E0001002D0000002D0000002DA8
:104260000000002D0001002C0000002C0000002C9C
:104270000000002C0001002B0000002B0000002B90
:104280000000002B0001002A0000002A0000002A84
:104290000000002A00010029000000290000002978
:1042A000000000290000002900010028000000286B
:1042B000000000280000002800000028000100275E
:1042C0000000002700000027000000270000002752
:1042D0000001002600000026000000260000002645
:1042E0000000002600010025000000250000002538
:1042F000000000250000002500000025000100242A
:10430000000000240000002400000024000000241D
:104310000001002300000023000000230000002310
:104320000000002300000023000000230001002201
:1043300000000022000000220000002200000022F5
:1043400000000022000100210000002100000021E7
:1043500000000021000000210000002100000021D9
:1043600000010020000000200000002000000020CC
:1043700000000020000000200000002000000020BD
:104380000001001F0000001F0000001F0000001FB0
:104390000000001F0000001F0000001F0001001EA1
:1043A0000000001E0000001E0000001E0000004370
:1043B000686F6F736520636F6C6F723A0046616956
:1043C0006C207374617473004D37303220430046A3
:1043D00061726D206E756D626572004D3630300011
:1043E0004D3234004D323320257300052E2E0052FD
:1043F0006573756D696E67207072696E74005375B0
:1044000070706F727400537461746973746963734C
:1044100020200043616C6962726174696F6E0041B3
:1044200075746F4C6F61642066696C616D656E7444
:10443000004368616E6765206578747275646572A3
:1044400000556E6C6F61642066696C616D656E7499
:1044500000456A6563742066696C616D656E740001
:104460004C6F61642066696C616D656E74004E6F9F
:104470002053442063617264005072696E74206638
:10448000726F6D20534400526573756D65207072B4
:10449000696E74005061757365207072696E740086
:1044A000507265686561740054756E65004C69767C
:1044B000652061646A757374205A00496E666F20C6
:1044C00073637265656E0046696E697368696E67CD
:1044D000206D6F76656D656E747300536F756E64D5
:1044E0002020202020205B6C6F75645D00536F7569
:1044F0006E642020202020205B6D7574655D005364
:104500006F756E64202020205B73696C656E745D2E
:1045100000536F756E642020202020205B6F6E6337
:10452000655D00536F756E642020202020205B6C39
:104530006F75645D004372617368206465742E203A
:10454000205B4E2F415D0043726173682064657487
:104550002E2020205B6F6E5D0043726173682064C3
:1045600065742E20205B6F66665D004D6F6465206C
:104570002020205B537465616C74685D004D6F642E
:104580006520202020205B4E6F726D616C5D0046BF
:10459000696C2E2073656E736F7220205B6F6E5D89
:1045A0000046696C2E2073656E736F72205B6F66B8
:1045B000665D004368616E67652066696C616D6564
:1045C0006E7400466C6F77005370656564004661D9
:1045D0006E20737065656400426564004E6F7A7A80
:1045E0006C650053657474696E6773005072696E10
:1045F000742061626F7274656400596573004E6F58
:104600000053746F70207072696E740046696C6537
:1046100020696E636F6D706C6574652E20436F6EDC
:1046200074696E756520616E797761793F004D61BF
:10463000696E00627573793A2070617573656420E4
:10464000666F7220696E70757400627573793A20B6
:1046500070617573656420666F7220757365720092
:10466000627573793A2070726F63657373696E67F0
:10467000002046004731205A00204600473120459F
:10468000004D3833006F6B0A000000211042206398
:10469000308440A550C660E770088129914AA16B1B
:1046A000B18CC1ADD1CEE1EFF131121002733252B3
:1046B00022B5529442F772D662399318837BB35A6B
:1046C000A3BDD39CC3FFF3DEE36224433420040183
:1046D00014E664C774A44485546AA54BB5288509BB
:1046E00095EEE5CFF5ACC58DD55336722611163053
:1046F00006D776F6669556B4465BB77AA71997380B
:1047000087DFF7FEE79DD7BCC7C448E5588668A792
:10471000784008611802282338CCC9EDD98EE9AF5A
:10472000F9488969990AA92BB9F55AD44AB77A96F2
:104730006A711A500A333A122AFDDBDCCBBFFB9EAA
:10474000EB799B588B3BBB1AABA66C877CE44CC5C2
:104750005C222C033C600C411CAEED8FFDECCDCDFA
:10476000DD2AAD0BBD688D499D977EB66ED55EF492
:104770004E133E322E511E700E9FFFBEEFDDDFFC4A
:10478000CF1BBF3AAF599F788F8891A981CAB1EBEF
:10479000A10CD12DC14EF16FE18010A100C230E318
:1047A000200450254046706760B9839893FBA3DAD4
:1047B000B33DC31CD37FE35EF3B1029012F322D268
:1047C000323542145277625672EAB5CBA5A8958964
:1047D000856EF54FE52CD50DC5E234C324A01481B8
:1047E000046674476424540544DBA7FAB79987B874
:1047F000975FE77EF71DC73CD7D326F2369106B008
:104800001657667676154634564CD96DC90EF92F73
:10481000E9C899E9898AB9ABA94458654806782757
:1048200068C018E1088238A3287DCB5CDB3FEB1E13
:10483000FBF98BD89BBBAB9ABB754A545A376A16A7
:104840007AF10AD01AB32A923A2EFD0FED6CDD4DA3
:10485000CDAABD8BADE89DC98D267C076C645C45F7
:104860004CA23C832CE01CC10C1FEF3EFF5DCF7CB3
:10487000DF9BAFBABFD98FF89F176E367E554E7447
:104880005E932EB23ED10EF01E7C3C3E5E2B3D3F31
:104890002F5B5D3B2C2A225C0020003E003E002066
:1048A000003E003E0054656D7065726174757265FE
:1048B0002063616C6962726174696F6E2066616900
:1048C0006C65642E20436F6E74696E756520776920
:1048D0007468207072657373696E672074686520F0
:1048E0006B6E6F622E0054656D70657261747572C7
:1048F000652063616C6962726174696F6E20646FB8
:104900006E652E20436F6E74696E756520776974CD
:1049100068207072657373696E6720746865206BB8
:104920006E6F622E005A3020284C4544206F6E294D
:1049300020005A3120284C4544206F6666290050DB
:104940002E492E4E2E442E412E2073746174650024
:1049500054656D70657261747572652063616C6910
:1049600062726174696F6E206661696C656400547F
:10497000656D70657261747572652063616C6962E2
:10498000726174696F6E2069732066696E697368FD
:10499000656420616E64206163746976652E2054BD
:1049A000656D702E2063616C6962726174696F6EEF
:1049B0002063616E2062652064697361626C656466
:1049C00020696E206D656E752053657474696E671D
:1049D000732D3E54656D702E2063616C2E004578FA
:1049E000747275646572004D6F7665205A004D6F64
:1049F00076652059004D6F76652058001B5B324A62
:104A0000437261736820646574656374696F6E20B6
:104A100063616E1B5B313B30486265207475726E5A
:104A20006564206F6E206F6E6C7920696E1B5B323F
:104A30003B30484E6F726D616C206D6F6465001B7A
:104A40005B324A5741524E494E473A1B5B313B302D
:104A500048437261736820646574656374696F6E3E
:104A60001B5B323B304864697361626C656420692A
:104A70006E1B5B333B3048537465616C7468206D0A
:104A80006F6465004175746F6C6F6164696E672057
:104A900066696C616D656E7420617661696C6162D6
:104AA0006C65206F6E6C79207768656E2066696C26
:104AB000616D656E742073656E736F72206973200B
:104AC0007475726E6564206F6E2E2E2E00455252E4
:104AD0004F523A2046696C616D656E742073656E45
:104AE000736F72206973206E6F7420726573706FBC
:104AF0006E64696E672C20706C65617365206368F5
:104B000065636B20636F6E6E656374696F6E2E00F4
:104B100043757272656E74005573656420647572B6
:104B2000696E67207072696E740050494420636139
:104B30006C2E2066696E6973686564005049442074
:104B400063616C2E202020202020202020202000A7
:104B5000506C656173652077616974004D31313740
:104B6000204669727374206C617965722063616C90
:104B70002E005072696E742070617573656400490F
:104B80006E76616C6964205049442063616C2E200C
:104B9000726573756C74732E204E6F742073746F0E
:104BA00072656420746F20454550524F4D2E004D64
:104BB000353030004731205A3135204631353030DC
:104BC00000473931004731205835302059313930CC
:104BD00020453020463730303000473930004D37DF
:104BE0003032004D3730322043004D3730322055BF
:104BF000004D373032004D373032204300473120EE
:104C00005A3135204631353030004739310047318F
:104C10002058353020593139302045302046373042
:104C20003030004D383300473930004D3834004DB6
:104C3000313034205330004D3834004D373032207D
:104C40004300473120583130205931383020463424
:104C5000303030004731205A313020463133303047
:104C60002E303030004D313430205330004D313053
:104C70003420533000473120452D302E3037353029
:104C8000302046323130302E3030303030004D312F
:104C900030370047312058353020593535204533DD
:104CA0002E363237373300473120583230302059D2
:104CB00035352045302E34393338360047312058C9
:104CC000323030205937352045332E36323737339E
:104CD00000473120583530205937352045302E34A3
:104CE000393338360047312058353020593935208E
:104CF00045332E3632373733004731205832303083
:104D0000205939352045302E343933383600473173
:104D1000205832303020593131352045332E36324B
:104D2000373733004731205835302059313135205D
:104D300045302E343933383600473120583530204D
:104D4000593133352045332E36323737330047312A
:104D5000205832303020593133352045302E363608
:104D60003137340047312058323030205931353511
:104D70002045322E36323737330047312058313014
:104D800030205931353520453200473120583735EC
:104D900020593135352045322E35004731204631F6
:104DA000303830004731205A302E313530204637E8
:104DB0003230302E303030004731205835302059D5
:104DC000313535004731204634303030004D3230F7
:104DD00034205331303030004731205A35204637A7
:104DE0003230302E30303000473120452D312E35D5
:104DF000303030302046323130302E3030303030AC
:104E0000004D3833004739300047323100473932DE
:104E10002045302E3000473120583130302E3020A0
:104E20004531322E352046313030302E300047317A
:104E3000205836302E302045392E30204631303043
:104E4000302E300047312058352E302045342E305A
:104E50002046313030302E30004731205A302E324B
:104E6000302046313030302E300047312058353533
:104E70002E30204532352046313430302E30004738
:104E80003120592D322E302046313030302E300036
:104E9000473120583234302E30204532352E3020E4
:104EA0002046323230302E30004739322045302E05
:104EB00030004731205A302E332046313030302EEA
:104EC00030004731205835352E302045382E3020DF
:104ED00046323030302E300047312058352E3020C9
:104EE0004533322E302046313830302E30004731B5
:104EF000205835352E30204533322E302046313083
:104F000037332E30004731205A302E34204631308E
:104F100030302E3000473120592D332E302046318D
:104F20003030302E30004D38330047393220453094
:104F30002E3000473238004D313039205332313570
:104F4000004D31393020533630004D31343020534C
:104F50003630004D3130342053323135004D313050
:104F6000370053657474696E67732053746F72658C
:104F7000640053746F7265642073657474696E673E
:104F80007320726574726965766564004861726445
:104F9000636F6465642044656661756C7420536555
:104FA0007474696E6773204C6F6164656400563277
:104FB00000000000C8420000C8420000C8430000D2
:104FC0008C4300004843000048430000404100007B
:104FD000F042E8030000E8030000C8000000881366
:104FE000000000409C4400409C4400000000000081
:104FF0000000204E00000000204100002041CDCCE8
:10500000CC3E000020400000000000000000000036
:105010000000CDCCCC3E3D0A8141FF08433EB09913
:10502000AB438F42FC42E65A343F4C62B04500002D
:10503000000000404000003442000000000000007A
:105040000000000041000000E03F0000C8420000F6
:10505000C842000040410000F042C0030000C0030D
:105060000000C800000088130000454550524F4D15
:10507000204572726F7200436F6E74696E756520A1
:105080007769746820616E6F7468657220626F77EB
:1050900064656E3F00250020202020202000202075
:1050A000202020200045524153494E4720616C6C1E
:1050B000206461746100466163746F7279205245A7
:1050C0005345540000007F43008054430000524386
:1050D00000000000000080C09A99193E0000000006
:1050E000000080C09A99193E43616E6E6F7420650E
:1050F0006E746572207375626469723A200053445D
:105100002063617264206F6B006F70656E526F6F09
:1051100074206661696C656400766F6C756D652ED0
:10512000696E6974206661696C6564005344206926
:105130006E6974206661696C00536F7274696E6782
:105140002066696C657300536F6D652066696C65D8
:10515000732077696C6C206E6F7420626520736FAA
:10516000727465642E204D61782E204E6F2E206F54
:10517000662066696C657320696E203120666F6CED
:1051800064657220666F7220736F7274696E672037
:105190006973203130302E001F1F1F1F1F1F1F1F5C
:1051A0002E002E004E6F7720667265736820666948
:1051B0006C653A20004E6F7720646F696E672066D9
:1051C000696C653A20002220706F730022207061A4
:1051D00072656E743A2200535542524F5554494EEF
:1051E000452043414C4C207461726765743A22003B
:1051F000747279696E6720746F2063616C6C2073C0
:1052000075622D67636F64652066696C65732077CE
:1052100069746820746F6F206D616E79206C65769B
:10522000656C732E204D4158206C6576656C206945
:10523000733A0057726974696E6720746F206669EB
:105240006C653A200046696C652073656C65637413
:105250006564002053697A653A200046696C6520D0
:105260006F70656E65643A20001000C90210012C51
:10527000014001220170011801B0010E01F001048A
:10528000015002FA00B002F0003003E600D003DC67
:10529000009004D2007005C800A006BE000008B44B
:1052A00000B009AA00D00BA000600E960060118C1F
:1052B000000015820020197800C01D6E00A0226435
:1052C00000B0275A00902C500000314600E0343CDA
:1052D0000010383200903A2800603C1E00A03D14B7
:1052E00000803E0A00203F000070012C0190012741
:1052F00001B0012201C0011D01F0011801100213CB
:105300000130020E016002090190020401C002FF97
:10531000000003FA004003F5008003F000D003EB27
:10532000002004E6007004E100E004DC004005D742
:1053300000C005D2004006CD00D006C8008007C3DB
:10534000003008BE00F008B900C009B400B00AAFD0
:1053500000B00BAA00D00CA500000EA000500F9BBF
:1053600000C01096005012910000148C00C01587E8
:1053700000B0178200B0197D00D01B7800001E73AA
:105380000040206E0090226900F024640040275FF6
:105390000090295A00E02B5500102E500020304B71
:1053A0000010324600E033410090353C00103737A2
:1053B0000070383200A0392D00B03A2800A03B23FD
:1053C00000603C1E00103D1900903D1400103E0F7F
:1053D00000703E0A00C03E0500003F000090137DB3
:1053E00000B0157800F0177300601A6E00F01C69A9
:1053F00000A01F640050225F0020255A00E02755BE
:1054000000902A5000202D4B00A02F4600F0314183
:105410000010343C00F0353700A037320020392D21
:1054200000603A2800703B2300603C1E00203D19BC
:1054300000C03D1400403E0F00A03E0A00F03E05B3
:1054400000403F0000703FFBFF903FF6FFB03FF190
:10545000FFC03FECFFD03FE7FFE03FE2FFF03FDD62
:10546000FFF03FD8FF20484F54454E442054484554
:10547000524D414C2052554E41574159002048450C
:10548000415442454420544845524D414C205255C8
:105490004E4157415900544845524D414C205255B8
:1054A0004E415741590042454420544845524D41D0
:1054B0004C2052554E415741590020544845524DB9
:1054C000414C2052554E41574159202820505245B9
:1054D0004845415420484F54454E442900205448E3
:1054E00045524D414C2052554E415741592028209C
:1054F000505245484541542048454154424544296D
:105500000050524548454154204552524F520042A6
:1055100045442050524548454154204552524F522F
:10552000004572723A204D415854454D50003A2082
:105530004578747275646572207377697463686501
:1055400064206F66662E204D415854454D5020749E
:1055500072696767657265642021004572723A203E
:105560004D415854454D50204245440054656D709E
:105570006572617475726520686561746564206226
:105580006564207377697463686564206F66662E4E
:10559000204D415854454D502074726967676572BB
:1055A00065642021004572723A204D494E54454DA4
:1055B00050204245440054656D7065726174757287
:1055C000652068656174656420626564207377692D
:1055D0007463686564206F66662E204D494E54459D
:1055E0004D502074726967676572656420210045BB
:1055F00072723A204D494E54454D50003A2045783C
:105600007472756465722073776974636865642069
:105610006F66662E204D494E54454D502074726978
:10562000676765726564202100746D6332313330C1
:105630005F686F6D655F656E74657228617865730C
:105640005F6D61736B3D307825303278290A0074C4
:105650006D63323133305F686F6D655F6578697493
:1056600020746D63323133305F73675F686F6D69CB
:105670006E675F617865735F6D61736B3D30782530
:105680003032780A0046696C616D656E742073650E
:105690006E736F7200537761707065640046726F4D
:1056A0006E742F6C6566742066616E730041786954
:1056B000730041786973206C656E677468004C6F85
:1056C0006F73652070756C6C657900456E647374DA
:1056D0006F70206E6F742068697400456E64737417
:1056E0006F70004D6F746F7200456E6473746F70ED
:1056F0007300576972696E67206572726F7200423B
:105700006564202F20486561746572004E6F7420B7
:10571000636F6E6E6563746564004865617465727D
:105720002F546865726D6973746F7200506C656197
:10573000736520636865636B203A0053656C66741B
:10574000657374206572726F7220210046696C6106
:105750006D656E742073656E736F723A0050726976
:105760006E742066616E3A00457874727564657275
:105770002066616E3A0053656C66746573742066CA
:1057800061696C6564202000416C6C20636F7272EB
:1057900065637420202020202000436865636B69C6
:1057A0006E672073656E736F727320004368656364
:1057B0006B696E67206265642020202020004368AA
:1057C00065636B696E67205A2061786973202000D9
:1057D000436865636B696E6720592061786973203F
:1057E0002000436865636B696E67205820617869A3
:1057F00073202000436865636B696E6720686F746F
:10580000656E64202000436865636B696E67206580
:105810006E6473746F7073004572726F72202D2006
:10582000737461746963206D656D6F72792068614E
:1058300073206265656E206F766572777269747425
:10584000656E00436172642072656D6F76656400F9
:105850004361726420696E736572746564002D2DF6
:105860002D2D2D2D2D2D2D2D2D2D2D2D2D2D2D2D68
:105870002D2D0043616C6962726174696E672068E6
:105880006F6D65000000000000110A04505255536E
:105890004133444657002079303D25640A00207882
:1058A000303D25640A004F4B0A004552524F5220AA
:1058B00061643D25640A002020207A303D25640A79
:1058C00000207A303D25640A002079303D25640AA5
:1058D000002078303D25640A0078797A63616C5F36
:1058E00066696E645F706F696E745F63656E746520
:1058F00072320A0020746F6F206C6F6E67206578BB
:1059000074727573696F6E2070726576656E7465FA
:10591000640020636F6C6420657874727573696FBE
:105920006E2070726576656E74656400462564202D
:1059300025640A00352E302E3100726300626574D2
:105940006100616C706861006465760078797A63E3
:10595000616C5F73706972616C322063783D25649D
:105960002063793D2564207A303D256420647A3DAA
:105970002564207261646975733D25642061643D0E
:1059800025640A0001021020200808102040102081
:1059900040800201020108040201010204081020F3
:1059A00040808040201008040201800402018040F1
:1059B000201008040201080402010102040810205A
:1059C0004080010204081020408010080408801064
:1059D0002040044080102040048000002200250068
:1059E00028002B002E0031003400020100000501C8
:1059F00008010B010505050507050808080802024E
:105A000002020A0A08080404040401010101010158
:105A100001010303030303030303040707070C0C3B
:105A20000C0C0C0C0C0C0202020206060606060602
:105A300006060B0B0B0B0B0B0B0B07070A0A0A0ACC
:105A40000A0A050505040404080802746D6332316E
:105A500033305F676F746F5F7374657020256420E7
:105A60002564202564202564200A002E006F7065BF
:105A70006E206661696C65642C2046696C653A200D
:105A80000022206661696C65643A2042756666652D
:105A9000722066756C6C21002200256920686F7584
:105AA0007273202569206D696E75746573005449A1
:105AB0004D454F55543A004D3131300046756C6CB0
:105AC0002052582042756666657200656E71756574
:105AD000696E6720220053544F505045442E2000D9
:105AE0005072696E7465722073746F707065642093
:105AF00064756520746F206572726F72732E204614
:105B0000697820746865206572726F7220616E64B6
:105B100020757365204D39393920746F2072657393
:105B2000746172742E202854656D7065726174758D
:105B300072652069732072657365742E20536574D5
:105B40002069742061667465722072657374617275
:105B500074696E6729004E6F20436865636B7375C7
:105B60006D2077697468206C696E65206E756D6252
:105B700065722C204C617374204C696E653A20006C
:105B8000636865636B73756D206D69736D617463B4
:105B9000682C204C617374204C696E653A20004477
:105BA0006F6E65207072696E74696E672066696CCD
:105BB00065004E6F204C696E65204E756D62657292
:105BC000207769746820636865636B73756D2C203A
:105BD0004C617374204C696E653A20004C696E65A7
:105BE000204E756D626572206973206E6F74204C53
:105BF000617374204C696E65204E756D6265722B01
:105C0000312C204C617374204C696E653A20004D34
:105C10004D55204F4B2E20526573756D696E672E62
:105C20002E2E004D4D55204F4B2E20526573756D15
:105C3000696E6720706F736974696F6E2E2E2E0007
:105C40004D4D55204F4B2E20526573756D696E6713
:105C50002074656D70657261747572652E2E2E00EC
:105C60004D4D55206E6565647320757365722061B6
:105C70007474656E74696F6E2E204669782074683E
:105C80006520697373756520616E64207468656E44
:105C900020707265737320627574746F6E206F6EFE
:105CA000204D4D5520756E69742E00506C656173E2
:105CB000652072656D6F76652066696C616D656ED5
:105CC0007420616E64207468656E207072657373F1
:105CD00020746865206B6E6F622E00456A65637480
:105CE000696E672066696C616D656E74004D4D5517
:105CF0002073746172747320726573706F6E64695F
:105D00006E670A004D4D55206E6F7420726573707A
:105D10006F6E64696E670A000000803F55558541CB
:105D20000000803F0000C84100000040555505427A
:105D30000000C03F00004842000020405555854209
:105D4000000070C1ABAAA642000060C10000A041E3
:105D50000000C0C00000204100002041ABAA3A4131
:105D6000000020C15555D540000048C25555054298
:105D70004D373031204530004D373031204531002E
:105D80004D373031204532004D373031204533001A
:105D90004D373031204534004D3730312045340007
:105DA0004D373031204533004D37303120453200FA
:105DB0004D373031204531004D37303120453000EE
:105DC00046696C616D656E74206E72206F7574200B
:105DD0006F662072616E67652100773235783230E8
:105DE000636C5F63666D0A00773235783230636CBE
:105DF0005F656E7465720A00504154393132355F07
:105E00005245535F593D256868750A005041543921
:105E10003132355F5245535F583D256868750A0039
:105E2000062833D036C23E013F154132423B43F291
:105E3000443B45F24622473B48F2493B4AF05898DA
:105E4000590C5A085B0C5C086110679B6E22710745
:105E50007208FF095A0D000EF019045E0820642B29
:105E60006D322FFF0000A0400000A0400000004065
:105E700025336420737465703D253264206D73632F
:105E80006E743D2534640A0046696C616D656E74FC
:105E9000206F7574206F662072616E6765202564BF
:105EA000200A0067636F64655F4D3730312062659B
:105EB00067696E0A0046696C2E2073656E736F7297
:105EC00020726573706F6E736520697320706F6FD9
:105ED000722C2064697361626C652069743F0046AE
:105EE000696C616D656E7420657874727564696E35
:105EF000672026207769746820636F727265637407
:105F000020636F6C6F723F0057616974696E672020
:105F1000666F72206E6F7A7A6C6520616E642062A3
:105F2000656420636F6F6C696E670053656C6620F3
:105F300074657374204F4B0053656C6620746573F1
:105F4000742073746172742020006C63645F7365E5
:105F50006C66636865636B5F617869732025642C88
:105F60002025640A004D3834004731205A3135204D
:105F70004631303030004732382057002563204109
:105F8000584953205347313D25640A0041786973CD
:105F9000206C656E67746820646966666572656EFC
:105FA00063653A252E33660A004D65617375726527
:105FB000642061786973206C656E6774683A252E79
:105FC00033660A004D3234004D32332025730061B0
:105FD00075746F25692E670022206661696C65649F
:105FE0003A204275666665722066756C6C210045C4
:105FF0006E717565696E6720746F207468652066C0
:10600000726F6E743A2022004572726F723A0022EB
:1060100000456E717565696E6720746F20746865E0
:106020002066726F6E743A2022006563686F3A00D2
:106030004572723A205052494E542046414E2045F6
:1060400052524F52005072696E742066616E207316
:1060500070656564206973206C6F77657220746861
:10606000656E206578706563746564004572723A88
:1060700020455854522E2046414E204552524F52F0
:106080000045787472756465722066616E20737065
:10609000656564206973206C6F776572207468652C
:1060A0006E206578706563746564002F2F206163CE
:1060B00074696F6E3A706175736500526573656ED1
:1060C000640048656174696E672064697361626C1D
:1060D0006564206279207361666574792074696DE6
:1060E00065722E0025533A20256C640A25530A0058
:1060F000004D363030004653454E534F525F5245A7
:10610000434F564552006673656E736F725F7570CC
:1061100064617465202D204D3630300A0066736549
:106120006E736F725F6572725F636E74203D2030B4
:106130000A004731204533204632303000473120B5
:10614000452D332046323030004D373031000000CD
:106150002100240027002A002D0030003300010117
:106160000000040107010A010000200023002600AE
:1061700029002C002F00320000010000030106015D
:10618000090100000A0B02090C0D0E0807030401A7
:1061900000000000000000000000000000000000FF
:1061A00000000000000000000000000000001211CC
:1061B00010000000000000000000000000000000CF
:1061C00000000000000000000000000000000000CF
:1061D00000000000000000002563252E3132533AF4
:1061E0002573252B30362E316600202020202020DC
:1061F0002020202020202020202020202020003EA1
:10620000003E0020003E003E0020004E6F742073D0
:1062100070696E6E696E67005370696E6E696E6745
:10622000004C65667420686F74656E642066616EEC
:106230003F0046726F6E74207072696E74206661E2
:106240006E3F0046616E2074657374007A014A01E6
:1062500011241FBECFEFD1E2DEBFCDBF00E00CBFE7
:1062600016E0A0E0B2E0E4E9F8E703E00BBF02C00B
:1062700007900D92A63BB107D9F729E1A6EBB6E04E
:1062800001C01D92A43DB207E1F711E3C7E2D1E3DB
:1062900000E006C021970109802FFE010F9461BB29
:1062A000C632D10780E00807A9F70F94F78F0D9445
:1062B00039BC0C9400002F923F924F925F926F92E4
:1062C0007F928F929F92AF92BF92CF92DF92EF9286
:1062D000FF920F931F93CF93DF93CDB7DEB7C857CD
:1062E000D1090FB6F894DEBF0FBECDBF80917E13EB
:1062F00090917F13892B11F40C94527182E090E0FD
:10630000909327028093260281E493E00F94370A4A
:106310008823B1F080914013909141136AE270E0BC
:1063200005960F94B8BB009711F0DC011C92809188
:1063300040139091411305960F941F2F0C945F6C9E
:10634000C0906D15D0906E1586010D571C4E46E01D
:1063500050E06DE770E1C8010F94EBAE892B09F0B6
:10636000EDC086E493E00F94370A882309F49BC0BC
:1063700088E50F94959E182F89E50F94959E8111BD
:1063800012600F942D838091B70601E0080F0093EF
:10639000B706811105C08AE496E10F94745A0EC0C5
:1063A00048EC5FEA60E070E08AE496E10F942F5ACF
:1063B000882331F010924A161092B70601E007C008
:1063C000033049F710924A161092B70600E081E0B8
:1063D0000E9407A80E94FEA782E00E9483A610FFE9
:1063E00015C086E69FE00F94E8B561E0680F86E689
:1063F0009FE00F94FAB585E09FE00F94F5B5BC01DE
:106400006F5F7F4F85E09FE00F9414B611FF15C0BA
:1064100088E69FE00F94E8B561E0680F88E69FE0AA
:106420000F94FAB583E09FE00F94F5B5BC016F5F60
:106430007F4F83E09FE00F9414B681E00E9407A88D
:1064400082E00E9483A680E892E10F94AD2D40E0A7
:1064500061E081E00F947B6E0F942D83002321F087
:1064600061E08CEB9DE01BC0E0910E0DF0E0EE0FC3
:10647000FF1FE159FA4E1182108240E060E082E68F
:1064800092E10E94DAFB182F81E00E9407A861E0E8
:10649000112319F08EEA9DE002C081EA9DE00F947D
:1064A0009B580C945F6C85E593E00F94370A882322
:1064B00079F080913E0E882331F060E070E080E852
:1064C0009FE30E9441F081E080930C020C945F6C8A
:1064D00083E693E00F94370A882311F40C945F6CE1
:1064E00081E080930C028091790E811104C00E949A
:1064F00081E70C945F6C813011F00C945F6CE0E9E3
:10650000FDE084918F01882339F00F94FC0F0F5F19
:106510001F4FF8018491F7CF8AE00F94FC0FEFE84A
:10652000F7E184918F01882311F40C94EC6A0F94A5
:10653000FC0F0F5F1F4FF8018491F5CF44E050E04E
:1065400068E770E1C8010F94EBAE892B09F00EC12A
:10655000860109571C4E49E050E06EE670E1C80123
:106560000F94EBAE892BD9F4F601E057FC4E108165
:10657000153431F01855143010F00C945F6C01C0D4
:1065800013E04AE050E060E070E0C6018F569C4E98
:106590000F94A2AC812F0F94AC490C945F6C49E02E
:1065A00050E064E670E1C8010F94EBAE892B61F511
:1065B000F601E057FC4E1081153431F018551430B7
:1065C00010F00C945F6C01C013E04AE050E060E012
:1065D00070E0C6018F569C4E0F94A2ACE12FF0E004
:1065E000E05FF84F40E051E0008002C056954795CB
:1065F0000A94E2F7842F880F880F81506823812F37
:106600000F948E4B0C945F6C49E050E06AE570E1AA
:10661000C8010F94EBAE892B11F00C945F6CF6015E
:10662000E057FC4E8081853449F008EA902E980EA0
:10663000F3E0F91510F40C945F6C02C013E0912E96
:10664000E92CF12C5701AA0CBB1CF501E25DFD4FB2
:106650001081012F0F70712E7294BFE07B22272DC5
:106660002770722E111F1127111F61816770660F2D
:10667000162BF501E15DFD4F8081882E869486946E
:106680008694382D3370832E1A821982C6018F5654
:106690009C4EDC012C912223E1F14AE050E0BE0146
:1066A0006F5F7F4F0F94A2AC062F0F7089819A8184
:1066B000009779F1FC012081222359F14AE050E052
:1066C000BE016F5F7F4F0F94A2AC6770762E8981F9
:1066D0009A810097F1F0DC012C912223D1F04AE05D
:1066E00050E0BE016F5F7F4F0F94A2AC162F1F705A
:1066F00089819A81009769F0FC012081222349F069
:106700004AE050E0BE016F5F7F4F0F94A2AC637010
:10671000862EF501E25DFD4F972D97709295907F43
:10672000612F679566276795902B962B9083612F35
:1067300066951181107E882D8370880F880F880FD1
:10674000162B182B1183C701875E9D4FD701A35EBF
:10675000BD4FB701605F784FFC0120814C91DB0198
:106760006C91892D0E9469BA0C945F6C80E793E06C
:106770000F94370A882321F00E94D0AF0C945F6CED
:1067800080E893E00F94370A882309F4B5C186E8BE
:1067900093E00F94370A882391F08091FE0E8823AE
:1067A00011F40C945F6C0F94588A60936016709388
:1067B000611680936216909363160C945F6C8BE85D
:1067C00093E00F94370A882349F08091D00E8F937D
:1067D0008091CF0E8F938AE797E03DC08FE893E0DA
:1067E0000F94370A882329F140915E1350915F136B
:1067F0002CE3249FC001259F900D11249F938F931C
:1068000040915C1350915D13249FC001259F900D12
:1068100011249F938F9383E697E09F938F930F9418
:1068200018B00F900F900F900F900F900F900C9446
:106830005F6C83E993E00F94370A8823C9F0809155
:10684000FE0E882391F080912A078F93809129076B
:106850008F9380E697E09F938F930F9418B00F90DB
:106860000F900F900F900C945F6C8EE497E0F0C047
:1068700086E993E00F94370A882321F010922807C5
:106880000C945F6C8AE993E00F94370A882349F0EF
:1068900060E085EA9FE00F94FAB561E086E590E15B
:1068A000FECD8FE993E00F94370A882321F00F94EF
:1068B00050640C945F6C86EA93E00F94370A882347
:1068C00019F18091FE0E8823C9F08AEA95E5DC0172
:1068D0008093FC1F9093FD1FA093FE1FB093FF1F9A
:1068E00088E08093FB1F98E10FB6F894A8959093E9
:1068F00060000FBE80936000F894FFCF8CEA93E0B5
:106900000F9435110C945F6C8EEB93E00F94370A63
:10691000882339F1809140139091411341E061E067
:1069200003960F949B148091941890919518A091C0
:106930009618B09197188093411990934219A0939B
:106940004319B09344198CE898E10E9469EE8C01D8
:106950000F94FC0F0A30110531F70F9478450C9411
:106960005F6C81EC93E00F94370A882381F00F94D9
:106970007F6681E080933B078091401390914113A3
:1069800041E060E004960F949B140C945F6C85ECDE
:1069900093E00F94370A882309F45EC08091FE0EBD
:1069A000882309F453C0109271156091CE1970912B
:1069B000CF198BE390E00F9493AF6091CE19709153
:1069C000CF1983E590E00F9493AF19821B821A824E
:1069D000CE0101960F94235A00E010E0FF24F394B7
:1069E0008091020E9091030E2091040E3091050EBD
:1069F000821B930B8F779927892B81F00F94580F67
:106A0000F09271156091CE197091CF1990E00F94AA
:106A100093AF0F5F1F4F10927115E2CF64E670E0E5
:106A2000CE0101960F94FA59811103C0033111056B
:106A3000BCF281E0809371156091CE197091CF19ED
:106A40008AE090E00F9493AF0C945F6C8BE695E036
:106A50000F9440B00C945F6C88EC93E00F94370A6D
:106A6000882361F00CEC13E0F80181918F018823F9
:106A700011F40C94EC6A0F94FC0FF6CF87ED93E0C1
:106A80000F94370A882361F00BED13E0D8018D9144
:106A90008D01882311F40C94EC6A0F94FC0FF6CF4F
:106AA0008AEF93E00F94370A81110C945F6C8FEF9B
:106AB00093E00F94370A882341F060E070E088EF9C
:106AC0009FE00E9452D20C945F6C82E094E00F949D
:106AD000370A882321F00F94588A0C945F6C87E062
:106AE00094E00F94370A882311F40C945F6C80E0D3
:106AF0000F942D0C0C945F6C8EE50F94959E8AAFCD
:106B000081110C945F6C87E40F94959EF82E882376
:106B100011F40C94C9420F948C9E0F94D3B76C342B
:106B2000710509F404C27CF56430710509F4FCC0F8
:106B300054F46230710509F4E2C00CF0E9C077FF4B
:106B40006DC00C94BD426C31710509F43FC15CF419
:106B50006A30710509F435C16B30710511F00C9480
:106B6000BD4280E02FC16E31710509F471C16B34F3
:106B7000710511F00C94BD4208E210E0F9E2EF2E2D
:106B8000F7E0FF2EB5C16835710511F40C945F6C08
:106B9000ECF46135710511F40C94844154F46F34B4
:106BA000710509F431C76035710509F459C70C94B2
:106BB000BD426635710511F40C942D42673571059F
:106BC00011F00C94BD4281E00C942E426C3571059D
:106BD00011F40C9436427CF46A35710511F40C946E
:106BE00032426B35710511F00C94BD4281E0809307
:106BF00071190C945F6C6236710511F40C94964215
:106C00006336710511F00C94BD421092FE0E60E0E7
:106C100084EC9FE00F94FAB50C94B8428091190F60
:106C200081110C945F6C0F945CA96091470E709178
:106C3000480E8091490E90914A0E0F9411B16B014C
:106C40007C0140900B1050900C1060900D107090D3
:106C50000E108090080D9090090DA0900A0DB09034
:106C60000B0DA5019401C301B2010F9473B620E08E
:106C700030E048EC52E40F947AAA9B01AC01C701C2
:106C8000B6010F94BFB81816D4F4A3019201C50140
:106C9000B4010F9473B620E030E048EC52E40F9456
:106CA0007AAAA70196010F9474B60F94D9B760938E
:106CB000470E7093480E8093490E90934A0E809130
:106CC000C510882311F40C945D6C88E50F94959E93
:106CD00081110C945D6C89E50F94959E81110C9443
:106CE0005D6C8AE50F94959E81110C945D6C85E432
:106CF0000F94959E81110C94346C0C945D6C809172
:106D0000190F81110C945F6C0F941CAA81E008C0CC
:106D10008091190F81110C945F6C0F941CAA80E074
:106D20000F94A6A30C945F6C80E50F94959E882326
:106D300039F00F948C9E0F94D9B76B017C0103C07E
:106D4000C12CD12C760183E50F94959E882361F0A8
:106D50000F948C9E20E030E04AE754E40F947AAA26
:106D60000F94D9B76B017C01C114D104E104F10483
:106D700021F084EF93E10F94AD2D0F942D830F94A8
:106D8000588AC60ED71EE81EF91E0F94588A6093C3
:106D900076197093771980937819909379190F94D5
:106DA000588A6C157D058E059F0510F00C945F6C5C
:106DB0000F944F7D80E00F948E8380E00E9483A625
:106DC000EECF81E00F94B39E0C945F6C88E50F9436
:106DD000959E8EAF0F94819E1B012C0189E50F9427
:106DE000959E682E0F94819E26966CAF7DAF8EAFD8
:106DF0009FAF26978AE50F94959ED82E0F94819E7B
:106E00004B015C0187E50F94959E782E83E40F94E7
:106E1000959E7F928F93CD2C2696ECACFDAC0EAD5B
:106E20001FAD2697262DB201A1018EAD0F94996B4F
:106E30000F900F90BEADB1110C945F6C61100C946B
:106E40005F6C71100C945F6CD1100C945F6C08C671
:106E50000F942D8381E00F949E098C0180E090E0D7
:106E6000A8E4B4E48093210290932202A093230229
:106E7000B093240260E070E080E291EC0F94531331
:106E800080910A108F93809109108F938091081040
:106E90008F93809107108F93809106108F9380912C
:106EA00005108F93809104108F93809103108F931E
:106EB000809102108F93809101108F938091001028
:106EC0008F938091FF0F8F9388ED95E49F938F931D
:106ED00082E397E09F938F930F9418B0C8010F94AB
:106EE0007D090FB6F894DEBF0FBECDBF0C945F6C6A
:106EF000B801012E000C880B990B0F9413B10E945E
:106F00003B9F9F938F937F936F931F930F93FF925A
:106F1000EF920F9418B00F5F1F4F0FB6F894DEBFBB
:106F20000FBECDBF0F36110519F70C945F6C0F948F
:106F3000540F8A3F30F082ED93E10E947CFC0C9468
:106F40005F6C80910F0D882341F08091100D882394
:106F500021F08091110D811106C081E080937D1395
:106F60008FE490E197C58BE893E10E947CFC40E0C0
:106F700060E082E59CE10E94DAFB882309F493C07B
:106F800080E090E0A0EAB0E48093071090930810AE
:106F9000A0930910B0930A102091031030910410AF
:106FA00040910510509106106091FF0F70910010F4
:106FB0008091011090910210FEE06F2EFDE07F2E77
:106FC0007F926F92812C912CA8E4AA2EA2E4BA2E73
:106FD000BBE0CB2EB0E1DB2EE12CF12C00EA10E47B
:106FE0000F9476348092071090920810A0920910A6
:106FF000B0920A1080E090E0A4E3B3E48093031021
:1070000090930410A0930510B09306106091FF0FA9
:107010007091001080910110909102107F926F92F8
:107020008501740120E030E044E353E40F947634AA
:107030000F942D838AE29CE10E947CFCE8EFFEE144
:10704000259135914591549120930310309304106C
:107050004093051050930610E4EFFEE165917591A1
:10706000859194916093FF0F7093001080930110AD
:1070700090930210E0900710F09008100091091012
:1070800010910A107F926F920F9476340F942D8393
:1070900041E060E080E00F947B6E0F900F900F90C6
:1070A0000F900F900F9020E030E04CE052E46091A0
:1070B000660D7091670D8091680D9091690D0F9428
:1070C000BFB818160CF0A4C08091FE0E8111A0C0AC
:1070D00080E090E0A8ECB2E4809307109093081051
:1070E000A0930910B0930A1020910310309104105E
:1070F00040910510509106106091FF0F70910010A3
:107100008091011090910210EEE0FDE0FF93EF936B
:10711000812C912C18E4A12E12E4B12E0BE0C02E8C
:1071200000E1D02EE12CF12C08EC12E40F9476341F
:1071300080E090E0ACE0B2E48F8F98A3A9A3BAA35B
:107140000E9496A719821A821B821C82CE01019688
:107150000F943F761092130D1092120D19821A821D
:107160001B821C821D82CE0101960F94745A0F90CF
:107170000F902F8D38A149A15AA16091660D709191
:10718000670D8091680D9091690D0F94BFB8181626
:1071900094F582E492E10E94CDFB64E080E00E94DD
:1071A000C6A782E00E9437A886E69DE00E940BB148
:1071B0000E9463AA8AE094E00E9463AACE014F96DF
:1071C0000E940BB10E9463AA8CE094E00E9463AA23
:1071D00088EE93E00E94BFA40E94E59E40E053E544
:1071E00067E070E0CE0101960F942F5A882309F4CE
:1071F000C0CF10E001C011E064E878E581E00E94B2
:1072000079A781E00E9407A8111102C080E0F8C3AD
:1072100081E00E9407A881E090E09093270280938C
:107220002602E1E3F0E184918F01882339F00F9485
:10723000FC0F0F5F1F4FF8018491F7CF8AE00F9486
:10724000FC0F1A821982C090660DD090670DE090F5
:10725000680DF090690D20E030E040EA50E4C7018D
:10726000B6010F9462B70F94D3B725E0269FA00113
:10727000279F500D1124BA01550F880B990B0F94BD
:1072800013B13B01382E292E20E030E04CE052E4CF
:107290000F940DB187FF06C0612C712CACE03A2E23
:1072A000B2E42B2EC101262D372D492F522DC701B7
:1072B000B6010F94BFB8181674F420E030E040EA2D
:1072C00050E4F101662D772D8F2F922D0F9474B617
:1072D0003B01382E292E2F923F927F926F9280E1B0
:1072E00097E09F938F930F9418B020E030E040EF29
:1072F00051E4F101662D772D8F2F922D0F9473B6E7
:1073000020E030E04CE852E40F9474B60F94D3B709
:107310007093130D6093120D84E090E09093400EF3
:1073200080933F0E81E090E09093EF0E8093EE0EFD
:107330008FEC9AE20F94AD2D80E090E0A0EAB0E4EB
:107340008093071090930810A0930910B0930A102F
:1073500020910310309104104091051050910610B7
:107360006091FF0F709100108091011090910210B8
:10737000BEE04B2EBDE05B2E5F924F92812C912C94
:1073800018E4A12E12E4B12E0BE0C02E00E1D02EA5
:10739000E12CF12C00EA10E40F94763480E090E0C8
:1073A000A0EAB1E48093FF0F90930010A093011026
:1073B000B093021080E090E0A0E7B2E48093031065
:1073C00090930410A0930510B0930610E09007105E
:1073D000F09008100091091010910A105F924F92DE
:1073E0009C01AD0160E070E080EA91E40F94763496
:1073F0008AE999E9A9E1BEE3809307109093081008
:10740000A0930910B0930A1020910310309104103A
:1074100040910510509106106091FF0F709100107F
:1074200080910110909102105F924F921AE9E12E23
:1074300019E9F12E09E11EE30F9476340F942D83A0
:107440000FB6F894DEBF0FBECDBF2091660D309110
:10745000670D4091680D5091690DF101662D772DF2
:107460008F2F922D0F94BFB818163CF488EE93E03E
:107470000E94BFA40E94E59EE8CF60E086EA9FE0FC
:107480000F94FAB580E090E0A0EAB0E48093071092
:1074900090930810A0930910B0930A102091031044
:1074A0003091041040910510509106106091FF0F2B
:1074B0007091001080910110909102100EE0402E0A
:1074C0000DE0502E5F924F92812C912CE8E4AE2E6D
:1074D000E2E4BE2EFBE0CF2EF0E1DF2EE12CF12C1A
:1074E00000EA10E40F947634E4EFFEE165917591C3
:1074F000859194916093FF0F709300108093011019
:1075000090930210E8EFFEE1259135914591549159
:1075100020930310309304104093051050930610ED
:10752000E0900710F09008100091091010910A10D7
:107530005F924F920F9476340F942D8360E070E049
:1075400080E89FEB0F9453130F900F900F900F90C4
:10755000882309F45BCE3091071027963FAF279719
:10756000409108102B964FAF2B97509109102F96F2
:107570005FAF2F9760910A1063966FAF63976F9319
:107580005F934F933F9383E097E09F938F930F9484
:1075900018B00F900F900F900F900F900F908EEAF1
:1075A0009FE09FAF8EAF44244A94542C13E2C12E27
:1075B000D12CE12CF12C8201B6010D2C000C880B92
:1075C000990B0F9413B14B015C0197012F5F3F4F53
:1075D0003BAF2AAFDF92CF923F932F9347EC56E019
:1075E0005F934F930F9418B00F900F900F900F90E0
:1075F0000F900F908FEF4816580611F40C944371BA
:10760000BE016F5F7F4F8EAD9FAD0E9452D2A5012C
:107610009401F101662D772D8F2F922D0F940DB1CE
:107620001816A4F495E0E916F10471F095E0C90E7E
:10763000D11CAFEF4A1A5A0AEEADFFAD3296FFAF3A
:10764000EEAFEAACFBACB7CF05E010E0C801875263
:10765000984FDC01AA0FBB1FBFAFAEAF3801B3E03C
:107660006B0E711C25E0209FC001219F900D1124FD
:107670001BAE1AAEFC01BD966596FFAFEEAF6597E7
:10768000AEE04A2EADE05A2EC301029705970CF0EA
:10769000B6C165966EAD7FAD65978AAC9BAC680D43
:1076A000791D072E000C880B990B0F9413B12696A9
:1076B0006CAF7DAF8EAF9FAF26977F926F92BAEB84
:1076C000AB2EB6E0BB2EBF92AF920F9418B0709263
:1076D000EF0E6092EE0E20E030E040EF51E426968F
:1076E0006CAD7DAD8EAD9FAD26970F9473B620E047
:1076F00030E040E251E40F947AAA20E030E040EA22
:1077000050E40F9462B720E030E048E452E40F9474
:1077100074B60F94D3B77093130D6093120D80E07D
:1077200090E0A0EAB0E48093071090930810A09333
:107730000910B0930A102091031030910410409169
:107740000510509106106091FF0F7091001080910C
:107750000110909102105F924F92812C912C18E4AD
:10776000A12E12E4B12E0BE0C02E00E1D02EE12CB0
:10777000F12C00EA10E40F94763480E090E0A0EA67
:10778000B1E48093FF0F90930010A0930110B09389
:107790000210812C912CF0E7AF2EF2E4BF2E8092E4
:1077A000031090920410A0920510B0920610E09081
:1077B0000710F09008100091091010910A105F92C4
:1077C0004F92812C912C28E4A22E22E4B22E20E0AC
:1077D00030E040E752E4BC01CD010F9476342AE951
:1077E00039E949E15EE32093071030930810409394
:1077F000091050930A102091031030910410409109
:107800000510509106106091FF0F7091001080914B
:107810000110909102105F924F921AE9E12E19E93E
:10782000F12E09E11EE30F9476340F942D830FB6E9
:10783000F894DEBF0FBECDBF2091660D3091670D6D
:107840004091680D5091690D26966CAD7DAD8EAD61
:107850009FAD26970F94BFB818163CF488EE93E0BE
:107860000E94BFA40E94E59EE7CF80E090E0A0EADE
:10787000B0E48093071090930810A0930910B09380
:107880000A1020910310309104104091051050917E
:1078900006106091FF0F709100108091011090917F
:1078A00002105F924F92812C912CE8E4AE2EE2E41C
:1078B000BE2EFBE0CF2EF0E1DF2EE12CF12C00EA12
:1078C00010E40F947634E4EFFEE1659175918591B3
:1078D00094916093FF0F7093001080930110909328
:1078E0000210E8EFFEE125913591459154912093E6
:1078F0000310309304104093051050930610E0904D
:107900000710F09008100091091010910A105F9272
:107910004F920F9476340F942D8360E070E080E8EE
:107920009FEB0F945313AAADBBAD1596BBAFAAAF97
:10793000BFEF6B1A7B0A0F900F900F900F90811181
:1079400003C00F94F29D5BC027967FAD27972B96BF
:107950006FAD2B972F969FAD2F9763968FAD639743
:10796000272F362F492F582F60910710709108103C
:107970008091091090910A100F9473B6162F072F5B
:10798000F82EE92E20914F10309150104091511057
:1079900050915210D801F7016B2F7A2F8F2F9E2F05
:1079A0000F947AAA0F94D3B77A836983EF92FF92E8
:1079B0000F931F938091690D8F938091680D8F9322
:1079C0008091670D8F938091660D8F93EEE8F6E0BE
:1079D000FF93EF930F9418B0BE016F5F7F4F8EAD92
:1079E0009FAD0E9452D22EAD3FAD2E5F3F4F3FAFB5
:1079F0002EAF0FB6F894DEBF0FBECDBF45CE81E0EF
:107A00000F94F29D0C945F6C0FEF10E096E8C92E76
:107A100096E0D92E1093BF190093BE1984E6E82E84
:107A2000F12C84E690E00E94BFA451E0E51AF10831
:107A3000C1F780915F138F9380915E138F931F9393
:107A40000F93DF92CF920F9418B0055011090F9049
:107A50000F900F900F900F900F90E1F60C945F6CC9
:107A600081E08093580E20910F0D8091A80F909186
:107A7000A90F222341F02091100D222321F05090D4
:107A8000110D51100FC0029749F081E080937D13D2
:107A90008AE290E10F9444760C945F6C1092580E39
:107AA0000C945F6C0297D1F380913F0E9091400E41
:107AB00028969FAF8EAF2897A091EE0EB091EF0E53
:107AC0002C96BFAFAEAF2C9781E090E09093400E24
:107AD00080933F0E83E190E09093EF0E8093EE0E43
:107AE00081E00E9483A60F946A4F0E94B78C80E0C9
:107AF00090E0A0EAB0E48093071090930810A09360
:107B00000910B0930A102091031030910410409195
:107B10000510509106106091FF0F70910010809138
:107B20000110909102100EE0602E0DE0702E7F92F9
:107B30006F92E5E58E2E982CA82CE1E4BE2EFBE09A
:107B4000CF2EF0E1DF2EE12CF12C00EA10E40F94AF
:107B50007634E2EAFFE165917591859194916093A5
:107B6000FF0F709300108093011090930210E6EACB
:107B7000FFE1259135914591549120930310309365
:107B800004104093051050930610E0900710F090F9
:107B900008100091091010910A107F926F92812CA9
:107BA000912CB8ECAB2EB2E4BB2E0F9476340F942C
:107BB0002D830F900F900F900F9005EC1FE0C801E0
:107BC0000F94F5B5019639F00E5F1F4F053DEFE0BC
:107BD0001E07A9F75AAE80E00F949E0960969FAFEA
:107BE0008EAF609712EA412E1FE1512E612C712C4D
:107BF000C30163E070E00F9432BB24967FAF6EAF99
:107C000024971C0160FF06C0B2E08B2E912C881ACD
:107C1000990A14019AAC9920A1F16114710489F1B7
:107C200024968EAD9FAD2497880F991F2496AEACF5
:107C3000BFAC24978A0D9B1D820D931D880F991F41
:107C40008D53904F0F94F5B5BC01990F880B990B8C
:107C50000F9413B12AE037ED43E25CE30F947AAA64
:107C600020917315309174154091751550917615CA
:107C70000F9474B622966CAF7DAF8EAF9FAF2297F4
:107C800006C022961CAE1DAE1EAE1FAE229720E08F
:107C900030E040EA50E420930710309308104093FE
:107CA000091050930A102091031030910410409154
:107CB0000510509106106091FF0F70910010809197
:107CC000011090910210AEE0BDE0BF93AF93812C04
:107CD000912CE0EAAE2EE1E4BE2EFBE0CF2EF0E1E7
:107CE000DF2EE12CF12C00EA10E40F9476340F948F
:107CF0002D83F20185919591A591B4918093FF0F09
:107D000090930010A0930110B0930210F2013496EA
:107D100085919591A591B49180930310909304104F
:107D2000A0930510B093061063E070E18FEF9FE021
:107D30000F94F90AE0900710F090081000910910D4
:107D400010910A10209103103091041040910510F9
:107D5000509106106091FF0F7091001080910110FA
:107D600090910210BEE08B2EBDE09B2E9F928F92D1
:107D7000812C912CE6E1AE2EE3E4BE2E0F947634F6
:107D80000F942D830F900F900F900F90BAACBB20E3
:107D900081F06114710469F020E030E040E85FE3B5
:107DA00022966CAD7DAD8EAD9FAD22970F9473B6CC
:107DB00004C060E070E080E291EC0F9453138823DC
:107DC00009F48EC0C0900710D0900810E090091000
:107DD000F0900A10A701960160E070E080EA90E45C
:107DE0000F9473B62DEC3CEC4CEC5DE30F940DB1AD
:107DF00087FD7BC02AAD2223A1F0A7019601229620
:107E00006CAD7DAD8EAD9FAD22970F9473B69F770D
:107E100020E030E040E85FE30F94BFB818160CF4A0
:107E200069C0C090660DD090670DE090680DF0902D
:107E3000690D80910F078823A9F00F941E0C8823E9
:107E400089F0C701B6010E943B9F20914F103091ED
:107E5000501040915110509152100F9462B79B01F5
:107E6000AC0103C020E030E0A901A7E024968EAD6C
:107E70009FAD2497A89F8001A99F100D1124020D8A
:107E8000131D000F111F000F111F0E581A4E609185
:107E90000710709108108091091090910A100F94AA
:107EA00073B6F80161837283838394838091EE0EAD
:107EB0009091EF0E01979093EF0E8093EE0EFFEFEF
:107EC0006F1A7F0A81E00E9483A628E0420E511CAF
:107ED00039E06316710409F08BCE412C512C0EC091
:107EE0000DEA402E02E2502E09C01EE3412E13E19E
:107EF000512E04C0BBEF4B2EB2E15B2E80E090E030
:107F0000A0EAB0E48093071090930810A0930910A2
:107F1000B0930A1020910310309104104091051085
:107F2000509106106091FF0F709100108091011028
:107F300090910210EEE0FDE0FF93EF93812C912CE5
:107F4000E0EAAE2EE1E4BE2EFBE0CF2EF0E1DF2E24
:107F5000E12CF12C00EA10E40F9476340F942D8379
:107F60000F900F9049E06416710421F060E0C201A7
:107F70000C94B74A60968EAD9FAD60970F947D09C3
:107F80000E94648C60910C0D70910D0D072E000CF9
:107F9000880B990B0F9413B1905820914F1030918A
:107FA000501040915110509152100F9462B70E949E
:107FB000758C80EC9FE00F94E8B5082FCE010196F8
:107FC0009BAF8AAF10E08090930290909402A090B3
:107FD0009502B090960222968CAE9DAEAEAEBFAE2C
:107FE00022975FE7252E55E1352E66EC862E65E15A
:107FF000962E22962CAD3DAD4EAD5FAD22972983D6
:108000003A834B835C83AAADBBAD8D91BBAFAAAF66
:108010000F94959E882319F00F94819E1BC0013008
:1080200009F026C1123028F4112341F08EEB9FE0B5
:108030000AC0123031F08CEB9FE005C08FEB9FE05F
:1080400002C08DEB9FE00F94E8B5682F880F770B87
:10805000880B990B611571058105910509F408C11B
:108060000F9413B12FE632E143E85AE30F947AAA52
:108070006B017C019F7727E139ED4EEC5DE30F94B6
:10808000BFB818160CF033C0E8E0F0E684915F0149
:10809000882341F00F94FC0FFFEFAF1ABF0AF501E0
:1080A0008491F6CFE6E0F0E184915F01882341F00E
:1080B0000F94FC0FFFEFAF1ABF0AF5018491F6CFC2
:1080C00042E0C701B6010F949F10EDEFFFE08491ED
:1080D0007F01882341F00F94FC0FFFEFEF1AFF0A96
:1080E000F7018491F6CF8AE00F94FC0FC1C020E025
:1080F00030E040E05FE3C701B601123009F463C02D
:10810000133009F48AC0113071F10F947AAA2B014F
:108110003C0142E7A42E45E1B42EA3019201D50112
:1081200015966D917D918D919C9118970F9474B6D1
:10813000F5016583768387839087A7019601618126
:108140007281838194810F9474B6D50111966D93D9
:108150007D938D939C931497BCE1AB0EB11C8A1454
:108160009B04D9F685C00F947AAA2B013C0132E713
:10817000A32E35E1B32EA3019201F501658176812D
:10818000878190850F9474B6D50115966D937D9374
:108190008D939C931897A701960119966D917D91E7
:1081A0008D919C911C970F9474B6F501618772872D
:1081B00083879487FCE1AF0EB11C26ECA21625E163
:1081C000B206C9F655C00F947AAA2B013C0123E7E9
:1081D000A22E25E1B22EA3019201D5015C966D91EC
:1081E0007D918D919C915F970F9474B6F501648F8A
:1081F000758F868F978FA70196016081718182812B
:1082000093810F9474B6D5016D937D938D939D9357
:108210005D012A163B06F9F62BC00F947AAA2B01B2
:108220003C019FE8A92E95E1B92EA3019201F50129
:1082300060817181828193810F9474B6D5016D93B1
:108240007D938D939D935D01A701960158966D9145
:108250007D918D919C915B970F9474B6F501608F21
:10826000718F828F938FFBE9AF16F5E1BF06E9F6B8
:108270001F5F143009F0BDCE0F94824F81E08093D0
:1082800072150E94108DE0910E0D24E0E29FF00126
:108290001124ED57F04F20E030E04FE253E46081CD
:1082A0007181828193810F94BFB8181684F48091F4
:1082B0000F07882361F00F941E0C882341F08091F2
:1082C000120D9091130DC29714F00C94B56C81E0CF
:1082D00090E0909327028093260281EF94E10F941F
:1082E000AD2D28964EAD5FAD28975093400E40932C
:1082F0003F0E2C968EAD9FAD2C979093EF0E8093F2
:10830000EE0E1092580E34C180917215882309F434
:1083100095C0E3EFFFE084918F01882339F00F943B
:10832000FC0F0F5F1F4FF8018491F7CF67E070E0FB
:1083300080E090E00F948510E1EFFFE084918F01E1
:10834000882339F00F94FC0F0F5F1F4FF8018491C1
:10835000F7CF67E070E080E090E00F948510EEEDDD
:10836000FFE084918F01882339F00F94FC0F0F5F99
:108370001F4FF8018491F7CF65E070E080E090E056
:108380000F948510ECECFFE084918F01882339F085
:108390000F94FC0F0F5F1F4FF8018491F7CF8AE015
:1083A0000F94FC0F00E010E0B9EC6B2EBFE07B2EC9
:1083B00087ECA82E8FE0B82EE12CF12C4801F8EACA
:1083C0008F0E911CF3018491A9ECCA2EAFE0DA2E36
:1083D000882341F00F94FC0FFFEFCF1ADF0AF6015C
:1083E0008491F6CFF401EE0DFF1DEE58FA4E618137
:1083F00072818381948145E00F949F10F4E0EF0E29
:10840000F11C2CE1E216F104E9F6F5018491F7EC98
:10841000EF2EFFE0FF2E882341F00F94FC0FFFEFBB
:10842000EF1AFF0AF7018491F6CF0C5111090C33B2
:10843000FFEF1F0709F0C0CF0C945F6CE9EAFFE083
:1084400084918F01882311F40C94EC6A0F94FC0F33
:108450000F5F1F4FF8018491F5CF86EE0F94280C23
:108460000C945F6C109271190C945F6C85E40F94FE
:10847000959E811102C00F942D8368E3662E63E000
:10848000762E7FEFA72E7FE0B72EEBE98E2EE0E170
:108490009E2ED12CD3018D913D010F94959E882362
:1084A000C9F1B3E0DB120CC00F948C9EF501608320
:1084B0007183828393838BE090E10E94ADE02AC0B8
:1084C0000F948C9E9B01AC01D4016D917D918D9197
:1084D0009C910F9474B6F5016083718382839383BA
:1084E000E0900710F09008100091091010910A1008
:1084F0002091031030910410409105105091061006
:108500006091FF0F70910010809101109091021006
:108510000F94FB47D394F4E0AF0EB11C24E0820E1D
:10852000911C34E0D312B6CF0C945F6C81E0809341
:10853000FE0E0F94588A60936016709361168093B4
:108540006216909363166091FE0E84EC9FE00F9488
:10855000FAB569E277E081EC9FE00E9452D2109276
:10856000410E60E08FEF9FE00F94FAB50C945F6CC2
:1085700082E00E9483A60C945F6C80916D159091AF
:108580006E158D579C4E9F938F9384E99FE00C94BA
:108590002B348DE40F94959E882311F40C94FC6980
:1085A000E0914013F0914113319681918032E9F3CB
:1085B0008930D9F380538A3060F080916D159091A5
:1085C0006E158D579C4E9F938F938FE79FE00C9471
:1085D0002B340F948C9E0F94D3B7AB01BC01CA010E
:1085E0005093150D4093140D4B3C510511F40C9410
:1085F000E2520CF05CC14135510511F40C94E24D8E
:108600000CF0C1C04A31510509F4EEC3ACF5443158
:10861000510509F453C394F44131510509F444C39D
:1086200034F44230510508F48CC20C94E5694231AF
:10863000510511F40C94004E0C94E5694731510535
:1086400009F480C37CF44531510509F477C3463100
:10865000510511F00C94E569109266161092671698
:108660000C94F7694831510509F484C34931510527
:1086700009F4ADC30C94E5694032510509F4AEC567
:108680000CF05AC04D31510511F40C94F76954F4B3
:108690004B31510509F4B6C34C31510509F4A1C45D
:1086A0000C94E5694E31510509F4C7C44F315105A9
:1086B00011F00C94E5690F94588A00914F0E1091B7
:1086C000500E2091510E3091520E6B017C01C01A58
:1086D000D10AE20AF30AC701B60128EE33E040E00E
:1086E00050E00F9438B6CA01B9012CE330E040E005
:1086F00050E00F9438B67F936F93C701B60120E620
:108700003AEE40E050E00F9438B63F932F9380E765
:108710009FE09F938F938E010F5F1F4F1F930F93C7
:108720000F9471B0EAE2F0E684910FB6F894DEBFE0
:108730000FBECDBF7F01EDC54D32510509F44BC6CB
:10874000C4F44A32510509F4FFC54C32510511F009
:108750000C94E5698FEF0F94280C60E070E088EFCF
:108760009FE00F9414B60E9478910E945A910C9445
:10877000F7694F32510509F435C64934510509F4FA
:1087800077C60C94E5694E36510511F40C94054FEB
:108790000CF042C04C35510511F40C94814E0CF58F
:1087A0004435510511F40C94004E7CF442355105CA
:1087B00011F40C94FC4D4335510511F00C94E5690E
:1087C00081E0809350130C94F7694535510511F4FD
:1087D0000C94474E4635510511F40C94624E0C949E
:1087E000E5694A36510511F40C94AC4D54F4483601
:1087F000510509F49AC64936510509F4CBC60C94C3
:10880000E5694B36510511F40C94DC4D4D3651059C
:1088100009F4DFC70C94E5694837510511F40C944D
:108820000F510CF54237510511F40C942E505CF4A5
:108830004037510509F498C64137510511F40C949D
:10884000184F0C94E5694337510511F40C94554FBA
:108850004737510511F00C94E569E3E0F6E08491A7
:108860008F010C9418514E3B510511F40C94834C1C
:108870005CF44937510511F40C9413514C385105EF
:1088800009F477C60C94E569483C510511F40C9441
:108890003152493C510511F00C94E56948E3E42E4E
:1088A00043E0F42E03E410E1D12C0C949D52873F59
:1088B00041E0940711F40C944E5B0CF08AC08C32AA
:1088C00061E0960711F40C949755C4F5803D91052D
:1088D00011F40C948554A4F48D3C910511F40C947E
:1088E000805314F40C943B538E3C910511F40C947A
:1088F0002F548F3C910511F40C944E540C94E5695F
:108900008D3D910511F40C94135564F4813D91054E
:1089100011F40C94AD548C3D910511F40C94025556
:108920000C94E569823E910511F40C943455803F16
:10893000910511F40C94F7690C94E5698F35B1E059
:108940009B0711F40C94F7690CF58F32F1E09F0747
:1089500011F40C9438576CF48D3231E0930711F414
:108960000C94CF558E32914011F40C9423570C94F3
:10897000E569803351E0950711F40C948B568E35E0
:10898000914011F40C94FA680C94E569843FA1E0DD
:108990009A0711F40C94465B6CF48039E1E09E0771
:1089A00011F40C94FE5A8339914011F40C94025B3B
:1089B0000C94E569853F21E0920711F40C944A5B21
:1089C000863F914011F00C94E5690F9478110C9456
:1089D000F7698D3843E094070CF04FC08B3853E0B3
:1089E000950714F00C94F7698D3B62E0960711F43B
:1089F0000C9497690CF58835B2E09B0711F40C9440
:108A0000DD5E5CF48D3F914011F00C94E569EAE283
:108A1000F0E684918F010C94065E893522E092077E
:108A200011F40C94BF638A35924011F00C94E569FF
:108A30000E943DE70C94F7698C3543E0940711F4EC
:108A40000C94C2636CF48E3B62E0960711F40C94B4
:108A5000A3698335934011F40C941E5E0C94E56970
:108A60008D35B3E09B0711F40C94936484389340E4
:108A700011F40C94AF660C94E5698339F3E09F0719
:108A800011F40C943C683CF5803933E0930711F401
:108A90000C940A686CF48E3853E0950711F40C942A
:108AA000D5678F38934011F40C94D8670C94E5691E
:108AB0008139A3E09A0711F40C94F7698239934045
:108AC00011F00C94E569109218070E9491E00F9440
:108AD0000E1E0C94F7698639E3E09E0711F40C949E
:108AE000CA686CF4843923E0920711F40C9444684A
:108AF0008539934011F40C949A680C94E569803A96
:108B000043E0940709F4D6C3873E934011F00C94D8
:108B1000E5691092190F10929C0F8091230D90918E
:108B2000240DA091250DB091260D809342139093B2
:108B30004313A0934413B09345130F94FF850C94F3
:108B4000F769E0914013F09141138F010E5F1F4FC1
:108B500080E50F94959E882371F00F948C9E0F945E
:108B6000D9B76B017C01AA24A394672B682B692BCE
:108B700031F4A12C04C0A12CC12CD12C760183E5A9
:108B80000F94959E882391F00F948C9E20E030E006
:108B90004AE754E40F947AAA0F94D9B76B017C0189
:108BA000BB24B394672B682B692B09F4B12C6AE2C0
:108BB00070E0C8010F94B8BB009711F0DC011C9263
:108BC000F801CF0121912032E1F3A11007C0B110CB
:108BD00005C0222319F00F941F2F04C08AEE92E1E2
:108BE0000F94AD2D81E08093460E1092450E0F94A8
:108BF0002D830F94588A6093761970937719809318
:108C0000781990937919C114D104E104F10419F190
:108C10000F94588AC60ED71EE81EF91E84E090E015
:108C200090932702809326020F94588A6C157D0535
:108C30008E059F0510F00C94F76C0E947AAA8111A2
:108C40000C94F76C0F944F7D81E00F948E8380E03D
:108C50000E9483A6E9CF84E090E09093270280935E
:108C600026020E947AAA811109C00F944F7D81E0EB
:108C70000F948E8380E00E9483A6F3CF82E090E081
:108C8000909327028093260280916616882331F004
:108C90008FEE93E40F94AD2D0C94F76981EF94E17E
:108CA0000F94AD2D0C94F76981EE92E10F94AD2DE8
:108CB00017981698159814980C94F769E6E7F6E05B
:108CC00084918F01882339F00F94FC0F0F5F1F4FA1
:108CD000F8018491F7CF8AE00F94FC0F10924719A6
:108CE000109246198AEB96E10E94ABEB8BE1EAEB1E
:108CF000F6E1DE01119601900D928A95E1F740E0D0
:108D000050E0BE016F5F7F4F8DE094E00F940B7BCE
:108D1000CE0101960F944B0AE8E6F6E084918F01AC
:108D2000882339F00F94FC0F0F5F1F4FF8018491D7
:108D3000F7CF8AE00F94FC0F0C94F7690F944C194D
:108D40000C94F76980914013909141136AE270E0AE
:108D500004960F94B8BB009711F0DC011C9280912F
:108D600040139091411341E061E004960F949B14ED
:108D70000C94F76980916816811114C060E086E652
:108D80009FE00F94FAB560E088E69FE00F94FAB593
:108D900060E085E69FE00F94FAB560E084E69FE02E
:108DA0000F94FAB580916716882329F081E08093AB
:108DB0006616109268160F94588A60934F0E70933F
:108DC000500E8093510E9093520E0C94F76980913F
:108DD0006616882311F40C94F7691092661681E0E8
:108DE000809368160C94F76980916716882311F4B4
:108DF0000C94F76983E50F94959E81110C94036D93
:108E00000C94F76980916616882309F4B8C002E8CB
:108E100016E1F80181918F01882319F00F94FC0F5E
:108E2000F8CFEEE8FDE084918F01882339F00F94AC
:108E3000FC0F0F5F1F4FF8018491F7CFE9E5F5E0D4
:108E400084918F01882339F00F94FC0F0F5F1F4F1F
:108E5000F8018491F7CF6091411970914219809186
:108E60004319909144194AE00F941410ECE8FDE086
:108E700084918F01882339F00F94FC0F0F5F1F4FEF
:108E8000F8018491F7CF6091391970913A19809166
:108E90003B1990913C194AE00F9414108AE00F940A
:108EA000FC0F0F94588A40E6C42E4AEED42EE12CD3
:108EB000F12CA70196010F9438B649015A0160912F
:108EC0004F0E7091500E8091510E9091520EA7014D
:108ED00096010F9438B68401021B130BC8016CE392
:108EE00070E00F941EBBCB019927EAE0F0E0BF01D0
:108EF0000F9432BB282FCB01BF010F9432BB805D92
:108F00008093B619205D2093B7191092B81956EBCB
:108F1000E52E59E1F52E6701D6018D916D0188236B
:108F200019F00F94FC0FF8CF8AE30F94FC0FC801DF
:108F30006CE370E00F941EBB6AE070E00F9432BBEC
:108F4000605D6093B619805D8093B7191092B8196F
:108F5000F70181917F01882319F00F94FC0FF8CF5E
:108F6000EAE8FDE084918F01882311F40C94F769FD
:108F70000F94FC0F0F5F1F4FF8018491F5CF809184
:108F80006816882371F0EAE7FDE084918F01882359
:108F900009F4CFCE0F94FC0F0F5F1F4FF80184919F
:108FA000F6CF80913E0E882371F0EEE6FDE08491CD
:108FB0008F01882309F4BDCE0F94FC0F0F5F1F4F64
:108FC000F8018491F6CFEEE5FDE084918F018823CE
:108FD00009F4AFCE0F94FC0F0F5F1F4FF80184917F
:108FE000F6CF80914013909141136AE270E00496AD
:108FF0000F94B8BB8C01892BA9F080916D159091CD
:109000006E156EE470E08D579C4E0F94B8BB60E215
:1090100070E00F94B8BB0196909341138093401376
:10902000D8011C92809140139091411341E060E07F
:1090300004960F949B140C94F7698091671688230B
:1090400011F40C94F7690F94784580914013909136
:1090500041136AE270E004960F94B8BB8C01892B2F
:10906000A9F080916D1590916E156EE470E08D57AA
:109070009C4E0F94B8BB60E270E00F94B8BB0196B1
:109080009093411380934013F8011082C0904013D5
:10909000D090411386010C5F1F4F80916716882383
:1090A00011F40C94F7698CE898E10E944EEA109252
:1090B00066161F8E1AA28AEB96E19093D6168093BD
:1090C000D5160115110591F0D60114968C918F32A9
:1090D00039F4BE01615E7F4FC8010F946C4706C032
:1090E00087ED96E19093D6168093D5166091D516AC
:1090F0007091D61619821C8222E0A801CE01019639
:109100000E94D4F38823A1F0CE0101960F94797ABE
:10911000882371F061E0CE0101960E9457EA009722
:1091200039F025EEFC0120831C820F94825AF82E20
:10913000CE0101960F944B0AFF2021F1E0E5FDE0FE
:1091400084917F01882341F00F94FC0FFFEFEF1A09
:10915000FF0AF7018491F6CFD8018D918D01882304
:1091600019F00F94FC0FF8CF8AE00F94FC0F1092C7
:1091700041191092421910924319109244190F94F8
:10918000391726C0E8E3FDE084917F01882341F090
:109190000F94FC0FBFEFEB1AFB0AF7018491F6CF97
:1091A000D8018D918D01882319F00F94FC0FF8CF11
:1091B000E6E3FDE084918F01882339F00F94FC0FE2
:1091C0000F5F1F4FF8018491F7CF8AE00F94FC0FD7
:1091D000CE014F960F944B0A0C94F7698091661656
:1091E00081110F942D8300914013109141130C5F56
:1091F0001F4F6AE270E0C8010F94B8BB7C0161E2C6
:1092000070E0C8010F94B8BB009719F08C010F5F94
:109210001F4FE114F10411F0D7011C9280E50F9467
:10922000959EF82E809140139091411308171907CD
:1092300008F4F12C80916716882311F40C94F769D7
:1092400041E04F2561E0C8010F949B1483E50F9422
:10925000959E8823B9F08091401390914113801717
:10926000910780F40F94819EAB01BC01409341199A
:109270005093421960934319709344198CE898E114
:109280000E9464E980916716882329F081E0809329
:10929000661610926816F1100C94F7690F94588AAC
:1092A00060934F0E7093500E8093510E9093520E18
:1092B0000C94F76980914013909141136AE270E039
:1092C00005960F94B8BB8C01892BA9F080916D1580
:1092D00090916E156EE470E08D579C4E0F94B8BB64
:1092E00060E270E00F94B8BB0196909341138093B5
:1092F0004013F8011082809140139091411321E0B6
:109300002093651641E060E005960F949B140C9441
:10931000F769882341F00F94FC0F3FEFE31AF30A3B
:10932000F7018491F6CF7801D7018D917D018823D3
:1093300019F00F94FC0FF8CF8AE00F94FC0FC801CE
:109340000F941F2F0C94F76983E50F94959E882343
:1093500011F40C94F7690F948C9E0F94D3B7F62EEA
:10936000E72E862F9E2D8C0180E50F94959E8823F5
:1093700031F00F3F110509F010F40C94146D0DE05D
:1093800010E0E7E9F2E0819191918017910711F4E3
:109390000C94F769B2E0EF3CFB07A9F70630110522
:1093A00039F48F2D9E2D9093BF198093BE1904C060
:1093B00017FF02C00C94F76961E0802F0F943D887D
:1093C0006F2D802F0F940F886F2D7E2D802F0F947F
:1093D00079880C94F7698AE50F94959E0E946C71C8
:1093E0000C94F76984E090E0909327028093260222
:1093F0000E94FEA70F944F7D81E00F948E8360E062
:1094000080E00E94C6A787E29DE00E94F1A661E08D
:1094100080E00E94C6A71E9903C081E29DE002C0C1
:1094200084E29DE00E94F1A662E080E00E94C6A76F
:109430001D9903C08BE19DE002C08EE19DE00E947A
:10944000F1A663E080E00E94C6A71C9903C085E1F5
:109450009DE002C088E19DE00E94F1A60E947AAAE8
:10946000882341F20E94FEA70F94608B0C94F76949
:1094700080E50F94959E882331F00F948C9E0F9475
:10948000D9B760933F0282E50F94959E882341F0FF
:109490000F948C9E0F94D9B770934302609342024D
:1094A00081E50F94959E882331F00F948C9E0F9444
:1094B000D9B760933E0283E50F94959E882341F0CF
:1094C0000F948C9E0F94D9B7709341026093400221
:1094D000809143028F93809142028F9380913F024B
:1094E0001F928F9384E296E09F938F930BE216E096
:1094F0001F930F930F9418B0809141028F93809126
:1095000040028F9380913E021F928F938DE196E0EF
:109510009F938F931F930F930F9418B00FB6F894E7
:10952000DEBF0FBECDBF0C94F769BE016F5F7F4FEA
:1095300088E690E00F94349C81110C94F76983E5E0
:109540000F94959E882311F40C94F76919810F9458
:109550008C9E11110C94F7690F94D3B7709370150A
:1095600060936F150C94F76963E08CE196E00E94BC
:1095700011A683E50F94959E882311F40C94F76946
:109580000F948C9E0F94D3B77093130D6093120DAC
:109590000C94F769BE016F5F7F4F89E690E00F94EE
:1095A000349C81110C94F769EAE6FFE084918F0105
:1095B000882339F00F94FC0F0F5F1F4FF80184913F
:1095C000F7CFE98124E0E29FF0011124ED57F04F3D
:1095D000608171818281938141E00F949F10E7E661
:1095E000FFE084918F01882339F00F94FC0F0F5F07
:1095F0001F4FF8018491F7CFE981F0E0EE0FFF1FD4
:10960000E159FA4E60817181072E000C880B990B8D
:109610000F9413B141E00F949F10E3E6FFE08491B3
:109620008F01882339F00F94FC0F0F5F1F4FF80153
:109630008491F7CF609108077091090780910A071C
:1096400090910B0741E00F949F10E0E6FFE08491BA
:109650008F01882339F00F94FC0F0F5F1F4FF80123
:109660008491F7CF6091120D7091130D072E000CAD
:10967000880B990B0F9413B141E00F949F10EDE507
:10968000FFE084918F01882339F00F94FC0F0F5F66
:109690001F4FF8018491F7CF60E070E0CB010F9489
:1096A0008510EBE5FFE084918F01882339F00F945A
:1096B000FC0F0F5F1F4FF8018491F7CF6091830F6C
:1096C0007091840F8091850F9091860F41E00F94E7
:1096D0009F10E8E5FFE084918F01882339F00F9413
:1096E000FC0F0F5F1F4FF8018491F7CF60916F154A
:1096F00070917015072E000C880B990B0F9413B105
:1097000041E00F949F10E4E5FFE084918F018823EE
:1097100039F00F94FC0F0F5F1F4FF8018491F7CFC2
:10972000E981F0E0E95EF04F608170E080E090E078
:109730000F948510EFE4FFE084918F01882339F0C6
:109740000F94FC0F0F5F1F4FF8018491F7CF6091CA
:10975000160F70E080E090E00F948510EBE4FFE0DE
:1097600084918F01882339F00F94FC0F0F5F1F4FF6
:10977000F8018491F7CF6091660D7091670D80912B
:10978000680D9091690D41E00F949F10E7E4FFE0B0
:1097900084918F01882339F00F94FC0F0F5F1F4FC6
:1097A000F8018491F7CF6091620D7091630D809103
:1097B000640D9091650D41E00F949F108AE00F9425
:1097C000FC0F81E090E090932702809326020C9496
:1097D0005271BE016F5F7F4F8DE690E00F94349C15
:1097E00081110C94F76988E19BE20F94AD2D81E023
:1097F00090E090934E0D80934D0D8091FE0E882346
:1098000029F060E081E090E00E94F8F683E50F9493
:10981000959E882379F019810F948C9E111106C0B2
:109820000F94D3B77093701560936F1581E0809398
:10983000040212C082E50F94959E882369F0198175
:109840000F948C9E111106C00F94D3B770937015AE
:1098500060936F15109204020F94588A4B015C01BB
:10986000F9800F2D10E0F801EE0FFF1FE159FA4EBD
:1098700060817181072E000C880B990B0F9413B136
:10988000F801EE0FFF1FEE0FFF1FED57F04F11E035
:1098900020813181428153810F94BFB818160CF09A
:1098A00010E01093270D81E090E0909327028093C1
:1098B00026021092590E4F2DC501B4010E946DA3CE
:1098C0008AE09BE20F94AD2D82E090E09093270216
:1098D0008093260290934E0D80934D0D8091FE0E45
:1098E000882329F060E082E090E00E94F8F60F946F
:1098F000588A6093761970937719809378199093AA
:1099000079190C94F7698EEF9AE20F94AD2D83E0EC
:1099100090E090934E0D80934D0D8091FE0E882324
:1099200029F060E081E090E00E94F8F683E50F9472
:10993000959E882361F00F948C9E0F94D3B77093FB
:10994000130D6093120D81E0809304020FC082E535
:109950000F94959E882351F00F948C9E0F94D3B74B
:109960007093130D6093120D109204020F94588A95
:109970004B015C011092590E6091120D7091130D04
:10998000072E000C880B990B0F9413B111E0209156
:1099900008073091090740910A0750910B070F946F
:1099A000BFB818160CF010E01093270D81E090E07E
:1099B000909327028093260204E41FE0B0E4EB2E8C
:1099C000BFE0FB2E8CE3C82E8FE0D82E8091270DB0
:1099D0006091120D7091130D8823B9F08091590E8A
:1099E000811113C0072E000C880B990B0F9413B133
:1099F000209108073091090740910A0750910B0701
:109A00000F94BFB81816BCF08BC0072E000C880B43
:109A1000990B0F9413B120910807309109074091D9
:109A20000A0750910B070F940DB187FF79C0809101
:109A30000402811175C00F94588ADC01CB0188198A
:109A40009909AA09BB09893E9340A105B10508F40B
:109A50005EC08091FE0E811156C0E0910E0D24E093
:109A6000E29FF0011124ED57F04F40805180628059
:109A70007380F8018491A4E4AA2EAFE0BA2E882363
:109A800041F00F94FC0FFFEFAF1ABF0AF50184916C
:109A9000F6CF42E0C301B2010F949F10F701849109
:109AA000F0E4AF2EFFE0BF2E882341F00F94FC0FAF
:109AB000FFEFAF1ABF0AF5018491F6CF60910E0D4A
:109AC00070E080E090E00F948510F6018491ECE363
:109AD000AE2EEFE0BE2E882341F00F94FC0FFFEF77
:109AE000AF1ABF0AF5018491F6CF60910807709113
:109AF000090780910A0790910B0741E00F949F108E
:109B00008AE00F94FC0F0F94588A4B015C010F946C
:109B10004F7D80E00F948E8380E00E9483A656CF15
:109B200085EF9AE20F94AD2D82E090E090932702AA
:109B30008093260284E090E090934E0D80934D0D2B
:109B40000F94588A609376197093771980937819D7
:109B5000909379190C94F76983E50F94959E882367
:109B600019F10F948C9E20E030E0A9010F940DB103
:109B700087FD0FC00F948C9E20E030E04FE753E448
:109B80000F94BFB8181644F00F948C9E0F94D3B75F
:109B900005C060E070E002C06FEF70E07093BF1925
:109BA0006093BE190C94F7698FEF90E09093BF1902
:109BB0008093BE190C94F7691092BF191092BE19C8
:109BC0000C94F7690F9419200F942D83149A0F9415
:109BD00085831092BF191092BE1968EE73E080E081
:109BE00090E00F9440898EE094E00F94AD2D80E0DA
:109BF0000E9483A60C94F769109250130C94F76995
:109C000083E50F94959E882399F00F948C9E20E015
:109C100030E04AE754E40F947AAA0F94D9B76093DE
:109C20008E0270938F0280939002909391021DC0D8
:109C300088E50F94959E81110C941B6D89E50F9416
:109C4000959E81110C941B6D8AE50F94959E811150
:109C50000C941B6D85E40F94959E81110C941B6DE3
:109C60000F942D83149A0F9485838FEF9FEF909319
:109C7000430280934202909341028093400280937A
:109C80003F0280933E02109251130C94F76983E5D2
:109C90000F94959E882311F40C94F7690F948C9E71
:109CA00020E030E04AE754E40F947AAA0F94D9B741
:109CB0006093721970937319809374199093751946
:109CC0000C94F76983E50F94959E882311F40C9406
:109CD000F7690F948C9E20E030E04AE754E40F943B
:109CE0007AAA0F94D9B760938A0270938B028093FB
:109CF0008C0290938D028FE496E10F94745A0C9429
:109D0000F76928E333E03BAF2AAF03E410E172E7E1
:109D1000C72E7DE0D72EF12CAAADBBAD8D91BBAF88
:109D2000AAAF0F94959E882309F463C0B3E0FB1299
:109D300059C00F948C9E2B013C0120E030E040EA9A
:109D400051E40F940DB187FF45C0A3019201F801C2
:109D500064817581868197810F9462B74B015C01A4
:109D60009B01AC01609197107091981080919910AF
:109D700090919A100F947AAA60939710709398100C
:109D80008093991090939A10209050023090510235
:109D9000A5019401D1011C966D917D918D919C91AD
:109DA0001F970F947AAAF101648775878687978732
:109DB000D6016D917D918D919C910F9411B1A5016A
:109DC00094010F947AAA0F94D9B7F6016083718336
:109DD00082839383D80114964D925D926D927C920A
:109DE000179707C00F948C9EF80164837583868350
:109DF0009783F3940C5F1F4FF4E0CF0ED11C64E007
:109E0000862EF81089CF0C94F7698EE40F94959EF6
:109E1000882311F40C94F7690F94819E6093421388
:109E20007093431380934413909345130C94F769F4
:109E300083E50F94959E882379F08091401390914B
:109E400041134AE050E060E070E001960F94A2AC4C
:109E5000609360020C94F769EAE2F0E684918F0166
:109E6000882339F00F94FC0F0F5F1F4FF801849186
:109E7000F7CFC0906002D12CE12CF12CE5E3FFE09C
:109E800084918F01882339F00F94FC0F0F5F1F4FCF
:109E9000F8018491F7CF4AE0C701B6010F9414107E
:109EA0008AE00F94FC0F0C94F76986E50F94959E59
:109EB000882379F0E4E3F9E584918F01882311F494
:109EC0000C9499460F94FC0F0F5F1F4FF80184917B
:109ED000F5CF85E50F94959E382E8823D9F1E09033
:109EE0004013F0904113FFEFEF1AFF0AF092411375
:109EF000E0924013270167014601D6018D916D0163
:109F000090ED980F9A30C0F38E3211F00C94F769EF
:109F10005D013501F50181915F0190ED980F9A3057
:109F2000C0F38E3211F00C94F769CF018C01DC0183
:109F30002C90019620ED220D2A30C0F3822D0F9433
:109F4000832D81110C943A6DBDE22B120C94F769AC
:109F50000C943A6DE7E1FFE084918F01882339F09A
:109F60000F94FC0F0F5F1F4FF8018491F7CFE4E3CC
:109F7000F9E584918F01882339F00F94FC0F0F5F6E
:109F80001F4FF8018491F7CFEDEBFEE084918F0134
:109F9000882339F00F94FC0F0F5F1F4FF801849155
:109FA000F7CFE9EBFEE084918F01882339F00F941D
:109FB000FC0F0F5F1F4FF8018491F7CFEAEAFEE034
:109FC00084918F01882339F00F94FC0F0F5F1F4F8E
:109FD000F8018491F7CFEDE9FEE084918F018823A9
:109FE00039F00F94FC0F0F5F1F4FF8018491F7CFEA
:109FF000ECE8FEE084918F01882339F00F94FC0F88
:10A000000F5F1F4FF8018491F7CFEAE8FEE08491DB
:10A010008F01882339F00F94FC0F0F5F1F4FF80159
:10A020008491F7CFE3E8FEE084918F01882339F033
:10A030000F94FC0F0F5F1F4FF8018491F7CFEEE5EF
:10A04000FEE084918F01882311F40C9499460F94BB
:10A05000FC0F0F5F1F4FF8018491F5CFE1E1FDE0A8
:10A0600084918F01882339F00F94FC0F0F5F1F4FED
:10A07000F8018491F7CF6091FF0F709100108091EB
:10A0800001109091021042E00F949F10EDE0FDE06E
:10A0900084918F01882339F00F94FC0F0F5F1F4FBD
:10A0A000F8018491F7CF60910310709104108091B2
:10A0B00005109091061042E00F949F10E9E0FDE03A
:10A0C00084918F01882339F00F94FC0F0F5F1F4F8D
:10A0D000F8018491F7CF609107107091081080917A
:10A0E000091090910A1042E00F949F10E5E0FDE006
:10A0F00084918F01882339F00F94FC0F0F5F1F4F5D
:10A10000F8018491F7CF60910B1070910C10809141
:10A110000D1090910E1042E00F949F10EEE4F5E0C8
:10A1200084918F01882339F00F94FC0F0F5F1F4F2C
:10A13000F8018491F7CF80E00F940C830F9413B152
:10A1400020914710309148104091491050914A1089
:10A150000F9462B742E00F949F10E1E0FDE084911C
:10A160008F01882339F00F94FC0F0F5F1F4FF80108
:10A170008491F7CF81E00F940C830F9413B1209159
:10A180004B1030914C1040914D1050914E100F9447
:10A1900062B742E00F949F10EDEFFCE084918F01D5
:10A1A000882339F00F94FC0F0F5F1F4FF801849143
:10A1B000F7CF82E00F940C830F9413B120914F10CE
:10A1C0003091501040915110509152100F9462B73D
:10A1D00042E00F949F10E9EFFCE084918F01882307
:10A1E00039F00F94FC0F0F5F1F4FF8018491F7CFE8
:10A1F00083E00F940C830F9413B12091531030918E
:10A20000541040915510509156100F9462B742E08F
:10A210000F949F108AE00F94FC0F0C94F769109232
:10A2200025020C94F76981E0809325020C94F7696C
:10A23000882339F00F94FC0F0F5F1F4FF8018491B2
:10A24000F7CF8AE00F94FC0FEBEFF5E084918F01DC
:10A25000882339F00F94FC0F0F5F1F4FF801849192
:10A26000F7CF1E9B0DC0E7EDF2E184918F018823AB
:10A27000A1F00F94FC0F0F5F1F4FF8018491F7CFEF
:10A28000E2EDF2E184918F01882339F00F94FC0F05
:10A290000F5F1F4FF8018491F7CF8AE00F94FC0FF6
:10A2A000E3EFF5E084918F01882339F00F94FC0FE0
:10A2B0000F5F1F4FF8018491F7CF8091060182FF55
:10A2C0000DC0E7EDF2E184918F018823A1F00F9496
:10A2D000FC0F0F5F1F4FF8018491F7CFE2EDF2E121
:10A2E00084918F01882339F00F94FC0F0F5F1F4F6B
:10A2F000F8018491F7CF8AE00F94FC0FEBEEF5E0C4
:10A3000084918F01882339F00F94FC0F0F5F1F4F4A
:10A31000F8018491F7CF1D9B0DC0E7EDF2E1849128
:10A320008F018823A1F00F94FC0F0F5F1F4FF801DE
:10A330008491F7CFE2EDF2E184918F01882339F027
:10A340000F94FC0F0F5F1F4FF8018491F7CF8AE045
:10A350000F94FC0FE3EEF5E084918F01882339F030
:10A360000F94FC0F0F5F1F4FF8018491F7CF80917E
:10A37000060187FF0DC0E7EDF2E184918F0188238C
:10A38000A1F00F94FC0F0F5F1F4FF8018491F7CFDE
:10A39000E2EDF2E184918F01882339F00F94FC0FF4
:10A3A0000F5F1F4FF8018491F7CF8AE00F94FC0FE5
:10A3B000EBEDF5E084918F01882339F00F94FC0FC9
:10A3C0000F5F1F4FF8018491F7CF1C9B0DC0E7ED85
:10A3D000F2E184918F018823A1F00F94FC0F0F5FAD
:10A3E0001F4FF8018491F7CFE2EDF2E184918F01E4
:10A3F000882339F00F94FC0F0F5F1F4FF8018491F1
:10A40000F7CF8AE00F94FC0FE3EDF5E084918F0124
:10A41000882339F00F94FC0F0F5F1F4FF8018491D0
:10A42000F7CF01990FC0E7EDF2E184918F01882306
:10A4300011F40C9499460F94FC0F0F5F1F4FF80115
:10A440008491F5CFE2EDF2E184918F01882311F43C
:10A450000C9499460F94FC0F0F5F1F4FF8018491E5
:10A46000F5CF10910E0D84E50F94959E882301F190
:10A470000F948C9E0F94D9B7162F6623C9F0EAE289
:10A48000F0E684918F01882339F00F94FC0F0F5F61
:10A490001F4FF8018491F7CF0BEB12E1D8018D919A
:10A4A0008D01882311F40C94F7690F94FC0FF6CFFB
:10A4B00084E40F94959E882311F40C94F7690F940B
:10A4C0008C9E20E030E0A9010F940DB1811103C0F2
:10A4D0001092DA102EC00F948C9EB4E01B9FF001F6
:10A4E0001124E552FF4E6083718382839383C09071
:10A4F000DB10D090DC10E090DD10F090DE1020E05A
:10A5000030E0A901C701B6010F940DB1811106C059
:10A51000C12CD12C50EEE52E5FE3F52EC092DB105E
:10A52000D092DC10E092DD10F092DE1081E080939A
:10A53000DA100E94E1A40C94F769F70181917F0180
:10A540000F94959E8823A1F10F948C9E0F94D9B7F8
:10A55000F1E0FD15ACF0653C29E07207810591053D
:10A56000A0F4562F472F382F292F613CA3E07A07FC
:10A570008105910590F050EC43E030E020E00DC003
:10A58000562F472F382F292F08C050EC43E030E0DA
:10A5900020E064EC79E080E090E0F80164A375A32A
:10A5A00086A397A3E455FF4F5083418332832383CF
:10A5B000D3940C5F1F4FF4E0DF12BFCF0E944FE037
:10A5C0000C94F76928E3A22E23E0B22E33E4C32EC5
:10A5D00030E1D32E912CD5018D915D010F94959E84
:10A5E000882309F43EC00F948C9E7B018C01B1E05E
:10A5F000B91514F120E030E048E453E40F94BFB8FB
:10A6000018163CF4512C612C88E4782E93E4892EA2
:10A6100004C05E2C6F2C702E812E20E030E048ECC0
:10A6200052E4B701C8010F94BFB818164CF4E12CDE
:10A63000F12C08EC12E404C0562E6F2C782E812EDB
:10A64000852D962DA72DB82DF601848B958BA68B85
:10A65000B78BC701D801E456FF4F80839183A28353
:10A66000B3839394F4E0CF0ED11C14E0812E9810A4
:10A67000B2CF0C94F76983E50F94959E8823E9F097
:10A680000F948C9E6093771070937810809379105C
:10A6900090937A1084E50F94959E882311F40C947E
:10A6A000F7690F948C9E60937B1070937C1080935D
:10A6B0007D1090937E100C94F76980E50F94959E21
:10A6C000882351F00F948C9E6093771070937810CC
:10A6D0008093791090937A1082E50F94959E882349
:10A6E00051F00F948C9E60937B1070937C1080933C
:10A6F0007D1090937E1084E50F94959E0C94F769DD
:10A7000083E50F94959E882351F00F948C9E60935F
:10A710007F1070938010809381109093821084E555
:10A720000F94959E882351F00F948C9E6093831014
:10A7300070938410809385109093861082E40F9418
:10A74000959E882361F00F948C9E0F94D9B76093E7
:10A750008710709388108093891090938A1088E5F1
:10A760000F94959E882391F00F948C9E60938F1088
:10A7700070939010809391109093921060938B102F
:10A7800070938C1080938D1090938E1089E50F94A8
:10A79000959E882351F00F948C9E60938F10709338
:10A7A000901080939110909392108AE50F94959E4B
:10A7B000882351F00F948C9E6093931070939410A3
:10A7C000809395109093961085E40F94959E88231E
:10A7D00051F00F948C9E6093971070939810809313
:10A7E000991090939A1020E030E040E251E460919B
:10A7F0008B1070918C1080918D1090918E100F9411
:10A80000BFB8181664F480E090E0A0E2B1E4809351
:10A810008B1090938C10A0938D10B0938E1020E02D
:10A8200030E040E251E460918F107091901080917F
:10A830009110909192100F94BFB8181614F00C94C8
:10A84000F76980E090E0A0E2B1E480938F109093EC
:10A850009010A0939110B09392100C94F769A8E314
:10A86000EA2EA3E0FA2E0BE910E1B7EACB2EB0E115
:10A87000DB2ED7018D917D010F94959E882339F0B1
:10A880000F948C9EF80160837183828393830C5FA5
:10A890001F4FC016D10669F70C94F76983E50F9432
:10A8A000959E882351F00F948C9E6093C6107093F0
:10A8B000C7108093C8109093C91086E40F94959E9A
:10A8C000882381F00F948C9E20E030E040E752E432
:10A8D0000F9462B76093CA107093CB108093CC1022
:10A8E0009093CD108AE50F94959E882311F40C94D3
:10A8F000F7690F948C9E6093CE107093CF10809365
:10A90000D0109093D1100C94F76983E50F94959E25
:10A91000882351F00F948C9E6093D2107093D310C3
:10A920008093D4109093D51086E40F94959E88233D
:10A9300011F40C94F7690F948C9E20E030E040E70E
:10A9400052E40F9462B76093D6107093D71080933F
:10A95000D8109093D9100C94F76983E50F94959EC5
:10A96000882311F40C94F7690F948C9E0F94D3B73D
:10A970006115710551F06130710569F481E08093D2
:10A98000C5101092FF0E0C94F7691092C51010922A
:10A99000FF0E0C94F769EAE2F0E684918F018823B8
:10A9A00039F00F94FC0F0F5F1F4FF8018491F7CF20
:10A9B000E0ECF5E084918F01882339F00F94FC0FCF
:10A9C0000F5F1F4FF8018491F7CF00916D15109123
:10A9D0006E150D571C4ED8018D918D01882319F0ED
:10A9E0000F94FC0FF8CFE9E5FEE084918F018823F6
:10A9F00011F40C9499460F94FC0F0F5F1F4FF80150
:10AA00008491F5CF83E50F94959E882311F40C94DF
:10AA1000F7690F948C9E0F94D3B770935A0260938A
:10AA200059020C94F76983E50F94959E882309F4E5
:10AA300080CD0F948C9E0F94D3B76B017C0184E57D
:10AA40000F94959E882359F0BE016F5F7F4F8DED67
:10AA500090E00F94349C81110C94F7696ACDD092E8
:10AA60006402C092630265CD80E50F94959E8823B1
:10AA700011F40C94F7690F948C9E0F94D3B7D62ED3
:10AA8000862F972F7C0183E50F94959E882331F0C4
:10AA90000F948C9E0F94D3B78B0102C00FEF1FEF62
:10AAA000C8010196039710F00C94F769E7E9F2E00A
:10AAB0008FEC92E021913191E216F30611F40C949F
:10AAC000F7698E179F07B1F7F7FE02C00C94F7697C
:10AAD0000F942D83FD2C60E08D2D0F943D880F3F4A
:10AAE000FFEF1F0731F00130110571F401E010E0B4
:10AAF0000DC08D2D0F944EAA31E020E0892B09F076
:10AB000030E0032F122F02C000E010E08F2D0F94D1
:10AB10004EAA8017910711F40C94F7690F944F7D9A
:10AB200080E00F948E8380E00E9483A6EFCF83E5C0
:10AB30000F94959E882331F00F948C9E0F94D3B779
:10AB40008B0102C00EE610E080E50F94959E8823ED
:10AB500029F00F948C9E0F94D3B702C068EE73E077
:10AB60006B01770FEE08FF081016110694F4809120
:10AB7000010790910207029718F4C8010F948D4CB9
:10AB8000C701B6010F94408984E50F9411290C94F4
:10AB9000F769C701B6010F9440890C94F76980E505
:10ABA0000F94959E882351F00F948C9E6093AB1068
:10ABB0007093AC108093AD109093AE1089E40F9415
:10ABC000959E882381F00F948C9E2CEA35EC47E209
:10ABD0005EE30F947AAA6093AF107093B0108093E5
:10ABE000B1109093B21084E40F94959E882381F065
:10ABF0000F948C9E2CEA35EC47E25EE30F9462B72B
:10AC00006093B3107093B4108093B5109093B61006
:10AC100083E40F94959E882351F00F948C9E60934B
:10AC200000027093010280930202909303020F943A
:10AC3000E481EFE8F7E184918F01882339F00F94E4
:10AC4000FC0F0F5F1F4FF8018491F7CF0BE114E069
:10AC5000D8018D918D01882319F00F94FC0FF8CF46
:10AC60006091AB107091AC108091AD109091AE10CE
:10AC700042E00F949F100FE114E0F80181918F01E1
:10AC8000882319F00F94FC0FF8CF2CEA35EC47E23B
:10AC90005EE36091AF107091B0108091B11090910F
:10ACA000B2100F9462B742E00F949F1003E214E0D9
:10ACB000D8018D918D01882319F00F94FC0FF8CFE6
:10ACC0002CEA35EC47E25EE36091B3107091B4106A
:10ACD0008091B5109091B6100F947AAA42E00F942B
:10ACE0009F1007E214E0F80181918F01882319F089
:10ACF0000F94FC0FF8CF60910002709101028091D7
:10AD000002029091030242E00F949F108AE00F9498
:10AD1000FC0F0C94F76980E50F94959E882351F001
:10AD20000F948C9E6093B7107093B8108093B910F5
:10AD30009093BA1089E40F94959E882381F00F9424
:10AD40008C9E2CEA35EC47E25EE30F947AAA60937E
:10AD5000BB107093BC108093BD109093BE1084E420
:10AD60000F94959E882381F00F948C9E2CEA35ECED
:10AD700047E25EE30F9462B76093BF107093C01018
:10AD80008093C1109093C2100F94E481EFE8F7E133
:10AD900084918F01882339F00F94FC0F0F5F1F4FB0
:10ADA000F8018491F7CF0BE114E0D8018D918D016A
:10ADB000882319F00F94FC0FF8CF6091B7107091B1
:10ADC000B8108091B9109091BA1042E00F949F1082
:10ADD0000FE114E0F80181918F01882319F00F949D
:10ADE000FC0FF8CF2CEA35EC47E25EE36091BB1034
:10ADF0007091BC108091BD109091BE100F9462B7FD
:10AE000042E00F949F1003E214E0D8018D918D0170
:10AE1000882319F00F94FC0FF8CF2CEA35EC47E2A9
:10AE20005EE36091BF107091C0108091C11090914D
:10AE3000C2100F947AAA42E00F949F108AE00F94F8
:10AE4000FC0F0C94F76983E50F94959E882319F005
:10AE50000F948C9E03C060E070E0CB0160936A02A7
:10AE600070936B0280936C0290936D020C94F7695F
:10AE700085E40F94959E882359F00F948C9E0F942F
:10AE8000D3B724967FAF6EAF249777FF05C013C06A
:10AE900024961FAE1EAE249763961FAE63976496EA
:10AEA0001FAE649726E166962FAF669733E46896E7
:10AEB0003FAF68970EC063961FAE639764961FAE50
:10AEC00064974CE866964FAF669752E468965FAF1A
:10AED000689783E50F94959E882371F00F948C9E5C
:10AEE00063966FAF639764967FAF649766968FAFF4
:10AEF000669768969FAF689783E40F94959E882322
:10AF000049F00F948C9E0F94D3B7A7967FAF6EAF86
:10AF1000A79706C085E090E0A7969FAF8EAFA79752
:10AF2000A7968EAC9FACA79790924A0D8092490D40
:10AF30001092ED0E10924C0D10924B0D0F94588AFA
:10AF400062966CAF7DAF8EAF9FAF62972496AEAC2A
:10AF5000BFAC2497B7FC05C02AE0A8962FAFA897EE
:10AF600004C03DE2A8963FAFA8970F94588AE49694
:10AF70006CAF7DAF8EAF9FAFE49724968EAC9FAC45
:10AF8000249718141904B4F40BE214E0D8018D913D
:10AF90008D01882319F00F94FC0FF8CF8AE00F94ED
:10AFA000FC0F81E08093ED0E10924C0D10924B0D32
:10AFB0000C94F76905E514E0F80181918F0188236D
:10AFC00019F00F94FC0FF8CF8AE00F94FC0F0F9448
:10AFD000192024968EAC9FAC24978FE7892809F41A
:10AFE00051C08093160F62968CAC9DACAEACBFACDA
:10AFF00062976D968CAE9DAEAEAEBFAE6D97E0968D
:10B000008CAE9DAEAEAEBFAEE0972B961FAE2B972B
:10B010006E961FAE6E9720E46F962FAF6F973CE150
:10B02000A0963FAFA09746E4A1964FAFA197A296F6
:10B030001FAEA297A3961FAEA397A4961FAEA49788
:10B04000A5961FAEA597EFE78E2E912CA12CB12CC3
:10B050002A968CAE9DAEAEAEBFAE2A97FFE74F2EBE
:10B06000512C612C712CAC961CAE1DAE1EAE1FAEC9
:10B07000AC9721E0E9962FAFE9971AAE1EAE212CCE
:10B08000312C06C08093170FAECF80E00E9483A6BC
:10B09000A8958091180F882309F474C10F9435275F
:10B0A00024968EAC9FAC2497892859F49090830FF6
:10B0B0009AAEA090840FAEAE2090850F3090860F90
:10B0C0000AC0B0900807BAAE809009078EAE2090F3
:10B0D0000A0730900B072AAD3EADA101A2966FADD5
:10B0E000A297A3967FADA397A4968FADA497A5969C
:10B0F0009FADA5970F94BFB8181674F09AACA2969E
:10B100009FAEA297AEACA396AFAEA397A4962FAE78
:10B11000A497A5963FAEA5976E962FAD6E976F96A6
:10B120003FAD6F97A0964FADA097A1965FADA19749
:10B130006AAD7EADC1010F94BFB8181674F0BAACF9
:10B140006E96BFAE6E978EAC6F968FAE6F97A096D1
:10B150002FAEA097A1963FAEA1970F94588ADC011D
:10B16000CB01E4968CAC9DACAEACBFACE497881937
:10B170009909AA09BB09853C9940A105B10550F080
:10B180000F942D7D0F94588AE4966CAF7DAF8EAFEF
:10B190009FAFE497E9968FACE997882009F474C0D3
:10B1A0002AAD3EADA10163966FAD639764967FAD06
:10B1B000649766968FAD669768969FAD68970F9473
:10B1C0000DB187FFDFC00F94588ADC01CB01629676
:10B1D0008CAC9DACAEACBFAC629788199909AA093A
:10B1E000BB0989389341A105B10508F4CBC0D3014F
:10B1F000C2012A968CAC9DACAEACBFAC2A97881924
:10B200009909AA09BB092496AEACBFAC2497B595A1
:10B21000A79597958795AB2819F08093160F02C0D4
:10B220008093170F0F94588A6D966CAF7DAF8EAFD9
:10B230009FAF6D974B015C0162962CAD3DAD4EAD5D
:10B240005FAD6297821A930AA40AB50AAC968CAED7
:10B250009DAEAEAEBFAEAC9763968FAC6397A29631
:10B260008FAEA29764969FAC6497A3969FAEA39768
:10B270006696AFAC6697A496AFAEA4976896BFAC3F
:10B280006897A596BFAEA5972AAD3EADA10163967E
:10B290006FAD639764967FAD649766968FAD669742
:10B2A00068969FAD68970F94BFB8181614F00C9469
:10B2B00038700F94588ADC01CB016D968CAC9DAC34
:10B2C000AEACBFAC6D9788199909AA09BB0989383A
:10B2D0009341A105B10510F40C9438700F94588A6D
:10B2E00062966CAF7DAF8EAF9FAF6297DC01CB01F2
:10B2F00088199909AA09BB0920914B0D30914C0D71
:10B300001216130614F40C94636E2A968CAD9DAD40
:10B31000AEADBFAD2A97840D951DA61DB71D249611
:10B320008EAC9FAC2497B595A7959795879589285E
:10B3300011F40C9434708093160F80914B0D909102
:10B340004C0D019690934C0D80934B0D63969FACE2
:10B3500063976E969FAE6E976496AFAC64976F9648
:10B36000AFAE6F976696BFAC6697A096BFAEA0973C
:10B3700068968FAC6897A1968FAEA19721E0E99669
:10B380002FAFE99720E030E040EA51E463966FADDB
:10B39000639764967FAD649766968FAD669768965F
:10B3A0009FAD68970F9474B62AAD3EADA1010F947E
:10B3B0000DB187FF0EC0E8E8FCE084918F0188237F
:10B3C00009F4ECCD0F94FC0F0F5F1F4FF80184912F
:10B3D000F6CF0F94588ADC01CB01E0968CAC9DAC83
:10B3E000AEACBFACE09788199909AA09BB09813DA9
:10B3F0009740A105B10508F4B4C024968EAC9FAC6B
:10B400002497892881F0E090160FF12CE5E8FCE004
:10B4100084918F018823B9F00F94FC0F0F5F1F4FA9
:10B42000F8018491F7CFE090170FF12CE2E8FCE0EF
:10B4300084918F01882339F00F94FC0F0F5F1F4F09
:10B44000F8018491F7CF42E06AAD7EADC1010F945F
:10B450009F10EEE7FCE084918F01882339F00F9470
:10B46000FC0F0F5F1F4FF8018491F7CFB701FF0C5E
:10B47000880B990B0F9485108AE00F94FC0F2B9684
:10B480008FAC2B97882009F452C0A8969FACA89740
:10B49000891418F4282D2F5F59C02B968FAC2B9749
:10B4A000A8969FACA897891054C0282D2F5F2B9683
:10B4B0002FAF2B97E5962FADE597E6963FADE69734
:10B4C000E7964FADE797E8965FADE8976AAD7EAD3A
:10B4D000C1010F9473B66B017C0120E030E0A9013B
:10B4E0000F94BFB818165CF420E030E040EA50E456
:10B4F000C701B6010F940DB187FF2BC00AC020E031
:10B5000030E040EA50ECC701B6010F94BFB81816FE
:10B5100004F524966FAD2497661F6627661F80E0AA
:10B520000F94442381E08093ED0E0C94F7698AAC6C
:10B53000E5968FAEE5979EACE6969FAEE697E796CA
:10B540002FAEE797E8963FAEE89721E02B962FAF16
:10B550002B970F94588AE0966CAF7DAF8EAF9FAF5C
:10B56000E0970F94588A6B017C010F94588A6D966E
:10B570000CAD1DAD2EAD3FAD6D9762968CAC9DAC04
:10B58000AEACBFAC6297080D191D2A1D3B1DC01A39
:10B59000D10AE20AF30ADC01CB018C0D9D1DAE1D20
:10B5A000BF1D81389F44A241B10570F0E1E6FCE087
:10B5B00084918F01882309F4F1CC0F94FC0F0F5F65
:10B5C0001F4FF8018491F6CF80914B0D90914C0D57
:10B5D000A7968EAC9FACA797881699060CF055CD10
:10B5E000E5E0FCE084918F01882309F4D7CC0F9427
:10B5F000FC0F0F5F1F4FF8018491F6CF0F942D833E
:10B600000C94F76980916113882311F40C94F76905
:10B6100085E40F94959E882331F00F948C9E0F94AF
:10B62000D9B7162F01C01FEF86E40F94959E88238B
:10B6300031F00F948C9E0F94D9B7062F01C00FEFF5
:10B640001F920F931F921F9384EF9BE09F938F9302
:10B650000F9418B01F920F931F921F938CE299E5DD
:10B660009F938F930F949EA00FB6F894DEBF0FBEEA
:10B67000CDBF1AE00E94C988181614F40C94F7691B
:10B68000115011F00C943D700C94F7690F941F1336
:10B690000C94F7690F94AE110C94F7698091A61081
:10B6A0008F938091A5108F938091A4108F93809198
:10B6B000A3108F938091A2108F938091A1108F93EC
:10B6C0008091A0108F9380919F108F9380919E10F6
:10B6D0008F9380919D108F9380919C108F93809178
:10B6E0009B108F930AE210E61F930F931F930F9303
:10B6F00080919A108F93809199108F9380919810D8
:10B700008F93809197108F93809196108F93809153
:10B7100095108F93809194108F93809193108F93B5
:10B72000809192108F93809191108F9380919010BF
:10B730008F9380918F108F9380918E108F93809133
:10B740008D108F9380918C108F9380918B108F939D
:10B7500080918A108F93809189108F9380918810A7
:10B760008F93809187108F93809186108F93809113
:10B7700085108F93809184108F93809183108F9385
:10B78000809182108F93809181108F93809180108F
:10B790008F9380917F108F931F930F931F930F931D
:10B7A00080917E108F9380917D108F9380917C107B
:10B7B0008F9380917B108F9380917A108F938091DB
:10B7C00079108F93809178108F93809177108F9359
:10B7D0001F930F931F930F938091FE108F9380916F
:10B7E000FD108F938091FC108F938091FB108F93AD
:10B7F0008091FA108F938091F9108F938091F810B7
:10B800008F938091F7108F938091F6108F93809192
:10B81000F5108F938091F4108F938091F3108F9394
:10B820008091F2108F938091F1108F938091F0109E
:10B830008F938091EF108F931F930F931F930F930C
:10B84000809176108F93809175108F9380917410F2
:10B850008F93809173108F93809172108F9380914A
:10B8600071108F93809170108F9380916F108F93D0
:10B8700080916E108F9380916D108F9380916C10DA
:10B880008F9380916B108F9380916A108F9380912A
:10B8900069108F93809168108F93809167108F93B8
:10B8A0001F930F931F930F938091EE108F938091AE
:10B8B000ED108F938091EC108F938091EB108F930C
:10B8C0008091EA108F938091E9108F938091E81016
:10B8D0008F938091E7108F938091E6108F938091E2
:10B8E000E5108F938091E4108F938091E3108F93F4
:10B8F0008091E2108F938091E1108F938091E010FE
:10B900008F938091DF108F931F930F931F930F934B
:10B91000809166108F93809165108F938091641051
:10B920008F93809163108F93809162108F93809199
:10B9300061108F93809160108F9380915F108F932F
:10B9400080915E108F9380915D108F9380915C1039
:10B950008F9380915B108F9380915A108F93809179
:10B9600059108F93809158108F93809157108F9317
:10B970001F930F931F930F93809156108F93809175
:10B9800055108F93809154108F93809153108F9303
:10B99000809152108F93809151108F93809150100D
:10B9A0008F9380914F108F9380914E108F93809141
:10B9B0004D108F9380914C108F9380914B108F93EB
:10B9C00080914A108F93809149108F9380914810F5
:10B9D0008F93809147108F931F930F931F930F9313
:10B9E00084E499E09F938F930F9418B00FB6F89466
:10B9F000DEBF0FBECDBF2CEA35EC47E25EE36091BF
:10BA0000B3107091B4108091B5109091B6100F944E
:10BA10007AAA9F938F937F936F932CEA35EC47E23A
:10BA20005EE36091AF107091B0108091B110909171
:10BA3000B2100F9462B79F938F937F936F9380910F
:10BA4000AE108F938091AD108F938091AC108F9337
:10BA50008091AB108F931F930F931F930F9387E1E8
:10BA600099E09F938F930F9418B02CEA35EC47E23E
:10BA70005EE36091BF107091C0108091C1109091F1
:10BA8000C2100F947AAA9F938F937F936F932CEA9F
:10BA900035EC47E25EE36091BB107091BC10809181
:10BAA000BD109091BE100F9462B79F938F937F93B8
:10BAB0006F938091BA108F938091B9108F9380917A
:10BAC000B8108F938091B7108F931F930F931F938C
:10BAD0000F9382EE98E09F938F930F9418B00FB658
:10BAE000F894DEBF0FBECDBF8091C5101F928F931B
:10BAF0001F930F931F930F9320E030E040E752E431
:10BB00006091D6107091D7108091D8109091D91073
:10BB10000F947AAA9F938F937F936F938091D51000
:10BB20008F938091D4108F938091D3108F938091B5
:10BB3000D2108F931F930F931F930F938091D11067
:10BB40008F938091D0108F938091CF108F9380919D
:10BB5000CE108F9320E030E040E752E46091CA10AD
:10BB60007091CB108091CC109091CD100F947AAA47
:10BB70009F938F937F936F938091C9108F93809140
:10BB8000C8108F938091C7108F938091C6108F93A8
:10BB90001F930F931F930F9381EE97E09F938F93C3
:10BBA0000F9418B00FB6F894DEBF0FBECDBF8091D2
:10BBB000DA108823E9F08091DE108F938091DD10F8
:10BBC0008F938091DC108F938091DB108F931F9364
:10BBD0000F931F930F938BEB97E09F938F930F948B
:10BBE00018B00FB6F894DEBF0FBECDBF0C94F76946
:10BBF0001F930F938CE997E09F938F930F9418B046
:10BC00000F900F900F900F900C94F769882339F0E4
:10BC10000F94FC0F0F5F1F4FF8018491F7CFE9E4F9
:10BC2000FEE084918F01882311F40C94F7690F943E
:10BC3000FC0F0F5F1F4FF8018491F5CF8AE50F9439
:10BC4000959E882309F489C00F948C9E6B017C011A
:10BC500020E030E040E751EC0F94BFB887FD38C0DA
:10BC600020E030E040EA50ECC701B6010F940DB17E
:10BC7000181674F1F7FAF094F7F8F094C092A71040
:10BC8000D092A810E092A910F092AA10EAE2F0E691
:10BC900084918F01882339F00F94FC0F0F5F1F4FA1
:10BCA000F8018491F7CFE7EBF5E084918F018823C9
:10BCB00039F00F94FC0F0F5F1F4FF8018491F7CFFD
:10BCC0008AE00F94FC0F8AE00F94FC0F0C94F76944
:10BCD000EAE2F0E684918F01882339F00F94FC0F9B
:10BCE0000F5F1F4FF8018491F7CFE7EBF5E08491E8
:10BCF0008F01882339F00F94FC0F0F5F1F4FF8015D
:10BD00008491F7CFEBEDF5E084918F01882339F032
:10BD10000F94FC0F0F5F1F4FF8018491F7CF61EF75
:10BD20007FEF8FEF9FEF0F948510E3EDF5E08491A7
:10BD30008F01882339F00F94FC0F0F5F1F4FF8011C
:10BD40008491F7CF6BEF7FEF8FEF9FEF0F9485100C
:10BD50008AE00F94FC0F0C94F769EAE2F0E6849114
:10BD60008F01882339F00F94FC0F0F5F1F4FF801EC
:10BD70008491F7CFE7EBF5E084918F01882339F0C8
:10BD80000F94FC0F0F5F1F4FF8018491F7CF8AE0EB
:10BD90000F94FC0F8091A7109091A810A091A9106A
:10BDA000B091AA10BC01CD01905842E00F949F10B1
:10BDB0008AE00F94FC0F0C94F7690F942D8385E4AF
:10BDC0000F94959E882329F00F948C9E6B017C0123
:10BDD00005C0C12CD12CE12C80ECF82E8CE40F9402
:10BDE000959E81110F948C9E8AE50F94959E8823D1
:10BDF00029F00F948C9E2B013C011CC020E030E008
:10BE000048EC51E46091071070910810809109107E
:10BE100090910A100F940DB187FF07C0412C512C4F
:10BE200008ED602E01E4702E05C0412C512C612CD0
:10BE300010E4712E88E50F94959E882349F00F94A5
:10BE40008C9E22966CAF7DAF8EAF9FAF22970CC0B9
:10BE5000812C912CB3E5AB2EB3E4BB2E22968CAE95
:10BE60009DAEAEAEBFAE229789E50F94959E882316
:10BE700049F00F948C9E26966CAF7DAF8EAF9FAF2E
:10BE8000269706C026961CAE1DAE1EAE1FAE269788
:10BE900080916113882311F40C94437088E694E038
:10BEA0000F94370A882311F40C94437021E02AAFD1
:10BEB0000F942D8310924C138091FE0E882329F04D
:10BEC00060E086E190E00E94F8F6309159026396B6
:10BED0003FAF639740915A0264964FAF6497E091E9
:10BEE0000E0DF0E0EE0FFF1FE159FA4E80819181B7
:10BEF00067969FAF8EAF6797A091BE19B091BF199B
:10BF00006996BFAFAEAF69978090FF0F9090001019
:10BF1000A0900110B09002102A968CAE9DAEAEAEED
:10BF2000BFAE2A9789829A82AB82BC82209103108D
:10BF30003091041040910510509106102E962CAFB0
:10BF40003DAF4EAF5FAF2E972D833E834F83588713
:10BF50008091071090910810A0910910B0910A10DB
:10BF600062968CAF9DAFAEAFBFAF629789879A875D
:10BF7000AB87BC8720910B1030910C1040910D10B5
:10BF800050910E102D873E874F87588BC701B60101
:10BF90000F9474B660930B1070930C1080930D1077
:10BFA00090930E106EE0262E6DE0362E3F922F926B
:10BFB000812C912C78EEA72E72E4B72EEBE0CE2EDA
:10BFC000E0E1DE2E6296ECACFDAC0EAD1FAD6297EB
:10BFD0002E962CAD3DAD4EAD5FAD2E972A966CAD35
:10BFE0007DAD8EAD9FAD2A970F9476340F942D833F
:10BFF00020910710309108104091091050910A10BB
:10C00000C301B2010F9474B67B018C0160930710D9
:10C01000709308108093091090930A1020910310D8
:10C020003091041040910510509106106091FF0F5F
:10C030007091001080910110909102103F922F9208
:10C04000812C912CF0E7AF2EF1E4BF2E0F947634C3
:10C050000F942D8322968CAC9DACAEACBFAC2297D6
:10C060008092FF0F90920010A0920110B0920210E7
:10C0700026962CAD3DAD4EAD5FAD269720930310B7
:10C08000309304104093051050930610E090071071
:10C09000F09008100091091010910A103F922F9211
:10C0A000812C912CA8E4AA2EA2E4BA2E26962CADBF
:10C0B0003DAD4EAD5FAD269722966CAD7DAD8EAD9C
:10C0C0009FAD22970F9476340F942D830F900F908D
:10C0D0000F900F900F900F9080916113811124C0E9
:10C0E00084E090E090932702809326020F94588A70
:10C0F0004B015C018FEA90E10E94CDFBCC24C394FC
:10C10000D12CE12CF12CD1100C9487700E947AAACA
:10C11000882311F40C9487709FB7F89480910201E2
:10C120008B7F809302019FBF1092B60680916113AE
:10C13000882319F00F946B6302C00E94C4C10F944E
:10C140002D8380916113811117C084E090E090935A
:10C1500027028093260241E060E082EF91E10E9495
:10C16000DAFB8093B606811104C082EC91E10E9453
:10C170007CFC81E00E9407A880916113882309F468
:10C180007AC0AAADA11173C080913E0E882329F018
:10C1900060E08091470D0F94836284E090E090937B
:10C1A00027028093260288ED90E10E94CDFBFF24B8
:10C1B000F39400E010E00E947AAA811139C00F9434
:10C1C0004F7D81E00F948E83043FB1E01B0711F493
:10C1D00000E010E08091010184608093010101156D
:10C1E0001105A1F48091010790910207009721F0B9
:10C1F0000197B9F4FF20A9F09FB7F894809102014C
:10C200008460809302019FBFF12C0BC004311105A3
:10C2100041F49FB7F894809102018B7F80930201D3
:10C220009FBF0F5F1F4F84E090E00E94BFA4C3CF69
:10C230009FB7F894809102018B7F809302019FBF8A
:10C2400080913E0E882399F00E94FEA762E080E074
:10C250000E94C6A780E59BE40E94F1A680E6809339
:10C2600053131092521360E080E00F9430608AAD57
:10C270000F94E8A16FC00E94FEA761E080E00E94D9
:10C28000C6A781E391E10E94F1A662E080E00E94EE
:10C29000C6A78EE191E10E94F1A684E090E0909320
:10C2A0002702809326020E942CAE0E947AAA811156
:10C2B0001AC00F944F7D81E00F948E830E9478AE58
:10C2C000882399F38091010790910207029720F447
:10C2D00088EE93E00F948D4C82E390E00E94BFA41F
:10C2E00084E50F9411290E94CEAC82E090E09093F7
:10C2F00027028093260286E40E948FAC0F94329D21
:10C300008091010790910207029720F484EF91E059
:10C310000F948D4C82E390E00E94BFA484E50F94BB
:10C3200011290E941DAC0E94BEAA811110C041E0DB
:10C3300060E081E491E10E94DAFB182F81E00E9425
:10C3400007A882E00E9483A611110E94F3AC80E04E
:10C350000E9407A8EAADE1114AC11092B606F4E0C6
:10C360002F2E312CA2E04A2E512CBEE06B2EBDE0C8
:10C370007B2E8091B606813009F439C11092B60641
:10C3800030922702209226020E94FEA760E080E001
:10C390000E94C6A781E991E10E94F1A661E081E0D7
:10C3A0000E94C6A78AEF95E40E94F1A662E081E0B0
:10C3B0000E94C6A78DE791E10E94F1A663E081E0AB
:10C3C0000E94C6A78BE691E10E94F1A661E080E0A1
:10C3D0000E94C6A78DE694E00E9463AAE090C0196F
:10C3E0000E2C000CFF0801E010E08091B6068111D0
:10C3F00068C00F944F7D81E00F948E838091C019A7
:10C40000082E000C990B9701281B390B37FF03C02E
:10C41000319521953109253031050CF444C08E1534
:10C420009F0514F401501109E816F90634F40F5F62
:10C430001F4F0430110564F009C00430110534F4B5
:10C440000115110529F401E010E002C003E010E03D
:10C4500061E080E00E94C6A781E496E00E9463AAA2
:10C4600062E080E00E94C6A781E496E00E9463AA91
:10C4700063E080E00E94C6A781E496E00E9463AA80
:10C48000602F80E00E94C6A78DE694E00E9463AA18
:10C49000E090C0190E2C000CFF0864E670E080E00C
:10C4A00090E00F9440890E947AAA882309F49DCFD6
:10C4B0000093B60664EF71E080E090E00F9440894D
:10C4C00094CF0E94FEA70F94608B50922702409257
:10C4D00026028091B606823009F454C0833009F0F8
:10C4E0007BC020E030E048E452E460910B10709192
:10C4F0000C1080910D1090910E100F9474B66093F3
:10C500000B1070930C1080930D1090930E10E09010
:10C510000710F09008100091091010910A10209156
:10C520000310309104104091051050910610609155
:10C53000FF0F7091001080910110909102107F9276
:10C540006F92812C912CA12CB0E4BB2EEBE0CE2E6F
:10C55000E0E1DE2E0F9476340E94FEA760E080E0DA
:10C560000E94C6A784EA91E10E94F1A662E080E001
:10C570000E94C6A780E59BE40E94F1A60F900F9051
:10C5800010E01EC080916113882321F080E00F9499
:10C59000E8A1EFCE0F94329DECCE0F944F7D81E059
:10C5A0000F948E8365E570E080E090E00F94408901
:10C5B000F1E0EF1AF10889F71F5F143109F4D9CEC1
:10C5C00063E0812F0E94C6A78CE195E00E9463AAD8
:10C5D000AAE0EA2EF12CE1CF0E94FEA762E080E003
:10C5E0000E94C6A782EB91E10E94F1A6C2CE81E033
:10C5F0000E9407A869968EAC9FAC69979092BF196C
:10C600008092BE199AAC91103FC020E030E040EA21
:10C6100050E460910B1070910C1080910D1090916E
:10C620000E100F9474B660930B1070930C108093DF
:10C630000D1090930E10E0900710F09008100091EC
:10C64000091010910A1020910310309104104091AC
:10C650000510509106106091FF0F709100108091AD
:10C66000011090910210EEE0FDE0FF93EF93812C1A
:10C67000912CA12CE0E4BE2EFBE0CF2EF0E1DF2ECA
:10C680000F9476340F900F90E0900710F090081000
:10C690000091091010910A102D813E814F8158851B
:10C6A00069817A818B819C81EEE06E2EEDE07E2E99
:10C6B0007F926F92812C912CF8E4AF2EF2E4BF2E82
:10C6C000ABE0CA2EA0E1DA2E0F9476340F942D83BE
:10C6D000E984FA840B851C852D813E814F81588524
:10C6E00069817A818B819C817F926F92812C912CC0
:10C6F000B0E7AB2EB1E4BB2E0F9476340F942D83AC
:10C70000CE010D960E94ADE080E1FE013196AFEFC3
:10C71000BFE001900D928A95E1F780E1EFEFFFE035
:10C72000ACEFBCE001900D928A95E1F76396AFAC57
:10C730006397A09259026496BFAC6497B0925A0274
:10C74000BF92AF9283E997E09F938F938E01015E32
:10C750001F4F1F930F930F9471B060E0C8010F94A7
:10C760009B5881EF94E10F94AD2D1092400E1092E2
:10C770003F0E0FB6F894DEBF0FBECDBF38C60F9484
:10C78000218C35C683E50F94959E882309F42FC626
:10C790000F948C9E0F94D3B76B017C012B0180E525
:10C7A0009BE40F94AD2DE6E2FEE084918F01882397
:10C7B00039F00F94FC0F0F5F1F4FF8018491F7CFF2
:10C7C0000D2C000CEE08FF08C701B6010F94851070
:10C7D0008AE00F94FC0F0F94588A4B015C01109271
:10C7E000590E6091120D7091130D072E000C880BDD
:10C7F000990B0F9413B120E030E0A9010F940DB113
:10C80000811111C060916F1570917015072E000C89
:10C81000880B990B0F9413B111E020E030E0A901CF
:10C820000F940DB1811110E0052C000C66087708FB
:10C8300081E2282E8EE0382E111115C08091590EFC
:10C8400081116CC0C301B2010F9413B12091660D28
:10C850003091670D4091680D5091690D0F94BFB8EC
:10C8600018168CF05BC0C301B2010F9413B1209174
:10C87000660D3091670D4091680D5091690D0F94D0
:10C880000DB187FF4BC00F94588ADC01CB0188198A
:10C890009909AA09BB09893E9340A105B10508F48D
:10C8A00034C0E3E2FEE084915F01882341F00F94FD
:10C8B000FC0FFFEFAF1ABF0AF5018491F6CF60912C
:10C8C000660D7091670D8091680D9091690D41E042
:10C8D0000F949F10F101849101E2A02E0EE0B02E82
:10C8E000882341F00F94FC0FFFEFAF1ABF0AF50148
:10C8F0008491F6CFC701B6010F9485108AE00F949A
:10C90000FC0F0F94588A4B015C010F944F7D80E01F
:10C910000F948E8380E00E9483A68ECF8FE897E1EC
:10C920000F94AD2D64C58FE30F94959E882309F471
:10C93000BCC00F941E0C1A821982882381F00FE666
:10C9400014E0D8018D918D01882319F00F94FC0F0C
:10C95000F8CF8AE00F94FC0F03E814E00AC00AE95C
:10C9600014E0F80181918F01882399F30F94FC0F53
:10C97000F8CFD8018D918D01882319F00F94FC0F09
:10C98000F8CF8AE00F94FC0F44244A94542C3201CF
:10C99000A3E28A2E912CA12CB12CB0EB2B2EBFE060
:10C9A0003B2E1AAE69817A81072E000C880B990BF9
:10C9B0000F9413B120914F103091501040915110AD
:10C9C000509152100F9462B76B017C012AAD211176
:10C9D0000DC0EDE1FEE084918F01882359F00F94A2
:10C9E000FC0F0F5F1F4FF8018491F7CFC301B20115
:10C9F0000F948510EAE1FEE084918F01882339F0DD
:10CA00000F94FC0F0F5F1F4FF8018491F7CFC50102
:10CA1000B4010F948510E7E1FEE084918F01882333
:10CA200039F00F94FC0F0F5F1F4FF8018491F7CF7F
:10CA300069817A81072E000C880B990B0F94851061
:10CA4000E4E1FEE084918F01882339F00F94FC0F1C
:10CA50000F5F1F4FF8018491F7CF20E030E04AE7E5
:10CA600054E4C701B6010F947AAA42E00F949F10D4
:10CA70008AE00F94FC0FFAADFF5FFAAFF63009F4CD
:10CA8000B6C4BE016F5F7F4FC1010E9438D2B2E0D1
:10CA90002B0E311CE5E08E0E911CA11CB11CFFEF8A
:10CAA0004F1A5F0A6F0A7F0A7DCF81E20F94959E2D
:10CAB000882309F44AC061E086EA9FE00F9418B623
:10CAC00088E090E09A838983BE016F5F7F4F80EB9F
:10CAD0009FE00E9452D288E190E09A838983BE0150
:10CAE0006F5F7F4F82EB9FE00E9452D280E390E025
:10CAF0009A838983BE016F5F7F4F84EB9FE00E9422
:10CB000052D280E590E09A838983BE016F5F7F4FA8
:10CB100086EB9FE00E9452D288E790E09A83898357
:10CB2000BE016F5F7F4F88EB9FE00E9452D20EEAFA
:10CB300014E0D8018D918D01882319F00F94FC0F1A
:10CB4000F8CF8AE00F94FC0F52C48AE50F94959EAB
:10CB5000882319F161E086EA9FE00F9418B61A82E3
:10CB6000198200EB1FE0BE016F5F7F4FC8010E947A
:10CB700052D20E5F1F4F0A3BBFE01B07A1F70FEB1E
:10CB800014E0F80181918F01882319F00F94FC0FB4
:10CB9000F8CF8AE00F94FC0F2AC483E50F94959E8A
:10CBA000882309F4CEC00F948C9E0F94D3B77A8358
:10CBB000698389E40F94959E882309F418C40F941F
:10CBC0008C9E0F94D9B7653008F011C4862F90E081
:10CBD0008852984FBE016F5F7F4F880F991F0E9448
:10CBE00052D209EC14E0D8018D918D01882319F0FF
:10CBF0000F94FC0FF8CF8AE00F94FC0F03E814E0C9
:10CC0000F80181918F01882319F00F94FC0FF8CF60
:10CC10008AE00F94FC0F5EEA252E5FE0352E442457
:10CC20004A94542C320173E2872E912CA12CB12C02
:10CC30001AAE1A821982FAADFF2331F0BE016F5F7E
:10CC40007F4FC1010E9438D269817A81072E000C82
:10CC5000880B990B0F9413B120914F103091501005
:10CC600040915110509152100F9462B76B017C01AA
:10CC70002AAD21110DC0E0E1FEE084918F018823EF
:10CC800059F00F94FC0F0F5F1F4FF8018491F7CFFD
:10CC9000C301B2010F948510EDE0FEE084918F0195
:10CCA000882339F00F94FC0F0F5F1F4FF801849118
:10CCB000F7CFC501B4010F948510EAE0FEE084913E
:10CCC0008F01882339F00F94FC0F0F5F1F4FF8017D
:10CCD0008491F7CF69817A81072E000C880B990B1C
:10CCE0000F948510E7E0FEE084918F01882339F0EE
:10CCF0000F94FC0F0F5F1F4FF8018491F7CF20E0D6
:10CD000030E04AE754E4C701B6010F947AAA42E042
:10CD10000F949F108AE00F94FC0FFAADFF5FFAAFFB
:10CD200025E0820E911CA11CB11C3FEF431A530A4F
:10CD3000630A730A42E0240E311CF63009F079CF01
:10CD400056C3E6EFFDE084918F01882309F44FC3B9
:10CD50000F94FC0F0F5F1F4FF8018491F6CF0F94D3
:10CD60002D838BE40F94959E882399F00F94569E03
:10CD70006B017C0120E030E0A9010F94BFB887FD72
:10CD800008C0C092C90FD092CA0FE092CB0FF092A8
:10CD9000CC0F82E50F94959E882361F00F94569EE8
:10CDA0006B017C0120E030E0A9010F940DB187FFF9
:10CDB00089C006C0C12CD12C40E8E42E4FEBF42EE4
:10CDC00084E40F94959E882329F00F94569E4B017E
:10CDD0005C0106C0812C912C30E8A32E3FEBB32ED2
:10CDE00087E50F94959E882329F00F94569E2B017A
:10CDF0003C0106C0412C512C20E8622E2FEB722EF4
:10CE000088E40F94959E882339F00F94569E6AAF5C
:10CE10007BAF8CAF9DAF08C020E030E040E85FEB17
:10CE20002AAF3BAF4CAF5DAF20E030E0A901C501B8
:10CE3000B4010F94BFB887FD45C020E030E0A901E0
:10CE4000C301B2010F94BFB887FD3CC020E030E0C1
:10CE5000A9016AAD7BAD8CAD9DAD0F94BFB887FDC8
:10CE600031C020E030E0A901C501B4010F940DB13B
:10CE7000882391F120E030E040E05FE3C501B40198
:10CE80000F947AAA6B017C012AAD3BAD4CAD5DAD30
:10CE9000C301B2010F947AAA4B015C01A70196016C
:10CEA000C701B6010F947AAA2BED3FE049E450E4A4
:10CEB0000F947AAA9B01AC01C501B4010F9462B72B
:10CEC0006B017C0120E030E0A901C701B6010F949D
:10CED000BFB887FF04C00BC0C12CD12C7601C09213
:10CEE000C50FD092C60FE092C70FF092C80FEAE2CA
:10CEF000F0E684918F01882339F00F94FC0F0F5FC7
:10CF00001F4FF8018491F7CFE8E8F7E084918F0193
:10CF1000882339F00F94FC0F0F5F1F4FF8018491A5
:10CF2000F7CF6091C90F7091CA0F8091CB0F90918C
:10CF3000CC0F42E00F949F108AE00F94FC0FE2E8C0
:10CF4000F7E084918F01882339F00F94FC0F0F5F75
:10CF50001F4FF8018491F7CFC090C50FD090C60F36
:10CF6000E090C70FF090C80F20E030E0A901C701A2
:10CF7000B6010F940DB1882349F042E0C701B60114
:10CF80000F949F108AE00F94FC0F31C2EDE7F7E099
:10CF900084918F01882311F40C9499460F94FC0F0F
:10CFA0000F5F1F4FF8018491F5CF0F940E1E1FC223
:10CFB00088E50F94959E882339F00F948C9E0F94EA
:10CFC000D9B780E00F94029D89E50F94959E882340
:10CFD00039F00F948C9E0F94D9B781E00F94029D85
:10CFE0008AE50F94959E882339F00F948C9E0F94B8
:10CFF000D9B782E00F94029D85E40F94959E882313
:10D0000009F4F5C10F948C9E0F94D9B783E00F9467
:10D01000029DEDC188E50F94959E882339F00F9409
:10D020008C9E0F94D9B780E00F94F19C89E50F9402
:10D03000959E882339F00F948C9E0F94D9B781E088
:10D040000F94F19C8AE50F94959E882339F00F94F4
:10D050008C9E0F94D9B782E00F94F19C85E40F94D5
:10D06000959E882309F4C3C10F948C9E0F94D9B761
:10D0700083E00F94F19CBBC181E0809318070E946C
:10D0800091E00F940E1EB3C188E50F94959E8823FE
:10D0900031F00F948C9E0F94D9B76093660289E5A6
:10D0A0000F94959E882331F00F948C9E0F94D9B7DE
:10D0B000609367028AE50F94959E882331F00F9460
:10D0C0008C9E0F94D9B76093680285E40F94959E67
:10D0D000882331F00F948C9E0F94D9B76093690226
:10D0E00016E6C12E12E0D12E0CE313E080E4A82E48
:10D0F00083E0B82E90EAE92E95E0F92ED6019D91B5
:10D100006D01F80181918F011F929F93282F082EA6
:10D11000000C330B3F938F93FF92EF920F9418B054
:10D120000F900F900F900F900F900F90A016B106D8
:10D1300029F75DC188E50F94959E882339F00F94F7
:10D140008C9E0F94D9B780E00F94D09C89E50F9402
:10D15000959E882339F00F948C9E0F94D9B781E067
:10D160000F94D09C8AE50F94959E882331F00F94FC
:10D170008C9E0F94D9B76093380285E40F94959EE6
:10D18000882309F434C10F948C9E0F94D9B760930F
:10D1900039022DC188E50F94959E882339F00F94AC
:10D1A0008C9E0F94D9B780E00F94AE9C89E50F94C4
:10D1B000959E882339F00F948C9E0F94D9B781E007
:10D1C0000F94AE9C8AE50F94959E882331F00F94BE
:10D1D0008C9E0F94D9B760933C0285E40F94959E82
:10D1E000882309F404C10F948C9E0F94D9B76093DF
:10D1F0003D02FDC085E40F94959E882309F4F7C095
:10D200000F948C9E0F94D9B76B017C018B01683011
:10D21000710569F06031710551F06032710539F0C6
:10D220006034710521F06038710509F0E0C00F9499
:10D230002D8380E091E05C010090130702C0B6945A
:10D24000A7940A94E2F7C6010E9446BA8093130796
:10D2500020911C0240912002682F83E00E9469BA4D
:10D2600040903F10509040106090411070904210DC
:10D27000A016B10670F5C801B5010F941EBB6B0175
:10D28000E12CF12CC701B6010F9411B19B01AC0147
:10D2900060915310709154108091551090915610D8
:10D2A0000F947AAA60935310709354108093551082
:10D2B00090935610A3019201C701B6010F9429B6AD
:10D2C00060933F10709340108093411090934210F0
:10D2D0008EC0C501B8010F941EBB6B01E12CF12C6F
:10D2E000C701B6010F9411B19B01AC0160915310BD
:10D2F0007091541080915510909156100F9462B710
:10D30000609353107093541080935510909356105F
:10D31000C301B201A70196010F9445BB20933F10B2
:10D3200030934010409341105093421060C0809160
:10D330006113882329F085E40F94959E811190C78D
:10D340000F945E6454C0809161138823D9F185E500
:10D350000F94959E882359F120E030E04FE253E48A
:10D360006091830F7091840F8091850F9091860F4B
:10D370000F94BFB81816C4F400E010E08091511368
:10D38000082E000C990B002E02C0959587950A94E3
:10D39000E2F780FD0F946B630F5F1F4F04301105A0
:10D3A00069F71092511323C00F94096020C083E4E1
:10D3B0000F94959E882319F00F946B6318C00F94F7
:10D3C0003B6415C00E94C4C112C080916D1590913C
:10D3D0006E158D579C4E9F938F9381EE9DE09F938A
:10D3E0008F930F9418B00F900F900F900F90109292
:10D3F000150D1092140D63C284E50F94959E882339
:10D4000009F4EEC00F942D83209140133091411305
:10D41000F90131968F01021B130B81918032D1F3F8
:10D420008930C1F390ED980F953020F18F3371F072
:10D43000E1EDFDE084918F01882309F4CDC00F94C4
:10D44000FC0F0F5F1F4FF8018491F6CF809161139D
:10D4500040E050E0882329F06FEC7BE28AEA92E119
:10D4600004C060E972E189E992E10E94D2C280932E
:10D47000460D06C00F948C9E0F94D9B76093460D4D
:10D480008091460D21E030E0082E01C0220F0A9461
:10D49000EAF790915113292B209351139091611326
:10D4A000992361F1805F809353131092521361E0CE
:10D4B00081E00F94306064E670E080E090E00F94CB
:10D4C000408980E380935313109252138091460D4C
:10D4D0008093470D8091401390914113FC01E00F20
:10D4E000F11F80818F3309F0EAC164E670E080E0CB
:10D4F00090E00F9440890F94C4A0E1C1882309F4FF
:10D5000032C0EAE2F0E684918F01882339F00F946B
:10D51000FC0F0F5F1F4FF8018491F7CFEFECFDE098
:10D5200084918F01882339F00F94FC0F0F5F1F4FF8
:10D53000F8018491F7CF6091460D70E080E090E0B3
:10D540000F9485108AE00F94FC0FEFE8F5E08491CA
:10D550008F01882309F440C00F94FC0F0F5F1F4F09
:10D56000F8018491F6CF86E40F94959E882399F074
:10D570000F948C9E6B017C0120E030E0A9010F9498
:10D58000BFB8181644F4C0922102D0922202E09251
:10D590002302F0922402EAE2F0E684918F018823CC
:10D5A00039F00F94FC0F0F5F1F4FF8018491F7CFF4
:10D5B000EDE7F5E084918F01882339F00F94FC0F9B
:10D5C0000F5F1F4FF8018491F7CF60910E0D70E04F
:10D5D00080E090E00F9485108AE00F94FC0F6FC1FB
:10D5E00084E40F94959E882309F408C10F948C9EBF
:10D5F0000F94D3B76330710509F061C186E395E0FC
:10D600009F938F930F9418B081E40F94959E0F9081
:10D610000F908823B9F08091401390914113DC0161
:10D6200011962C91283741F440E150E060E070E021
:10D6300002960F94A2AC04C00F948C9E0F94D3B7A3
:10D640008B0102C000E010E083E40F94959E8823D4
:10D6500039F00F948C9E0F94D3B7262F872F02C0DA
:10D6600020E080E11F71A22EB82EB1E0AB16B0E130
:10D67000BB0618F0A12CB0E1BB2EC501800F911F95
:10D680008130904128F080E090E15C01A01AB10A5D
:10D6900088E50F94959E882309F475C02091401366
:10D6A00030914113A9014F5F5F4F9E012F5F3F4FA4
:10D6B0006901F901E12CF12C9A01D9018C912F5FBC
:10D6C0003F4F8823A1F140E1E416F10469F1803273
:10D6D000A1F38A3061F190ED980F9A3018F4829599
:10D6E000807F07C09FE9980F9630A8F48295807FCD
:10D6F0008057AD014E5F5F4F11969C9120ED290F31
:10D700002A3010F4822B0BC02FE9290F263018F491
:10D710009755892B04C0F194E194F10808C08193D6
:10D720006FEFE61AF60AC8CFA0E1EA2EF12C5701F6
:10D73000E114F10441F1812C912CD6016D916D0120
:10D74000C801880D991D0F9418B6BFEF8B1A9B0A5C
:10D75000E814F90491F71F930F93FF92EF9289E079
:10D7600095E09F938F930F9418B06091CE197091AC
:10D77000CF198AE090E00F9493AF0F900F900F9025
:10D780000F900F900F906801E12CF12CA114B104BF
:10D7900009F495C08D2D0F94AA9E8C2D0F94AA9EEE
:10D7A0006091CE197091CF1980E290E00F9493AF01
:10D7B00010E1EFEFCE1ADE0AEE0AFE0AC60101976B
:10D7C0000F94E8B5082F6091CE197091CF1980E2BF
:10D7D00090E00F9493AF802F0F94AA9E1150F1E028
:10D7E000AF1AB10811F01111E4CF6091CE19709108
:10D7F000CF198AE090E00F9493AFC8CFEAE2F0E649
:10D8000084918F01882339F00F94FC0F0F5F1F4F15
:10D81000F8018491F7CFE0ECF5E084918F01882343
:10D8200039F00F94FC0F0F5F1F4FF8018491F7CF71
:10D8300000916D1510916E150D571C4ED8018D91EC
:10D840008D01882319F00F94FC0FF8CFEAECFDE06E
:10D8500084918F01882309F4BFCE0F94FC0F0F5FD2
:10D860001F4FF8018491F6CFC090080DD090090D9C
:10D87000E0900A0DF0900B0D20910B1030910C10E0
:10D8800040910D1050910E10C701B6010F9473B660
:10D890004B015C012DEC3CEC4CEC5DEB0F940DB1BD
:10D8A00087FD3AC02DEC3CEC4CEC5DE3C501B401C6
:10D8B0000F94BFB818160CF438C00F9400A781E07D
:10D8C00090E090932702809326020F94588A6093E9
:10D8D0007619709377198093781990937919E0915C
:10D8E0006D15F0916E15E058FC4E8081813019F075
:10D8F000863009F0D7C4EFE8F7E184918F018823DF
:10D9000039F00F94FC0F0F5F1F4FF8018491F7CF90
:10D910008AE00F94FC0FC6C4E0910E0DF0E0E150D8
:10D92000F14F80818111A3C409C0E0910E0DF0E098
:10D93000E150F14F8081882309F4BFCFC0920B10D2
:10D94000D0920C10E0920D10F0920E108BE090E14E
:10D950000E94ADE0E0910E0DF0E0E150F14F9081BA
:10D9600081E089270F94B39E9DC420E030E040E819
:10D970005FE360910B1070910C1080910D109091ED
:10D980000E100F9474B660930B1070930C1080936C
:10D990000D1090930E10E0900710F0900810009179
:10D9A000091010910A102091031030910410409139
:10D9B0000510509106106091FF0F7091001080913A
:10D9C000011090910210EEE0FDE0FF93EF93812CA7
:10D9D000912CE8ECAE2EE3E4BE2EFBE0CF2EF0E17E
:10D9E000DF2E0F9476340F900F900C94674182E0F5
:10D9F00090E090932702809326021092460E109298
:10DA0000450E0C9444460F94819EAB01BC0140939B
:10DA100041195093421960934319709344198CE84B
:10DA200098E10E9464E9E3CC0F948C9E0F94D3B7E5
:10DA30008B010C94C1490F942D8388E50F94959E1A
:10DA4000882319F0179A10920F0D89E50F94959E6F
:10DA5000882319F0169A1092100D8AE50F94959E5E
:10DA600085E40F94959E882311F40C94354E149AF6
:10DA70000C94354E1A8219824AE050E0BE016F5F65
:10DA80007F4FC7010F94A2AC78A36F8F89819A81D1
:10DA90008816990609F0ABCC4AE050E0BE016F5FF2
:10DAA0007F4FC6010F94A2AC7AA369A389819A81A2
:10DAB0006816790609F09BCC4AE050E0BE016F5F22
:10DAC0007F4FC5010F94A2AC7CA36BA389819A817F
:10DAD0000817190709F08BCC8FE790E09EA38DA360
:10DAE0005801EFEFAE1ABE0AD8018C918D3211F5B4
:10DAF00075016701BFEFCB1ADB0AF70180810F9434
:10DB0000832D382E811102C07601F3CFEA18FB086D
:10DB1000DE2CC70199278330910569F543E050E079
:10DB200068E479E5C5010F94EBAE892B09F042C09A
:10DB30001EA21DA2332009F45ACCCE0101960F94E7
:10DB40008652882309F453CCFE017F96DE0111969C
:10DB5000AE01495D5F4F219131918D919D91821769
:10DB6000930708F44CC02817390708F440CC4E1727
:10DB70005F0789F73CCC8530910571F445E050E0B2
:10DB800062E479E5C5010F94EBAE892B99F481E04D
:10DB900090E09EA38DA3CECF049761F444E050E0C3
:10DBA0006DE379E5C5010F94EBAE892B19F482E0A2
:10DBB00090E0EFCF8EEF8E0D823008F018CCD801B8
:10DBC00011968C9111978F7D823509F010CC1296A9
:10DBD0008C918F7D833409F00ACCB2E0DB1203C054
:10DBE00083E090E0D6CFF801838190ED980F9A30D2
:10DBF00008F0FDCB082E000C990B8E97CACF82E25D
:10DC000092E10E94CDFB44E15DE062E080E00E9491
:10DC1000F3A7D2011D912D01812F0F94832D811126
:10DC200008C067EC76E0812F110F990B0F9493AF2A
:10DC3000F0CF42E152E163E080E00E94F3A78091DF
:10DC4000010790910207029720F488EE93E00F9469
:10DC50008D4C82E390E00E94BFA484E50F941129CB
:10DC600084EF91E00E94BFA4809101079091020788
:10DC7000029720F488EE93E00F948D4C82E390E0BD
:10DC80000E94BFA484E50F94112984E090E0909352
:10DC90002702809326020F944F7D81E00F948E839C
:10DCA0000E947AAA8823B9F382E090E09093270239
:10DCB0008093260281E00E9407A80E94FEA780E0D0
:10DCC0000E9483A694CBAC96CCACDDACEEACFFACA2
:10DCD000AC97C80ED91EEA1EFB1EAC962CAD3DAD0E
:10DCE0004EAD5FADAC97281B390B4A0B5B0B2A96E8
:10DCF0006CAD7DAD8EAD9FAD2A970F9429B6A7016F
:10DD000096010F9445BBDA01C901840D951DA61D2E
:10DD1000B71D84319105A105B105E4F02C013D0149
:10DD20008C3E9105A105B1052CF06BEE462E512CD1
:10DD3000612C712C40E84416510461047104DCF03C
:10DD40005EEF852E912CA12CB12C84189508A60885
:10DD5000B7080AC034E1432E512C612C712C44E1E8
:10DD6000842E912CA12CB12C2A968CAE9DAEAEAEF9
:10DD7000BFAE2A9706C02A964CAE5DAE6EAE7FAEA1
:10DD80002A97E1EFFCE084918F01882339F00F940A
:10DD9000FC0F0F5F1F4FF8018491F7CFC301B20151
:10DDA0000F948510ECEEFCE084918F01882339F00C
:10DDB0000F94FC0F0F5F1F4FF8018491F7CF2A9645
:10DDC0006CAD7DAD8EAD9FAD2A970F948510E5EEBD
:10DDD000FCE084918F01882339F00F94FC0F0F5FD2
:10DDE0001F4FF8018491F7CF42E06E966FAD6E97AA
:10DDF0006F967FAD6F97A0968FADA097A1969FADC0
:10DE0000A1970F949F10EEEDFCE084918F01882381
:10DE100039F00F94FC0F0F5F1F4FF8018491F7CF7B
:10DE200042E0A2966FADA297A3967FADA397A4966A
:10DE30008FADA497A5969FADA5970F949F108AE0EC
:10DE40000F94FC0F80914B0D90914C0D039714F49F
:10DE50000C9485592A966CAD7DAD8EAD9FAD2A97F9
:10DE60000F9413B120E030E040E850E40F947AAA18
:10DE70004B015C016E962FAD6E976F963FAD6F971D
:10DE8000A0964FADA097A1965FADA197A2966FAD5A
:10DE9000A297A3967FADA397A4968FADA497A596BE
:10DEA0009FADA5970F9473B620ED3FE049E450E491
:10DEB0000F947AAA20E030E040E05FE30F947AAA62
:10DEC0009B01AC01C501B4010F9462B74B015C0129
:10DED000C701B6010F9413B120E030E04AE754E4E3
:10DEE0000F9462B76B017C01E8EDFCE084918F0137
:10DEF000882339F00F94FC0F0F5F1F4FF8018491B6
:10DF0000F7CF42E0C501B4010F949F10E2EDFCE0B1
:10DF100084918F01882339F00F94FC0F0F5F1F4FFE
:10DF2000F8018491F7CF42E0C701B6010F949F102A
:10DF30008AE00F94FC0F2AE939E949E15FE3C50162
:10DF4000B4010F947AAA4B015C016093E90E7093BF
:10DF5000EA0E8093EB0E9093EC0E9B01AC010F94B4
:10DF600074B6A70196010F9462B76093E50E7093A3
:10DF7000E60E8093E70E9093E80EA5019401C70189
:10DF8000B6010F947AAA20E030E040E05EE30F94FF
:10DF90007AAA6093E10E7093E20E8093E30E909361
:10DFA000E40EE4ECFCE084918F01882339F00F94B7
:10DFB000FC0F0F5F1F4FF8018491F7CF8AE00F9499
:10DFC000FC0FEEEBFCE084918F01882339F00F9475
:10DFD000FC0F0F5F1F4FF8018491F7CF6091E90E9E
:10DFE0007091EA0E8091EB0E9091EC0E42E00F944E
:10DFF0009F108AE00F94FC0FE8EBFCE084918F0106
:10E00000882339F00F94FC0F0F5F1F4FF8018491A4
:10E01000F7CF6091E50E7091E60E8091E70E90913A
:10E02000E80E42E00F949F108AE00F94FC0FE2EBA1
:10E03000FCE084918F01882339F00F94FC0F0F5F6F
:10E040001F4FF8018491F7CF6091E10E7091E20EBD
:10E050008091E30E9091E40E42E00F949F108AE0CD
:10E060000F94FC0F0C9485598093170F0C949D59B5
:10E07000E9961FAEE9970C94C25984E690E00E949D
:10E08000BFA40C943A5B1AAE0C94585FE12CF12CAF
:10E0900080910101846080930101E114F10409F091
:10E0A0004EC080910107909102070097F1F101970E
:10E0B000D1F14FEFE41AF40A51E0D51609F452C039
:10E0C000D51608F04AC084E090E00E94BFA40F94E7
:10E0D000588A950184010054184D264F3F4F06176A
:10E0E00017072807390710F00C94836084E890E143
:10E0F0000E94CDFB1F8E18A219A21AA2CE014F9624
:10E100000F943F760F942D83149ADD24D3940F94AB
:10E110004F7D81E00F948E83F4EFEF16F1E0FF0660
:10E1200009F0B6CFB3CFCC2021F29FB7F8948091FD
:10E1300002018460809302019FBFC12CBACF34E1F9
:10E14000E316F10409F0B5CF9FB7F894809102016E
:10E150008B7F809302019FBFACCF62E0D616E1F0C7
:10E160000C94836084E090E00E94BFA40E947AAA8D
:10E17000882369F2E0910E0DF0E0EE0FFF1FE159E8
:10E18000FA4E67968EAD9FAD6797918380830E940C
:10E19000E7D142E0D42EBBCF00910E0D10E0F80184
:10E1A000EE0FFF1FE159FA4E60817181072E000CBE
:10E1B000880B990B0F9413B1000F111F000F111F43
:10E1C000F801ED57F04F20813181428153810F9446
:10E1D00073B62B013C0120E030E0A9010F94BFB8D9
:10E1E00018165CF420E030E040E85FE3C301B201C0
:10E1F0000F940DB187FF16C00AC020E030E040E860
:10E200005FEBC301B2010F94BFB818165CF48FEA3C
:10E2100090E10E94CDFB0F94588A4B015C01D12CF8
:10E220000C94866064E081E00E94C6A7E0910E0D28
:10E2300094E0E99FF0011124ED57F04F8081918126
:10E24000A281B3818F8F98A3A9A3BAA3CE014F96C1
:10E250000E940BB10E9463AA14E1E12EF12C57CF6A
:10E260000F948C9E0F94D9B76093460D69C82DEC1E
:10E270003CEC4CEC5DE3C501B4010F94BFB818163B
:10E280000CF45CCB1ACBA5019401F101662D772D1E
:10E290008F2F922D0F940DB1181614F40C94163B79
:10E2A0000C94263BC858DF4F0FB6F894DEBF0FBE64
:10E2B000CDBFDF91CF911F910F91FF90EF90DF9035
:10E2C000CF90BF90AF909F908F907F906F905F9016
:10E2D0004F903F902F9008952F923F924F925F92D0
:10E2E0006F927F928F929F92AF92BF92CF92DF9266
:10E2F000EF92FF920F931F93CF93DF93CDB7DEB7CB
:10E30000C95CD1090FB6F894DEBF0FBECDBF6B96C6
:10E310008FAF6B9781E00F945C666B962FAD6B9718
:10E32000211125C01092130D1092120D19821A821C
:10E330001B821C82CE0101960F943F7661E080EC37
:10E340009FE00F94FAB560E08FEB9FE00F94FAB571
:10E3500060E08EEB9FE00F94FAB560E08DEB9FE0FC
:10E360000F94FAB560E08CEB9FE00F94FAB580E073
:10E370000E9407A80F946A4F0E945A9110920D0DA7
:10E3800010920C0D83E0EFE0FDE0DF011D928A9515
:10E39000E9F781E00F949E09C855DF4F9983888380
:10E3A000C85AD0408DE69CE10E94CDFB0F94CD0968
:10E3B00040E050E061E080E090E00F949D6640E036
:10E3C00050E061E081E090E00F949D66E0900710DE
:10E3D000F09008100091091010910A10209103107C
:10E3E0003091041040910510509106106091FF0F7C
:10E3F0007091001080910110909102100F94FB47D2
:10E400000E94D0DF1092250220E030E040EA50E484
:10E410006091FF0F70910010809101109091021097
:10E420000F9474B61B012C016093FF0F70930010C2
:10E43000809301109093021020E030E040EA50E415
:10E440006091031070910410809105109091061056
:10E450000F9474B69B01AC01609303107093041089
:10E460008093051090930610E0900710F09008102C
:10E470000091091010910A10AEE06A2EADE07A2EDC
:10E480007F926F92812C912CB0EAAB2EB1E4BB2E1F
:10E490008BE0C82E80E1D82EC201B1010F947634F2
:10E4A0000F942D830E94FEA749E85AE161E080E0C5
:10E4B0000E94F3A73090250281E080932502EEE2CE
:10E4C000FFE14490552441940CF4509484E00F945F
:10E4D000821D1092071010920810109209101092CD
:10E4E0000A102091031030910410409105105091B2
:10E4F00006106091FF0F70910010809101109091B3
:10E500000210E12CF12C87010F94FB470F94CD09E9
:10E51000E8E2FFE165917591859194912DEC3CECD9
:10E520004CE85FE30F947AAA6B017C01B201052CE1
:10E53000000C880B990B0F9413B19B01AC01C70120
:10E54000B6010F947AAA2091040D3091050D4091E7
:10E55000060D5091070D0F9474B67B018C016093EA
:10E56000040D7093050D8093060D9093070D80E0C8
:10E5700090E0A8E4B4E48093210290932202A09357
:10E580002302B09324022091000D3091010D40919F
:10E59000020D5091030D6091FC0C7091FD0C809167
:10E5A000FE0C9091FF0C7F926F92E5E58E2E982CD9
:10E5B000A82CE1E4BE2EF8E0CF2EFDE0DF2E0F9474
:10E5C00076340F942D830F94E71C1092250210923D
:10E5D0000710109208101092091010920A10209142
:10E5E0000310309104104091051050910610609175
:10E5F000FF0F709100108091011090910210E12C9A
:10E60000F12C87010F94FB470F94CD098AE0849D7C
:10E61000B001859D700D1124072E000C880B990BFD
:10E620000F9413B12091040D3091050D4091060D0A
:10E630005091070D0F9474B67B018C016093040D0B
:10E640007093050D8093060D9093070D80E090E088
:10E65000A8ECB3E48093210290932202A0932302BA
:10E66000B09324022091000D3091010D4091020DD4
:10E670005091030D6091FC0C7091FD0C8091FE0C8B
:10E680009091FF0C7F926F92A5E58A2E982CA5EDB4
:10E69000AA2EA0E4BA2E0F9476340F942D833092D4
:10E6A000250280E090E0A4E5B3E480930710909306
:10E6B0000810A0930910B0930A1020910310309114
:10E6C000041040910510509106106091FF0F709159
:10E6D00000108091011090910210E12CF12C04E5C2
:10E6E00013E40F94FB470F9492660F900F900F90D6
:10E6F0000F900F900F906B96BFAD6B97B11132C01A
:10E7000084E090E0909327028093260240E060E04E
:10E7100082E59CE10E94DAFB882321F08AE29CE1F9
:10E720000E947CFC80EF9BE10E947CFC8AE59BE1DF
:10E730000E947CFC82E090E0909327028093260266
:10E740008AE39BE10E94CDFB62E080E00E94C6A7C5
:10E7500061E070E080E090E00E94D8A984E39BE152
:10E760000E94F1A680E090E0A0EAB0E48093071058
:10E7700090930810A0930910B0930A10709025028E
:10E7800081E08093250284E00F94821DE0900710C1
:10E79000F09008100091091010910A1020910310B8
:10E7A0003091041040910510509106106091FF0FB8
:10E7B000709100108091011090910210EEE0FDE048
:10E7C000FF93EF93812C912CE0EAAE2EE1E4BE2E74
:10E7D000FBE0CF2EF0E1DF2E0F9476340F942D83E3
:10E7E0000F94E71C7092250282E00F941A830F9019
:10E7F0000F9020E030E040EA50E40F940DB1811119
:10E800000C944E866B96EFAD6B97EE23E9F0C855EE
:10E81000DF4F88819981C85AD0400F947D090E94AA
:10E8200049930E945C8F0E944C8D882311F40C94B4
:10E83000FE850F94540F803F11F00C944A8681E0BE
:10E840000F94280C0C944A868AEF0F94280C60E0F1
:10E8500070E088EF9FE00F9414B60F94926684ECFA
:10E86000E3E7F5E1DF011D928A95E9F7E4E1FFE1D5
:10E8700084918F01882339F00F94FC0F0F5F1F4F95
:10E88000F8018491F7CF61E070E080E090E00F94B0
:10E8900085100F943111BE016F5A7F4F8AE39BE1BF
:10E8A0000E94BBFB62968FAD6297843020F083E0BC
:10E8B00062968FAF629780E090E0A0EAB0E4809328
:10E8C000071090930810A0930910B0930A1024EF3A
:10E8D0003EE1C657DF4F39832883CA58D04082E7CC
:10E8E00095E1CE57DF4F99838883C258D0406C960C
:10E8F0009FAF8EAF6C97A8963FAF2EAFA89781E0E1
:10E9000090E0A0E0B0E0AE968CAF9DAFAEAFBFAFF1
:10E91000AE970F94926662966FAD629780E00E9408
:10E92000C6A7AE966CAD7DAD8EAD9FADAE970E9485
:10E93000D8A984E39BE10E94F1A665E575E585E52C
:10E9400091E40E94DE8CA896EEADFFADA89785916C
:10E950009591A591B4918093FF0F90930010A0938F
:10E960000110B0930210A896EEADFFADA8973496B3
:10E9700085919591A591B491809303109093041083
:10E98000A0930510B093061060E070E088E492E474
:10E990000E94DE8C0091F70F1091F80F2091F90F73
:10E9A0003091FA0F4091F30F5091F40F6091F50FF1
:10E9B0007091F60F8091EF0F9091F00FA091F10FF1
:10E9C000B091F20F3F932F931F930F937F936F9309
:10E9D0005F934F93BF93AF939F938F9380E89EE194
:10E9E0009F938F930F9418B00F942D834091EF0F46
:10E9F0005091F00F6091F10F7091F20F8091F30F31
:10EA00009091F40FA091F50FB091F60FC090F70F11
:10EA1000D090F80FE090F90FF090FA0F21E00FB6C8
:10EA2000F894DEBF0FBECDBF413157420CF420E059
:10EA30008131974214F00C945486822F90E0880F15
:10EA4000991FFC01E858F14EA590B490FC01E059E3
:10EA5000F14E85909490DF92CF929F928F92BF92C9
:10EA6000AF921F922F9387E59EE19F938F930F9410
:10EA700018B087E79CE19F938F930F9418B00F9481
:10EA8000192080916E008B7F80936E00EF988091AB
:10EA90006F008D7F80936F000FB6F894A8958091DA
:10EAA0006000886180936000109260000FBE109239
:10EAB000FB0C1092FA0C8CE991E09093F90C809386
:10EAC000F80C80EA91E09093F70C8093F60C00E04C
:10EAD00028EC30E0A601B401C5010F94B4290091DF
:10EAE000F70F1091F80F2091F90F3091FA0F409124
:10EAF000F30F5091F40F6091F50F7091F60F809124
:10EB0000EF0F9091F00FA091F10FB091F20F3F93A2
:10EB10002F931F930F937F936F935F934F93BF93A5
:10EB2000AF939F938F9387E19DE19F938F930F9472
:10EB300018B08091EF0F9091F00FA091F10FB0916C
:10EB4000F20F782E692E8091F30F9091F40FA0911F
:10EB5000F50FB091F60F582E492EC090F70FD090B8
:10EB6000F80FE090F90FF090FA0F0FB6F894DEBFAF
:10EB70000FBECDBF4EE8242E4CE1342E95E0C916D1
:10EB800097EFD9060CF46EC01A8219821F921F9259
:10EB9000A3E0AF93B4E8BF931F92E4E6EF93DF9254
:10EBA000CF924F925F926F927F923F922F920F94EB
:10EBB00018B00FB6F894DEBF0FBECDBF89819A8121
:10EBC000803D924030F089819A81803A954050F59D
:10EBD00012C0CE0101967C0100E010E024E833E091
:10EBE000A601652D742D872D962D0F943651811118
:10EBF0000C944587E8CFDE0111967D0100E010E01E
:10EC00002CE73CEFA60144565109652D742D872D44
:10EC1000962D0F943651882329F089819A8180534B
:10EC20009D4F1CC089819A818037984008F04AC066
:10EC3000FE0131967F0104EB10E024E833E0A601E9
:10EC4000485C5109652D742D872D962D0F943651F2
:10EC50008823C1F189819A8180569A4F9A8389834A
:10EC60000C9445870091F70F1091F80F2091F90F40
:10EC70003091FA0F4091F30F5091F40F6091F50F1E
:10EC80007091F60F8091EF0F9091F00FA091F10F1E
:10EC9000B091F20F3F932F931F930F937F936F9336
:10ECA0005F934F93BF93AF939F938F9386EC9CE1B9
:10ECB0009F938F930F9418B00FB6F894DEBF0FBEDA
:10ECC000CDBFD9C389819A8180349B40A0F49E0135
:10ECD0002F5F3F4F790104EB10E02CE73CEFA601DA
:10ECE0004C525140652D742D872D962D0F94365121
:10ECF00081110C94598680E0E981FA81882311F40E
:10ED00000C9461868091EF0F9091F00FA091F10F1C
:10ED1000B091F20F4091F30F5091F40F6091F50F05
:10ED20007091F60F0091F70F1091F80F2091F90FE5
:10ED30003091FA0FFF93EF931F930F935F934F93CD
:10ED40009F938F9383EF9CE19F938F930F9418B0C1
:10ED50004091F70F5091F80F6091F90F7091FA0FF1
:10ED600000E028EC30E0B401C5010F94B42985E03F
:10ED70008F9380E78F9387E29EE19F938F930F9409
:10ED800018B084E08F9388E38F9385E19EE19F9391
:10ED90008F930F9418B08091EF0F9091F00FA09186
:10EDA000F10FB091F20F6A968CAF9DAFAEAFBFAFCF
:10EDB0006A976896CEACDFAC68978091F30F90911C
:10EDC000F40FA091F50FB091F60FE2968CAF9DAFC6
:10EDD000AEAFBFAFE2978091F70F9091F80FA0917F
:10EDE000F90FB091FA0FA2968CAF9DAFAEAFBFAF47
:10EDF000A2971C0198E4291A310889E08F9380E6D4
:10EE00008F933F922F92E096AFADE097AF93AF967E
:10EE1000BFADAF97BF936896EFAD6897EF936796D6
:10EE2000FFAD6797FF9380E49DE19F938F930F94CD
:10EE300018B04091F70F5091F80F6091F90F709151
:10EE4000FA0F7A0120E931E0E0966EAD7FADE097F0
:10EE500068968EAD9FAD68970F94B429E0962EAD5D
:10EE60003FADE0973450EC963FAF2EAFEC970FB626
:10EE7000F894DEBF0FBECDBF812C912CD601B450CB
:10EE8000E896BFAFAEAFE897F601FC5FC258DF4F20
:10EE9000F983E883CE57D040382D3170A3963FAF29
:10EEA000A39780FC02C00C946786EF968FADEF9716
:10EEB000C158DF4F9881CF57D04000E020E931E0C2
:10EEC000A701EC966EAD7FADEC970F94B429C0907E
:10EED000F30FD090F40FE090F50FF090F60F8091C3
:10EEE000EF0F9091F00FA091F10FB091F20F01E0B0
:10EEF00028EC30E0A101B6010F94B429C090F30FC3
:10EF0000D090F40FE090F50FF090F60F8091EF0F96
:10EF10009091F00FA091F10FB091F20F0FEF28EC4C
:10EF200030E040E659E0B6010F94B4298091F70F24
:10EF30009091F80FA091F90FB091FA0F7C01A39670
:10EF40006FADA39780910B01662311F40C946F862B
:10EF5000816080930B010000840125E0000F111FE8
:10EF60002A95E1F7A3968FADA397882311F40C940B
:10EF7000728690EC492E55245A94652C752CC12C20
:10EF8000D12C90E4E3969FAFE397A12CB12C93B1E1
:10EF9000A70142195309292F207194FF02C00C9434
:10EFA000798688EE9FEF840F951F97FD02C00C9421
:10EFB0007D8680E090E0A80EB91E80910B012111A2
:10EFC0000C948786846080930B01000021110C94BF
:10EFD0008A862E143F0434F484E00E9416E0A1E0F7
:10EFE000EA1AF10881E00E9416E08BE599E00197AA
:10EFF000F1F7E396FFADE397F150E396FFAFE397A8
:10F00000F111C5CFB6E0B694A794BA95E1F7A396EF
:10F010002FADA397222311F40C9499868FE190E0F1
:10F020008C199D09800F911FFC01EA57F84FA082AF
:10F030008091EF0F9091F00FA091F10FB091F20F2E
:10F04000840D951DA61DB71D8093EF0F9093F00FB3
:10F05000A093F10FB093F20FC7010F2C000CAA0B75
:10F06000BB0B8093F70F9093F80FA093F90FB09319
:10F07000FA0F3FEFC31AD30A60E2C616D10409F0B3
:10F0800080CF0A57184FF0E2BF2EABE3CA2EADE196
:10F09000DA2ED8018D918D011F928F93DF92CF923E
:10F0A0000F9418B0BA940F900F900F900F90B1106A
:10F0B000F0CF89E39DE19F938F930F9418B0BFEF3A
:10F0C0008B1A9B0AEC96EEADFFADEC97E05CFF4F20
:10F0D000EC96FFAFEEAFEC970F900F90F0E28F162B
:10F0E000910409F0D9CEE6E8AE2EEBE0BE2E86EA1A
:10F0F0009BE0F501119211928E179F07D9F780E0DE
:10F1000090E0DC0175E0AA0FBB1F7A95E1F7AA57E2
:10F11000B84F40E0ED91F0E054E0F595E7955A9551
:10F12000E1F7EE0FFF1FEA57F44F208131812F5F87
:10F130003F4F318320834F5F403261F70196803229
:10F140009105F9F626E8C22E2BE0D22E00E010E061
:10F1500038E7E32E3DE1F32ED6018C9111969C9178
:10F16000B2E0CB0ED11C9F938F931F930F93FF920E
:10F17000EF920F9418B00F5F1F4F0F900F900F90EA
:10F180000F900F900F900031110531F78091880B8F
:10F190009091890BE8E8FBE031E021E04191519149
:10F1A0008417950710F4322FCA012F5F2031B1F771
:10F1B000032F1F923F939F938F938FE99DE19F931E
:10F1C0008F930F9418B0E4EAFBE00F900F900F902C
:10F1D0000F900F900F908EE0329122912A303105DE
:10F1E00010F40C949C868295807F2091860B309140
:10F1F000870B2037334010F00C94A386000F000FCC
:10F20000000F182F101B1F921F931F928F931F9296
:10F210000F9388E89DE19F938F930F9418B096E821
:10F22000492E97E0592E0FB6F894DEBF0FBECDBF22
:10F23000F201202F30E0012F10E0808190E02817AC
:10F24000390710F00C94A686821B930B982F80E050
:10F25000B8010F941EBB6F3F710519F010F06FEFEE
:10F2600070E06193AE16BF0641F700E010E0B3E82E
:10F27000AB2EBDE1BB2E81E8C82E8DE1D82EC80192
:10F28000A5E0880F991FAA95E1F7DC01AA57B84FAE
:10F290007D01912CF70181917F011F928F93BF9285
:10F2A000AF920F9418B093940F900F900F900F900F
:10F2B000F0E29F12EFCFDF92CF920F9418B00F5F62
:10F2C0001F4F0F900F9000321105C9F68DEF9DE191
:10F2D0002EED3BE0A6ECBBE0FC01459154914D9333
:10F2E0005D9302962A173B07B9F7612C712CE12C2C
:10F2F000F12C10E000E0A12C40E050E0EB964FAF85
:10F30000EB9726EC3BE0E8963FAF2EAFE897A0E006
:10F31000B0E080E090E0B12C4A01860C971C20E020
:10F3200030E014012A0E3B1E6EEF6B0DE3966FAFBB
:10F33000E397B1100C94AA866EEF620F683010F458
:10F340000C94B1862F5F3F4F2C30310591F7B39469
:10F350009096E896EEADFFADE8973296E896FFAF4F
:10F36000EEAFE897FCE0BF12DACFE816F9062CF40E
:10F370007C010A2DEB961FADEB974F5F5F4F443139
:10F38000510509F0BBCFA39420E2620E711C34E159
:10F39000A312B2CFFF92EF921F920F931F921F936F
:10F3A00083EB9DE19F938F930F9418B00FB6F89461
:10F3B000DEBF0FBECDBF93E4E916F10414F40C9444
:10F3C000E7861F920F931F921F9384EE9DE19F93F8
:10F3D0008F930F9418B01A5FE12EF12CA0E1EA1A76
:10F3E000F108E6E0EE0CFF1CEA95E1F76896EEAD59
:10F3F000FFAD6897EE0EFF1E0A5FC02ED12CF0E124
:10F40000CF1AD108F6E0CC0CDD1CFA95E1F7E096B6
:10F410002EAD3FADE097C20ED31EA0963FADA09794
:10F420003F936F966FAD6F976F93DF92CF92FF927E
:10F43000EF9283ED9DE19F938F930F9418B000E0BE
:10F4400028EC30E0A0964EAD5FADA097B601C701A5
:10F450000F94B4290FB6F894DEBF0FBECDBF81E084
:10F46000D2011D922D01B6EF4B16BCE05B06C1F731
:10F4700081110C94EA8610E080E49EE19F938F93C3
:10F480000F9418B00F94B44280916E008460809302
:10F490006E00EF9A80916F00826080936F0098E217
:10F4A00088E10FB6F894A895809360000FBE909302
:10F4B00060001092FB0C1092FA0C1092F90C109252
:10F4C000F80C1092F70C1092F60C0F900F9011237D
:10F4D00011F40C94878520E030E0A9016C96EEAD24
:10F4E000FFAD6C9761817281838194810F947AAAB8
:10F4F0002091FF0F309100104091011050910210A7
:10F500000F9474B66C96AEADBFAD6C9711966D93BB
:10F510007D938D939C931497C0900310D09004100A
:10F52000E0900510F090061020E030E0A90115965B
:10F530006D917D918D919C9118970F947AAAA70156
:10F5400096010F9474B66C96EEADFFAD6C97658323
:10F5500076838783908720E030E040E850ECC70155
:10F56000B6010F940DB187FF0CC080E090E0A0E8D9
:10F57000B0EC8093031090930410A0930510B09307
:10F58000061020E030E040E450E4609107107091F4
:10F5900008108091091090910A100F9474B660932E
:10F5A0000710709308108093091090930A10AE967C
:10F5B0008CAD9DADAEADBFADAE970196A11DB11D99
:10F5C000AE968CAF9DAFAEAFBFAFAE97A896AEADC7
:10F5D000BFADA8971896A896BFAFAEAFA8976C9688
:10F5E000EEADFFAD6C9738966C96FFAFEEAF6C97B3
:10F5F000AE968CAD9DADAEADBFADAE970597A105F6
:10F60000B10509F086C980E090E00E94BFA420E027
:10F6100030E040E950EC6091771570917815809159
:10F62000791590917A150F940DB187FF43C0E3EFE0
:10F63000FEE184918F01882339F00F94FC0F0F5F56
:10F640001F4FF8018491F7CF8AE00F94FC0FE1EC93
:10F65000FEE184918F01882339F00F94FC0F0F5F36
:10F660001F4FF8018491F7CF60917715709178154D
:10F670008091791590917A1542E00F949F10EDEBEF
:10F68000FEE184918F01882339F00F94FC0F0F5F06
:10F690001F4FF8018491F7CF42E060E070E080E90D
:10F6A00090EC0F949F100F943111F2E0AF96FFAFE2
:10F6B000AF9703C0AF961FAEAF971092A3151092ED
:10F6C000A4151092A5151092A6151092A7151092C8
:10F6D000A8151092A9151092AA1524E6EB962FAF43
:10F6E000EB976E961CAE1DAE1EAE1FAE6E976A9661
:10F6F0001CAE1DAE1EAE1FAE6A97CE01019664967B
:10F700009FAF8EAF6497DE01AF5BBF4F6696BFAF12
:10F71000AEAF66976A966CAD7DAD8EAD9FAD6A97C4
:10F720000F945FB7AA966CAF7DAF8EAF9FAFAA97CD
:10F730006A966CAD7DAD8EAD9FAD6A970F94EDB9B5
:10F74000C457DF4F688379838A839B83CC58D0402A
:10F750006E966CAD7DAD8EAD9FAD6E970F945FB71D
:10F76000C057DF4F688379838A839B83C059D04019
:10F770006E966CAD7DAD8EAD9FAD6E970F94EDB96D
:10F78000CC56DF4F688379838A839B83C459D040EA
:10F790006496EEADFFAD649720E411922A95E9F7E7
:10F7A0006696AEADBFAD6697E0E11D92EA95E9F7CA
:10F7B00080E090E00E94BFA48091A3159091A415D1
:10F7C000A091A515B091A615C655DF4F88839983E2
:10F7D000AA83BB83CA5AD0408091A7159091A815DF
:10F7E000A091A915B091AA15C255DF4F88839983BE
:10F7F000AA83BB83CE5AD040DE01AF5BBF4FC85651
:10F80000DF4FB983A883C859D040FE013196AC962A
:10F81000FFAFEEAFAC9700E0CC56DF4F8881998107
:10F82000AA81BB81C459D040B058E6968CAF9DAF39
:10F83000AEAFBFAFE697C057DF4F88819981AA81ED
:10F84000BB81C059D040B058EA968CAF9DAFAEAFE7
:10F85000BFAFEA97C457DF4F88819981AA81BB81E6
:10F86000CC58D040B058C258DF4F88839983AA83C0
:10F87000BB83CE57D040AC962EAC3FACAC9710E0DB
:10F8800062E7462E65E1562E74E0772EC12CD12C0E
:10F890007601013011F40C946887113011F40C9446
:10F8A0007487002311F1023081F4D20111962D9159
:10F8B0003D914D915C911497C258DF4F68817981D9
:10F8C0008A819B81CE57D0400BC0F20125813681C1
:10F8D00047815085EA966CAD7DAD8EAD9FADEA97C0
:10F8E0000F947AAA4B015C0106C0812C912C50E840
:10F8F000A52E5FE3B52E112301F1123081F4D20160
:10F9000011962D913D914D915C911497C258DF4F06
:10F91000688179818A819B81CE57D0400BC0F201EA
:10F920002581368147815085EA966CAD7DAD8EADDF
:10F930009FADEA970F947AAA04C060E070E080E877
:10F940009FE39B01AC01C501B4010F947AAA9B010E
:10F95000AC01C701B6010F9474B66B017C010023A2
:10F96000E1F11123D1F1023011F00C944887D2015A
:10F9700011962D913D914D915C911497AA966CAD85
:10F980007DAD8EAD9FADAA970F947AAA4B015C0115
:10F99000113011F40C946287123011F00C945587D9
:10F9A000D20111962D913D914D915C911497AA969B
:10F9B0006CAD7DAD8EAD9FADAA970F947AAA9B01D9
:10F9C000AC01C501B4010F947AAA9B01AC01C70137
:10F9D000B6010F9474B66B017C017A94F8E04F0E77
:10F9E000511C711056CFD101CD92DD92ED92FD9256
:10F9F0001D011F5F143009F043CF32E7232E35E19C
:10FA0000332EE4EFFEE1A096FFAFEEAFA097CA570A
:10FA1000DF4F1882C658D040C456DF4F1882CC59E9
:10FA2000D040C056DF4F1882C05AD04010E00023AB
:10FA300021F1013049F1023081F4D10111962D916B
:10FA40003D914D915C911497C258DF4F6881798147
:10FA50008A819B81CE57D0400BC0F1012581368130
:10FA600047815085EA966CAD7DAD8EAD9FADEA972E
:10FA70000F947AAA4B015C010AC0812C912C20E8DA
:10FA8000A22E2FE3B22E03C0812C912C5401D10160
:10FA900011964D905D906D907C901497A30192010A
:10FAA000AA966CAD7DAD8EAD9FADAA970F947AAA44
:10FAB0006B017C01D10115968D919D910D90BC91AA
:10FAC000A02DA6968CAF9DAFAEAFBFAFA697A09668
:10FAD000EEADFFADA09785919591A591B491CC55D0
:10FAE000DF4F88839983AA83BB83C45AD040A696EC
:10FAF0002CAD3DAD4EAD5FADA697CC56DF4F6881C6
:10FB000079818A819B81C459D0400F947AAA9B0144
:10FB1000AC01C701B6010F9473B6C655DF4F2881FB
:10FB200039814A815B81CA5AD0400F9474B6CC5552
:10FB3000DF4F288139814A815B81C45AD0400F94BC
:10FB400073B6A50194010F947AAACA57DF4F288192
:10FB5000C658D040C456DF4F3881CC59D040C0562B
:10FB6000DF4F4881C05AD040512F0F9474B6CA5706
:10FB7000DF4F688379838A839B83C658D0400023F4
:10FB8000A9F00130B9F00230D9F0A6962CAD3DAD08
:10FB90004EAD5FADA697E6966CAD7DAD8EAD9FADDB
:10FBA000E6970F947AAA6B017C010AC0C12CD12C74
:10FBB000760106C0C12CD12C90E8E92E9FE3F92EE6
:10FBC000A096EEADFFADA097349685909590A59048
:10FBD000B490A3019201C457DF4F688179818A8173
:10FBE0009B81CC58D0400F947AAA2B013C01A69659
:10FBF0002CAD3DAD4EAD5FADA697C057DF4F6881D0
:10FC000079818A819B81C059D0400F947AAA9B0147
:10FC1000AC01C301B2010F9474B6C255DF4F288105
:10FC200039814A815B81CE5AD0400F9474B6A501C8
:10FC300094010F9473B6A70196010F947AAACA573C
:10FC4000DF4F288139814A815B81C658D0400F94AB
:10FC500074B6CA57DF4F6883C658D040C456DF4FCA
:10FC60007883CC59D040C056DF4F8883C05AD040EB
:10FC7000192FA096AEADBFADA0971896A096BFAFB6
:10FC8000AEAFA097B8E02B0E311CE2E92E16E5E1ED
:10FC90003E0609F0CCCEDC01CB01B058C856DF4F90
:10FCA000E881F981C859D04081939193A193B19390
:10FCB000C856DF4FF983E883C859D0400F5FAC9630
:10FCC0002EAD3FADAC97205F3F4FAC963FAF2EAF10
:10FCD000AC97043009F0CFCD25968CAD9DADAEAD7F
:10FCE000BFAD2597AA968CAF9DAFAEAFBFAFAA9719
:10FCF0008D819E81AF81B885AE968CAF9DAFAEAF42
:10FD0000BFAFAE9789859A85AB85BC85A6968CAF2B
:10FD10009DAFAEAFBFAFA6978D859E85AF85B889E5
:10FD2000E6968CAF9DAFAEAFBFAFE69789819A8163
:10FD3000AB81BC81EA968CAF9DAFAEAFBFAFEA9707
:10FD400029968CAD9DADAEADBFAD2997C258DF4FA2
:10FD500088839983AA83BB83CE57D04089899A89A7
:10FD6000AB89BC89C457DF4F88839983AA83BB833F
:10FD7000CC58D040898D9A8DAB8DBC8DC057DF4F4C
:10FD800088839983AA83BB83C059D0408D8D9E8D73
:10FD9000AF8DB8A1CC56DF4F88839983AA83BB83EC
:10FDA000C459D0408D899E89AF89B88DC856DF4F20
:10FDB00088839983AA83BB83C859D0402D968CAD84
:10FDC0009DADAEADBFAD2D97CA57DF4F88839983E8
:10FDD000AA83BB83C658D04089A19AA1ABA1BCA17C
:10FDE000C456DF4F88839983AA83BB83CC59D04004
:10FDF0008DA19EA1AFA1B8A5C056DF4F888399837E
:10FE0000AA83BB83C05AD0408DA59EA5AFA5B8A933
:10FE1000CC55DF4F88839983AA83BB83C45AD040D3
:10FE200089A59AA5ABA5BCA5CE54DF4F888399833D
:10FE3000AA83BB83C25BD04061968CAD9DADAEAD55
:10FE4000BFAD6197CA54DF4F88839983AA83BB8370
:10FE5000C65BD04089A99AA9ABA9BCA9C654DF4FFB
:10FE600088839983AA83BB83CA5BD0408DA99EA94E
:10FE7000AFA9B8ADC254DF4F88839983AA83BB83EF
:10FE8000CE5BD04089AD9AADABADBCADCE53DF4FAC
:10FE900088839983AA83BB83C25CD04021968CADB2
:10FEA0009DADAEADBFAD2197CA53DF4F8883998317
:10FEB000AA83BB83C65CD04014E6C12CD12C76014A
:10FEC0004601570126013701A3019201AE966CADA0
:10FED0007DAD8EAD9FADAE970F947AAA9B01AC011C
:10FEE000AA966CAD7DAD8EAD9FADAA970F9473B6FB
:10FEF0002B013C01A5019401A6966CAD7DAD8EADA4
:10FF00009FADA6970F947AAA9B01AC01C301B201E1
:10FF10000F9473B62B013C01A7019601E6966CADD8
:10FF20007DAD8EAD9FADE6970F947AAA9B01AC0193
:10FF3000C301B2010F9473B6EA962CAD3DAD4EAD40
:10FF40005FADEA970F9462B7A2966CAF7DAF8EAFAC
:10FF50009FAFA297C457DF4F288139814A815B81C7
:10FF6000CC58D0400F947AAA9B01AC01C258DF4F05
:10FF7000688179818A819B81CE57D0400F9473B676
:10FF80002B013C01A5019401C057DF4F68817981A5
:10FF90008A819B81C059D0400F947AAA9B01AC0101
:10FFA000C301B2010F9473B64B015C01A701960126
:10FFB000CC56DF4F688179818A819B81C459D040BA
:10FFC0000F947AAA9B01AC01C501B4010F9473B6DA
:10FFD000C856DF4F288139814A815B81C859D0409A
:10FFE0000F9462B72B013C01C456DF4F2881398141
:10FFF0004A815B81CC59D040A2966CAD7DAD8EAD6F
:020000021000EC
:100000009FADA2970F947AAA9B01AC01CA57DF4F0C
:10001000688179818A819B81C658D0400F9473B6DC
:100020004B015C01C056DF4F288139814A815B81D9
:10003000C05AD040C301B2010F947AAA9B01AC010F
:10004000C501B4010F9473B64B015C01A701960181
:10005000CC55DF4F688179818A819B81C45AD04019
:100060000F947AAA9B01AC01C501B4010F9473B639
:10007000CE54DF4F288139814A815B81C25BD040F9
:100080000F9462B74B015C01C654DF4F2881398160
:100090004A815B81CA5BD040A2966CAD7DAD8EADCE
:1000A0009FADA2970F947AAA9B01AC01CA54DF4F6F
:1000B000688179818A819B81C65BD0400F9473B639
:1000C0006B017C01C254DF4F288139814A815B81F9
:1000D000CE5BD040C301B2010F947AAA9B01AC0160
:1000E000C701B6010F9473B66B017C01CE53DF4F8D
:1000F000288139814A815B81C25CD040C501B4014D
:100100000F947AAA9B01AC01C701B6010F9473B694
:10011000CA53DF4F288139814A815B81C65CD04058
:100120000F9462B76B017C01115009F0CDCEA296FD
:100130002CAD3DAD4EAD5FADA297C655DF4F68818A
:1001400079818A819B81CA5AD0400F9474B660939A
:10015000A3157093A4158093A5159093A615A301DC
:100160009201C255DF4F688179818A819B81CE5A85
:10017000D0400F9474B66093A7157093A815809320
:10018000A9159093AA15A50194016A966CAD7DAD51
:100190008EAD9FAD6A970F9474B66A966CAF7DAFC3
:1001A0008EAF9FAF6A97A70196016E966CAD7DAD3D
:1001B0008EAD9FAD6E970F9474B66E966CAF7DAF9B
:1001C0008EAF9FAF6E97EB969FADEB979150EB96EE
:1001D0009FAFEB9791119ECA6A966CAD7DAD8EADC7
:1001E0009FAD6A970F945FB76093931570939415C2
:1001F00080939515909396156A966CAD7DAD8EADF6
:100200009FAD6A970F94EDB9609397157093981509
:100210008093991590939A156E966CAD7DAD8EADC9
:100220009FAD6E970F94EDB9DC01CB01B058809370
:100230009B1590939C15A0939D15B0939E156E965B
:100240006CAD7DAD8EAD9FAD6E970F945FB7609333
:100250009F157093A0158093A1159093A2156A968F
:100260002CAD3DAD4EAD5FAD6A976E966CAD7DAD7C
:100270008EAD9FAD6E970F9473B66B017C01E894C1
:10028000F7F8B701A60180E69FE00F940CB62FE1C6
:1002900032E449E05BE3C701B6010F94BFB818161A
:1002A0006CF425E33AEF4EE85BE3C701B6010F9427
:1002B000BFB8181634F001E010E005C000E010E00F
:1002C00002C002E010E025E33AEF4EE85BE36A96F5
:1002D0006CAD7DAD8EAD9FAD6A979F770F94BFB823
:1002E00018167CF025E33AEF4EE85BE36E966CADB2
:1002F0007DAD8EAD9FAD6E979F770F94BFB81816EA
:1003000014F402E010E08091931590919415A0915F
:100310009515B0919615AE968CAF9DAFAEAFBFAFB1
:10032000AE9780919B1590919C15A0919D15B091D1
:100330009E15A6968CAF9DAFAEAFBFAFA69780912E
:10034000A3159091A415A091A515B091A615EE96B0
:100350008CAF9DAFAEAFBFAFEE97809197159091E8
:100360009815A0919915B0919A15E6968CAF9DAF0E
:10037000AEAFBFAFE69780919F159091A015A09169
:10038000A115B091A215EA968CAF9DAFAEAFBFAFED
:10039000EA978091A7159091A815A091A915B09101
:1003A000AA15C258DF4F88839983AA83BB83CE578F
:1003B000D040A4EFBEE1A096BFAFAEAFA09782E75A
:1003C000282E85E1382EF10181809280A380B480AF
:1003D00085819681A781B085AA968CAF9DAFAEAF7F
:1003E000BFAFAA97A096EEADFFADA097C590D590F0
:1003F000E590F490A5019401AE966CAD7DAD8EAD07
:100400009FADAE970F947AAA2B013C01AA962CAD12
:100410003DAD4EAD5FADAA97A6966CAD7DAD8EADF0
:100420009FADA6970F947AAA9B01AC01C301B201BC
:100430000F9474B6EE962CAD3DAD4EAD5FADEE971C
:100440000F9474B69B01AC01C701B6010F9473B64B
:100450006B017C01A096EEADFFADA0973496459060
:10046000559065907490E6962CAD3DAD4EAD5FAD68
:10047000E697C501B4010F947AAA4B015C01EA9694
:100480002CAD3DAD4EAD5FADEA97AA966CAD7DAD9E
:100490008EAD9FADAA970F947AAA9B01AC01C501BE
:1004A000B4010F9474B6C258DF4F288139814A8154
:1004B0005B81CE57D0400F9474B69B01AC01C30151
:1004C000B2010F9473B64B015C01A7019601C701FD
:1004D000B6010F947AAA6B017C01A5019401C501B4
:1004E000B4010F947AAA9B01AC01C701B6010F9425
:1004F00074B60F94F8B92DEC3CEC4CE45FE30F9428
:10050000BFB8181614F40EEF1FEFB8E02B0E311C15
:10051000A096EEADFFADA0973896A096FFAFEEAFD8
:10052000A09722E935E12215330509F04CCF0115DA
:10053000110509F07AC16E962CAD3DAD4EAD5FADA3
:100540006E976A966CAD7DAD8EAD9FAD6A970F9438
:1005500074B620E030E040E05FE30F947AAA6B01CC
:100560007C010F945FB72B013C016093931570934E
:1005700094158093951590939615C701B6010F9425
:10058000EDB96E966CAF7DAF8EAF9FAF6E976093F7
:100590009715709398158093991590939A15DC018F
:1005A000CB01B058AA968CAF9DAFAEAFBFAFAA97A4
:1005B00080939B1590939C15A0939D15B0939E15C9
:1005C00040929F155092A0156092A1157092A215AD
:1005D0001092A3151092A4151092A5151092A615AD
:1005E0001092A7151092A8151092A9151092AA158D
:1005F000A2961CAE1DAE1EAE1FAEA2976A961CAE92
:100600001DAE1EAE1FAE6A97CE57DF4FA881B981CF
:10061000C258D04011968D909D90AD90BC9014978B
:1006200015968D919D910D90BC91A02DAE968CAF9D
:100630009DAFAEAFBFAFAE97C657DF4FE881F98130
:10064000CA58D040C590D590E590F490A50194018A
:10065000C301B2010F947AAAA6966CAF7DAF8EAF9C
:100660009FAFA697AE962CAD3DAD4EAD5FADAE97AC
:10067000AA966CAD7DAD8EAD9FADAA970F947AAA68
:100680009B01AC01A6966CAD7DAD8EAD9FADA697DE
:100690000F9474B69B01AC01C701B6010F9473B6F9
:1006A0002091A3153091A4154091A5155091A61540
:1006B0000F9474B66B017C016093A3157093A4151D
:1006C0008093A5159093A61520E030E040E85FE305
:1006D0006A966CAD7DAD8EAD9FAD6A970F9474B682
:1006E0006A966CAF7DAF8EAF9FAF6A97C657DF4FEC
:1006F000E881F981CA58D040349685919591A591A9
:10070000B491A6968CAF9DAFAEAFBFAFA697A50133
:1007100094016E966CAD7DAD8EAD9FAD6E970F94CE
:100720007AAA4B015C01AE962CAD3DAD4EAD5FADEE
:10073000AE97C301B2010F947AAA9B01AC01C50127
:10074000B4010F9474B69B01AC01A6966CAD7DAD5F
:100750008EAD9FADA6970F9473B62091A7153091DB
:10076000A8154091A9155091AA150F9474B64B0184
:100770005C016093A7157093A8158093A9159093B9
:10078000AA1520E030E040E85FE3A2966CAD7DADB5
:100790008EAD9FADA2970F9474B6A2966CAF7DAF4D
:1007A0008EAF9FAFA297CE57DF4FA881B981C258B5
:1007B000D0401896CE57DF4FB983A883C258D04097
:1007C000C657DF4FE881F981CA58D0403896C657DE
:1007D000DF4FF983E883CA58D0402A163B0609F058
:1007E00013CF6A962CAD3DAD4EAD5FAD6A97C70194
:1007F000B6010F9462B76093A3157093A41580930C
:10080000A5159093A615A2962CAD3DAD4EAD5FAD4E
:10081000A297C501B4010F9462B76093A7157093B6
:10082000A8158093A9159093AA1580909315909080
:100830009415A0909515B090961540909F155090E6
:10084000A0156090A1157090A215809197159091B8
:100850009815A0919915B0919A156E968CAF9DAF91
:10086000AEAFBFAF6E9780919B1590919C15A091F4
:100870009D15B0919E156A968CAF9DAFAEAFBFAF80
:100880006A97A3019201C501B4010F947AAA6B0182
:100890007C016A962CAD3DAD4EAD5FAD6A976E960C
:1008A0006CAD7DAD8EAD9FAD6E970F947AAA9B0116
:1008B000AC01C701B6010F9473B66B017C019B01BB
:1008C000AC01C301B2010F9462B72B013C016A96DF
:1008D0006CAD7DAD8EAD9FAD6A979058A701960126
:1008E0000F9462B76A966CAF7DAF8EAF9FAF6A9779
:1008F0006E966CAD7DAD8EAD9FAD6E979058A70195
:1009000096010F9462B7CE57DF4F688379838A834D
:100910009B83C258D040A7019601C501B4010F9432
:1009200062B76B017C018090A3159090A415A090F4
:10093000A515B090A6158091A7159091A815A09126
:10094000A915B091AA156E968CAF9DAFAEAFBFAF93
:100950006E974092931550929415609295157092EF
:100960009615CE57DF4F88819981AA81BB81C258E5
:10097000D0408093971590939815A0939915B093B4
:100980009A156A968CAD9DADAEADBFAD6A9780935A
:100990009B1590939C15A0939D15B0939E15C092A6
:1009A0009F15D092A015E092A115F092A215C30157
:1009B000B2019058A50194010F947AAA2B013C0131
:1009C0006E962CAD3DAD4EAD5FAD6E976A966CAD3B
:1009D0007DAD8EAD9FAD6A970F947AAA9B01AC0155
:1009E000C301B2010F9473B66093A3157093A4155D
:1009F0008093A5159093A615CE57DF4F6881798116
:100A00008A819B81C258D0409058A50194010F94CF
:100A10007AAA4B015C016E962CAD3DAD4EAD5FAD3B
:100A20006E97C701B6010F947AAA9B01AC01C5016C
:100A3000B4010F9473B66093A7157093A8158093B3
:100A4000A9159093AA1580E090E00E94BFA417FD1D
:100A500053C043EA55E16BE975E183E995E10E94F2
:100A6000D78F4091A3155091A4156091A515709151
:100A7000A61585EE9FE00F940CB64091A7155091F6
:100A8000A8156091A9157091AA1589EE9FE00F94A1
:100A90000CB64091931550919415609195157091F5
:100AA00096158DED9FE00F940CB6409197155091DF
:100AB00098156091991570919A1581EE9FE00F94A9
:100AC0000CB640919B1550919C1560919D157091AD
:100AD0009E1585ED9FE00F940CB640919F155091A7
:100AE000A0156091A1157091A21589ED9FE00F945A
:100AF0000CB60E945C8F09C00E3F9FEF190729F4C6
:100B0000AF96AFADAF97A23049F038010BC0AF96AA
:100B10001FAEAF9766246A94762C04C0BEEF6B2E8E
:100B200077247A94C855DF4F88819981C85AD0407C
:100B30000F947D0980E090E0A0EAB0E48093071074
:100B400090930810A0930910B0930A1020910310FD
:100B50003091041040910510509106106091FF0FE4
:100B6000709100108091011090910210EEE0FDE074
:100B7000FF93EF93812C912CE0EAAE2EE1E4BE2EA0
:100B8000FBE0CF2EF0E1DF2EE12CF12C00EA10E4A7
:100B90000F9476340F942D830F900F9077FC20C024
:100BA00020E030E046E153E46091071070910810B6
:100BB0008091091090910A100F9474B660930710F9
:100BC000709308108093091090930A1065E575E5FD
:100BD00085E591E4F3D684E69AE10E947CFC5CD73B
:100BE00081E00E9407A882E00E9483A6BFEF6B16F7
:100BF0007B0631F487E29AE10E947CFC10E04BC056
:100C0000EEEF6E16EFEF7E0681F4AF96FFADAF9775
:100C1000FF2329F0F23031F080EE98E1EDCF85E648
:100C200099E1EACF85E299E1E7CFAF962FADAF9793
:100C3000211107C033E06316710498F085E699E14D
:100C400017C0AF966FADAF97623019F482EE99E19D
:100C500002C088E999E10E947CFC1614170454F341
:100C600009C0F301EE0FFF1FE952FD4F8081918112
:100C70000E947CFC6720609409F286EE0F94280C99
:100C80008FE59FE00F94E8B5813021F087E99AE184
:100C90000E947CFC11E00F94E71C2BC18FE29FE1C6
:100CA0000E947CFC10E025C183E0821B282F0C945D
:100CB0001D7529813A812059374F3A8329830C9435
:100CC0007C76F0E9CF1AF1E0DF0A0C94BE75E79666
:100CD0008FADE797E8969FADE8970C945D778E7F90
:100CE0000C94A97780E4482E512C612C712C0C9423
:100CF000BF7787E190E00C94D3778F3F910509F09F
:100D000014F40C94DB778FEF90E00C94DB778B7FFF
:100D10000C94E377B0E6EB16B9E0FB0614F00C9404
:100D2000F27784E00E9416E0EFEFEE1AFE0A0C94D0
:100D3000F277C6010C9412788150883011F00C942F
:100D4000EC780C94F37800E00C94017980E090E06A
:100D50000C942679EBE0BE1611F40C949C792223B6
:100D600011F02B3039F4E396FFADE397F83010F033
:100D70000C94A279B101620F731F6A57784FFB017F
:100D8000F081A396FFAFA397E896EEADFFADE8978D
:100D9000C080D18061E070E0022E02C0660F771F34
:100DA0000A94E2F76C217D21672B31F0A396FFAD09
:100DB000A397F13148F005C0A3966FADA3976131B9
:100DC00018F401960C94A27901970C94A27980E012
:100DD0000C94307A84EF91E00F94FA2A882311F46E
:100DE0000C943B7A14E0812C912C5401C12CD12C11
:100DF000760188EE93E00F94FA2A882311F40C947C
:100E00003B7A8091EF0F9091F00FA091F10FB0918C
:100E1000F20F092E000CAA0BBB0BC80ED91EEA1E3E
:100E2000FB1E8091F30F9091F40FA091F50FB091FC
:100E3000F60F092E000CAA0BBB0B880E991EAA1EDA
:100E4000BB1E1150B1F64090F70F5090F80F609014
:100E5000F90F7090FA0FC501B40122E096958795BD
:100E6000779567952A95D1F732E0F694E794D79471
:100E7000C7943A95D1F700E028EC30E0A201C60112
:100E80000F94B42911E00C943C7A81E00C947C76A8
:100E9000F2012581368147815085E6966CAD7DADA6
:100EA0008EAD9FADE6970C94C47CF201258136810E
:100EB00047815085E6966CAD7DAD8EAD9FADE697D2
:100EC0000C94DD7C60E070E080E89FE30C94DF7CB4
:100ED000112311F40C94ED7C812C912C40E8A42E6C
:100EE0004FE3B42E0C94C87C01110C94B37C0C9489
:100EF000ED7C81E00E9407A880E00F945C66812F62
:100F0000C753DF4F0FB6F894DEBF0FBECDBFDF91E2
:100F1000CF911F910F91FF90EF90DF90CF90BF90F6
:100F2000AF909F908F907F906F905F904F903F9089
:100F30002F900895CF93DF93EC018AED9FE00F94FB
:100F400038AF97FFFACF6AED7FE0CE010F94CFAFB5
:100F5000EC010F94588A6093D60F7093D70F80934B
:100F6000D80F9093D90FCE01DF91CF9108951F93A1
:100F7000CF93DF93C82FD62F172F6091B31980E03E
:100F80000E94C6A72C2F0C2E000C330B8091B51994
:100F900090E0A0E0B0E04091AF195091B01960919D
:100FA000B1197091B21984179507A607B70711F008
:100FB00080E201C08EE33F93CF931F93DF931F9294
:100FC0008F9381E69FE19F938F930E94DFA62DB7B9
:100FD0003EB7285F3F4F0FB6F8943EBF0FBE2DBF00
:100FE000DF91CF911F9108959F92AF92BF92CF92C0
:100FF000DF92EF92FF920F931F93CF93DF93CDB7C2
:10100000DEB765970FB6F894DEBF0FBECDBFF82EE2
:10101000E62ED72EC42EB52E862F972F0F94CAAE4C
:10102000982EA92E6AEE71E68E010F5F1F4FC80140
:101030000F94C3AE892D9A2D8031910514F08FE065
:1010400090E0F801E81BF90B1786BF92CF921F932F
:101050000F93DF92EF928F2D0F2C000C990B9F9323
:10106000FF928BE69FE19F938F930E94DFA60FB6BE
:10107000F894DEBF0FBECDBF65960FB6F894DEBF05
:101080000FBECDBFDF91CF911F910F91FF90EF90D9
:10109000DF90CF90BF90AF909F9008950F93E09115
:1010A000C719EE23B9F0E150E093C719F0E0CF0182
:1010B000880F991FE80FF91FEA5EF24F4281042E54
:1010C000000C550B660B770B00E021E080819181CD
:1010D0000E94ABA60F91089580919202882309F493
:1010E00048C08091921990919319A0919419B09150
:1010F00095194091AF195091B0196091B119709143
:10110000B219481759076A077B0744F48093AF194F
:101110009093B019A093B119B093B2198091961918
:1011200090919719A0919819B09199194091AF1980
:101130005091B0196091B1197091B2198417950747
:10114000A607B70744F48093AF199093B019A09302
:10115000B119B093B21961E080E00E94C6A7409136
:10116000AF195091B01960918E1970918F1980E26A
:101170003BDF8091AB0F82FF0BC0E0919019F091A3
:1011800091198091AF199091B0199183808386CF86
:101190000895CF938AEE9FE10E9424B8C82F813032
:1011A00011F40F9425608C2FCF910895CF92DF9288
:1011B000EF92FF92CF93DF93E091C6068E2FEE0F52
:1011C000990BAA0BBB0BFC013596EA31F10508F02F
:1011D00074C38827EE58FF4F8F4F0D9461BB8EEE7E
:1011E0009FE10E9424B8813019F40F94256002C059
:1011F00018162CF482EA92E29DDE8EEF5BC00F940B
:10120000588A613375478105910508F456C384E80F
:1012100092E20F9440B01092C6064FC3BADF181680
:101220000CF04BC388E492E09F938F9381E892E2A5
:101230009F938F938AED9FE09F938F930F94FCAFC2
:101240008DE792E277DE8DEF5AC0A3DF18160CF01F
:1012500034C386E492E09F938F938AE792E29F9350
:101260008F938AED9FE09F938F930F94FCAF0F9025
:101270000F900F900F900F900F90809146029091D9
:1012800047028335910574F41F9283E58F9385EFB0
:101290009FE19F938F930F9418B060E083E393E2F4
:1012A0000E9411A688E692E20F9440B084E692E292
:1012B00041DE8CEF8093C60600C36BDF18160CF07E
:1012C000FCC280E692E2F4CF64DF18160CF0F5C29F
:1012D00088E292E09F938F938BE592E29F938F93A6
:1012E0008AED9FE09F938F930F94FCAF8DE492E281
:1012F0000F9440B00E9406AF81E080936113809309
:10130000C6060F900F900F900F900F900F90D5C2C0
:10131000C0915313CC2309F409C18091220D81118E
:101320006CC0C43209F452C030F5C43109F445C070
:1013300088F4C131E1F130F4C03109F05CC089E4D6
:1013400092E258C0C231B1F1C33109F054C08DE30B
:1013500092E250C0C132A1F130F4C03209F04BC06A
:1013600085E392E247C0C23271F1C33209F043C053
:1013700089E292E23FC0C23591F178F4C03449F17C
:1013800028F4C033C1F581E292E234C0C03521F1C6
:10139000C13589F585E192E22DC0C43531F110F1F6
:1013A000C03631F1C13839F581E092E223C085E4DD
:1013B00092E220C081E492E21DC089E392E21AC069
:1013C00081E392E217C08DE292E214C085E292E2DC
:1013D00011C08DE192E20EC089E192E20BC081E181
:1013E00092E208C08DE092E205C089E092E202C07C
:1013F00085E092E29FDD8AE05DCF1092220D80EFC2
:101400008C0F853038F5D0E0609780916F02909115
:101410007002C817D90799F0DF93CF9383EF91E259
:101420009F938F930F9418B08FEE91E283DD83E04A
:101430008093C6060F900F900F900F9006C08BEE12
:1014400091E278DD83E08093C606D0937002C0936A
:101450006F0269C080EE8C0F853068F4D0E0A097F1
:10146000DF93CF938DED91E29F938F930F9418B0FC
:1014700089ED91E234C0C03379F464E670E080E035
:1014800090E00F9440898CEC91E29F938F930F949E
:1014900018B088EC91E241C0C03481F48BEB91E24A
:1014A0009F938F930F9418B087EB91E243DD86EF03
:1014B0009FEF9093700280936F0230C080EB8C0F8F
:1014C0008530B0F4D0E0C055D109DF93CF9389EADD
:1014D00091E29F938F930F9418B085EA91E22ADDF1
:1014E00083E08093C6060F900F900F900F901BC063
:1014F000C03649F488E991E29F938F930F9418B016
:1015000084E991E20AC0C13871F480E791E29F93C7
:101510008F930F9418B08CE691E20CDD83E08093FA
:10152000C6060F900F9010925313C7C1C09054136A
:10153000D0905513E0905613F090571384EFC80ED7
:1015400081E0D81EE11CF11C0F94588AC616D706FC
:10155000E806F90608F0B1C188E691E2EBDC82E02A
:10156000A9CE17DE18160CF064C088E292E09F93B3
:101570008F9383E691E29F938F938AED9FE09F93F1
:101580008F930F94FCAF0F900F900F900F900F90D0
:101590000F908091280281114AC0809166168111B6
:1015A00005C080913C07882309F441C08091140D47
:1015B0009091150D88359240D1F180913E0E8111A8
:1015C00036C08091FF0690910007981781F18091B5
:1015D000FF0690E027E530910007381789F0289F33
:1015E000F0011124EA57F84F4485558566857785C3
:1015F000452B462B472B09F09F5F8F5F8F70EBCFFA
:101600009923A9F080915602882389F00E94E7AFC0
:1016100083E591E20F9444768091E606882319F0E1
:1016200089E491E202C084E491E20F94447681E07F
:1016300041CEC090D60FD090D70FE090D80FF09049
:10164000D90F88EBC80E8BE0D81EE11CF11C0F945B
:10165000588AC616D706E806F90648F32EC181E473
:1016600090E20E9424B8813019F40F94256002C0E2
:101670001816C4F488E191E29F938F930F9418B0E9
:101680000F900F9080915602811102C00E9406AF08
:10169000C1E0C0934C13C09357020E94CEACC093DC
:1016A000C6060BC176DD1816C4F480914C1388234E
:1016B00051F010924C1388E091E29F938F930F9416
:1016C00018B00F900F908BEF90E29F938F930F9431
:1016D00018B081E0809352132EC085E490E20E94FE
:1016E00024B8813019F40F94256002C018161CF438
:1016F00081EE90E219C0C090D60FD090D70FE09045
:10170000D80FF090D90F20EEC20E23E9D21E24E0AC
:10171000E21EF11C0F94588AC616D706E806F90691
:1017200008F0CBC087EC90E29F938F930F9418B092
:101730001092521384E18093C6060F900F90BDC0A3
:1017400080915313843209F456C038F5843109F47A
:1017500049C090F4813109F43FC030F4803109F080
:101760007DC081E990E25BC08231C9F1833109F02B
:1017700075C085E890E253C08132B9F130F480320F
:1017800009F06CC08DE790E24AC0823289F1833261
:1017900009F064C081E790E242C08235A9F188F483
:1017A000803461F130F4803309F058C089E690E26A
:1017B00036C0803531F1813509F050C08DE590E2B9
:1017C0002EC0843539F118F1803639F1813809F0AD
:1017D00045C089E490E223C08DE890E220C089E80A
:1017E00090E21DC081E890E21AC089E790E217C03C
:1017F00085E790E214C08DE690E211C085E690E2A4
:101800000EC081E690E20BC089E590E208C085E554
:1018100090E205C081E590E202C08DE490E20E9472
:1018200024B8813059F40F94588A609354137093FC
:101830005513809356139093571302C0181674F4DF
:10184000809153131F928F938FEA90E29F938F930F
:101850000F9418B081E08093220D20C0C090D60F65
:10186000D090D70FE090D80FF090D90F88EEC80E27
:1018700083E0D81EE11CF11C0F94588AC616D706C7
:10188000E806F906D0F4809153131F928F9385E9EF
:1018900090E29F938F930F9418B081E08093C606D7
:1018A0000F900F900F900F9008C073DC18162CF457
:1018B00081E08093C60680935213DF91CF91FF9011
:1018C000EF90DF90CF90089510920D0D10920C0DB7
:1018D0000F94540F863E40F40E9431A36CE07DE0EB
:1018E00088EF9FE00C9438D208958F929F92AF9228
:1018F000BF92CF92DF92EF92FF920F931F93CF93FD
:10190000DF939B01AC01CFEFDFE0688579858A85A5
:101910009B850F9473B67B018C012C813D814E8198
:101920005F81688179818A819B81EEE0FDE0FF9390
:10193000EF93812C912CE0EAAE2EE1E4BE2EFBE089
:10194000CF2EF0E1DF2E0F9476340F942D830F907D
:101950000F90DF91CF911F910F91FF90EF90DF904B
:10196000CF90BF90AF909F908F900D943E4C609120
:101970000C0D70910D0D072E000C880B990B0F9418
:1019800013B120914F10309150104091511050914F
:1019900052100F9462B7A9DF10920D0D10920C0D2A
:1019A000089582E00F941A836093071070930810D3
:1019B0008093091090930A100D943E4C8F929F9241
:1019C000AF92BF92CF92DF92EF92FF920F931F934D
:1019D0004B015C01EFEFFFE0E084F18402851385A9
:1019E0002481358146815781608171818281938113
:1019F000EEE0FDE0FF93EF93EBE0CE2EE0E1DE2E94
:101A00000F9476340F900F901F910F91FF90EF90ED
:101A1000DF90CF90BF90AF909F908F900D942D83CB
:101A2000CF93DF930F949266CFEFDFE080E090E0FA
:101A3000A0EAB0E488879987AA87BB8765E575E542
:101A400085E591E4BBDF8DEC9CECACE4BEE38883E0
:101A50009983AA83BB8383E393E3A3E7B0EC8C83EE
:101A60009D83AE83BF8363E070E1CE010F94F90ADA
:101A700060E070E088E492E4A1DF8AE999E9A9E1F5
:101A8000BEE388879987AA87BB8765E575E585E505
:101A900091E4DF91CF9192CF2F923F924F925F923C
:101AA0006F927F928F929F92AF92BF92CF92DF926E
:101AB000EF92FF920F931F93CF93DF93CDB7DEB7D3
:101AC00027970FB6F894DEBF0FBECDBF2091250239
:101AD0002E83109225023091010F3F831092010F47
:101AE0001092000F0F949266BE016F5F7F4F83E0EC
:101AF00093E20E94BBFB8981843010F083E08983EC
:101B0000698180E00E94C6A761E070E080E090E01B
:101B10000E94D8A98DEF92E20E94F1A680E090E0A9
:101B2000A0EAB0E48093071090930810A0930910E6
:101B3000B0930A1065E575E585E591E43FDFE2EADB
:101B4000FFE185919591A591B4918093FF0F9093BA
:101B50000010A0930110B0930210E6EAFFE1859116
:101B60009591A591B4918093031090930410A09344
:101B70000510B093061063E070E18FEF9FE00F94C3
:101B8000F90A60E070E088E492E418DF80E1EFEFAA
:101B9000FFE0ACEFBCE001900D928A95E1F781E0A7
:101BA0008093250240E050E061E082E090E00F94F5
:101BB0009D668091110D811109C08091060186FFFB
:101BC00005C060E08DEA92E20E9411A61092250203
:101BD00060E070E080E291EC0F945313882389F366
:101BE0008091071090910810A0910910B0910A10EF
:101BF0008093731590937415A0937515B093761513
:101C00000AEA1FE132E0C32ED12CE12CF12C412C49
